:020000040000FA
:1000000000040020E508000079050000C508000094
:10001000830500008D05000097050000000000002A
:1000200000000000000000000000000009090000BE
:10003000A105000000000000AB050000B5050000B0
:10004000BF050000C9050000D3050000DD05000064
:10005000E7050000F1050000FB05000005060000B3
:100060000F06000019060000230600002D06000000
:1000700037060000410600004B0600005506000050
:100080005F06000069060000730600007D060000A0
:1000900087060000910600009B060000A5060000F0
:1000A000AF060000B9060000C3060000CD06000040
:1000B000D7060000E1060000EB060000F506000090
:1000C000FF06000009070000130700001D070000DD
:1000D00027070000310700003B070000450700002C
:1000E0004F07000059070000630700006D0700007C
:1000F00077070000810700008B07000095070000CC
:100100009F0700001FB500F003F88DE80F001FBD2A
:1001100000F0DEBB1FB56FF00100009040100390AF
:10012000029001904FF010208069000B420900F00E
:100130001F045DF822300120A04083434DF8223097
:10014000684600F044F91FBDF0B54FF6FF734FF459
:10015000B4751A466E1E11E0A94201D3344600E080
:100160000C46091B30F8027B641E3B441A44F9D14B
:100170009CB204EB134394B204EB12420029EBD17E
:1001800098B200EB134002EB124140EA0140F0BD8F
:10019000DD4992B00446D1E90001CDE91001FF220A
:1001A0004021684600F03AFB94E80F008DE80F000C
:1001B000684610A902E004C841F8042D8842FAD12B
:1001C00010216846FFF7C0FF1090AA208DF8440068
:1001D000FFF7A0FF00F0F2F84FF01024A069102202
:1001E0006946803000F001F9A069082210A900F0EA
:1001F000FCF800F0D7F84FF080510A6949690068AF
:100200004A43824201D8102070470020704710B541
:10021000D0E900214FF0805002EB8103026944696C
:100220006243934209D84FF01022536903EB8103D4
:100230000169406941438B4201D9092010BD5069D1
:10024000401C01D0002010BD0F2010BD70B501680A
:100250000446AE4D4FF01020062951D2DFE801F0E0
:10026000320318283B1DD4E90265646829463046EC
:1002700000F0CDF82A462146304600F0B6F8AA0034
:100280002146304600F09EFA002800D0032070BDC1
:1002900000F050FB4FF4805007E0201DFFF7ABFF4C
:1002A0000028F4D100F046FB60682860002070BD93
:1002B000241D94E80700920000F084FA0028F6D08C
:1002C0000E2070BD8069401C12D0201DFFF79FFFDB
:1002D0000028F6D109E08069401C09D0201DFFF7F5
:1002E0008AFF0028EDD1606820B12046FFF750FF5B
:1002F000042070BDFFF70EFF00F060F800F052F828
:10030000072070BD10B50C46182802D001200860E7
:1003100010BD2068FFF79AFF206010BD4FF0102439
:10032000A069401C05D0A569A66980353079AA2846
:1003300008D06069401C2DD060690068401C29D03D
:1003400060692CE010212846FFF7FEFE31688142EB
:100350001CD1A16901F18002C03105E030B108CAA9
:1003600051F8040D984201D1012000E000208A429A
:10037000F4D158B1286810B1042803D0FEE728460C
:1003800000F057F861496868086008E000F016F866
:1003900000F008F84FF480500168491C01D000F0CB
:1003A000A3FAFEE7BFF34F8F59480168594A01F499
:1003B000E06111430160BFF34F8FFEE74FF0102063
:1003C0008169491C02D0806900F0ADB87047524A7B
:1003D00001681160121D416811604F4A8168103236
:1003E0001160111DC068086070472DE9F041174683
:1003F0000D460646002406E03046296800F0A6F8BF
:10040000641C2D1D361DBC42F6D3BDE8F08170B5CD
:100410000C4605464FF4806608E0284600F083F855
:10042000B44205D3A4F5806405F58055002CF4D1C1
:1004300070BD4168044609B1012500E000254FF078
:1004400010267069A268920000F0BCF9C8B120467D
:1004500000F01AF89DB17669A56864684FF4002031
:1004600084420AD2854208D229463046FFF7CFFFA0
:100470002A4621463046FFF7B8FFFFF79FFFFFF7F8
:1004800091FFFFF747FEF8E72DE9FF414FF01024F9
:10049000616980680D0B01EB800000F6FF70010BB5
:1004A00000200090019002900246039068460123CC
:1004B0000BE0560902F01F0C50F8267003FA0CFCF2
:1004C00047EA0C0740F82670521CAA42F1D30AE012
:1004D0004A0901F01F0650F8225003FA06F6354388
:1004E00040F82250491C8029F2D3A169090B4A091E
:1004F00001F01F0150F822408B409C4340F82240FD
:10050000FFF765FFBDE8FF815809000000000020EB
:100510000CED00E00400FA050006004014480168F4
:100520000029FCD07047134A0221116010490B6862
:10053000002BFCD00F4B1B1D186008680028FCD056
:100540000020106008680028FCD07047094B10B5E7
:1005500001221A60064A1468002CFCD00160106861
:100560000028FCD00020186010680028FCD010BDC6
:1005700000E4014004E5014008208F49096809585A
:10058000084710208C4909680958084714208A49EF
:100590000968095808471820874909680958084711
:1005A0003020854909680958084738208249096878
:1005B000095808473C2080490968095808474020E5
:1005C0007D4909680958084744207B49096809584A
:1005D0000847482078490968095808474C20764957
:1005E000096809580847502073490968095808479D
:1005F0005420714909680958084758206E4909680C
:10060000095808475C206C49096809580847602068
:100610006949096809580847642067490968095801
:100620000847682064490968095808476C206249EE
:1006300009680958084770205F4909680958084740
:1006400074205D4909680958084778205A490968A3
:10065000095808477C2058490968095808478020EC
:1006600055490968095808478420534909680958B9
:100670000847882050490968095808478C204E4986
:1006800009680958084790204B49096809580847E4
:10069000942049490968095808479820464909683B
:1006A000095808479C204449096809580847A02070
:1006B0004149096809580847A4203F490968095871
:1006C0000847A8203C49096809580847AC203A491E
:1006D000096809580847B020374909680958084788
:1006E000B4203549096809580847B82032490968D3
:1006F00009580847BC203049096809580847C020F4
:100700002D49096809580847C4202B490968095828
:100710000847C8202849096809580847CC202649B5
:10072000096809580847D02023490968095808472B
:10073000D4202149096809580847D8201E4909686A
:1007400009580847DC201C49096809580847E02077
:100750001949096809580847E420174909680958E0
:100760000847E8201449096809580847EC2012494D
:10077000096809580847F0200F49096809580847CF
:10078000F4200D49096809580847F8200A49096802
:1007900009580847FC2008490968095808475FF4C8
:1007A0008070054909680958084700000348044952
:1007B000024A034B70470000000000206809000057
:1007C0006809000040EA010310B59B070FD1042A15
:1007D0000DD310C808C9121F9C42F8D020BA19BA0C
:1007E000884201D9012010BD4FF0FF3010BD1AB171
:1007F000D30703D0521C07E0002010BD10F8013BC6
:1008000011F8014B1B1B07D110F8013B11F8014BEC
:100810001B1B01D1921EF1D1184610BD02F0FF033F
:1008200043EA032242EA024200F005B870477047EB
:1008300070474FF000020429C0F0128010F0030C42
:1008400000F01B80CCF1040CBCF1020F18BF00F8C3
:10085000012BA8BF20F8022BA1EB0C0100F00DB872
:100860005FEAC17C24BF00F8012B00F8012B48BFD0
:1008700000F8012B70474FF0000200B51346944674
:100880009646203922BFA0E80C50A0E80C50B1F1E8
:100890002001BFF4F7AF090728BFA0E80C5048BFFC
:1008A0000CC05DF804EB890028BF40F8042B08BF9A
:1008B000704748BF20F8022B11F0804F18BF00F896
:1008C000012B7047014B1B68DB68184700000020B4
:1008D00009480A497047FFF7FBFFFFF713FC00BD0B
:1008E00020BFFDE7064B1847064A1060016881F3F8
:1008F0000888406800470000680900006809000097
:100900001D030000000000201EF0040F0CBFEFF3D9
:100910000881EFF30981886902380078182803D12B
:1009200000E00000074A1047074A12682C3212689C
:100930001047000000B5054B1B68054A9B589847B7
:1009400000BD000005030000000000205409000065
:1009500004000000001000000000000000FFFFFF86
:040960000090D00330
:10100000501200207DE501006D2F0000EDE401008D
:101010006D2F00006D2F00006D2F000000000000FC
:10102000000000000000000000000000D5E5010005
:101030006D2F0000000000006D2F00006D2F0000DC
:101040003DE6010043E601006D2F00006D2F00001A
:101050006D2F00006D2F00006D2F00006D2F000020
:1010600049E601006D2F00006D2F00004FE60100E2
:101070006D2F000055E601005BE6010061E601000E
:101080006D2F00006D2F00006D2F00006D2F0000F0
:101090006D2F00006D2F00006D2F00006D2F0000E0
:1010A00067E601006DE601006D2F00006D2F000066
:1010B0006D2F00006D2F00006D2F00006D2F0000C0
:1010C00073E601006D2F00006D2F00006D2F0000F2
:1010D0006D2F00006D2F00006D2F00006D2F0000A0
:1010E0006D2F00006D2F00006D2F00006D2F000090
:1010F0006D2F00006D2F00006D2F00006D2F000080
:101100006D2F00006D2F000000F002F81DF023FA93
:101110000AA090E8000C82448344AAF10107DA4552
:1011200001D11DF018FAAFF2090EBAE80F0013F062
:10113000010F18BFFB1A43F0010318476CDA0100D6
:101140008CDA01000A4410F8014B14F00F0508BFB7
:1011500010F8015B240908BF10F8014B6D1E05D083
:1011600010F8013B6D1E01F8013BF9D1641E03D05C
:10117000641E01F8015BFBD19142E4D3704700008B
:101180000023002400250026103A28BF78C1FBD890
:10119000520728BF30C148BF0B6070471FB500F031
:1011A0003DF88DE80F001FBD1EF0040F0CBFEFF3DC
:1011B0000880EFF30980014A10470000E79E000015
:1011C0008269034981614FF00100104470470000BB
:1011D000D511000001B41EB400B511F025FA01B418
:1011E0000198864601BC01B01EBD0000F0B4404627
:1011F000494652465B460FB402A0013001B506488D
:10120000004700BF01BC86460FBC80468946924617
:101210009B46F0BC70470000091100001DF098B912
:1012200070B51C4C054608202070A01C00F065F825
:101230005920A08029462046BDE8704007F026B816
:1012400010B507F02EF813490020891E087010BD54
:1012500070B50C460F49891E097829B1A0F16001CB
:10126000532906D3012011E0602802D043F2010087
:101270000CE020CC084E94E80E0006EB8000A0F5B0
:101280008050241FD0F8806E2846B047206070BD83
:10129000012070470A000020B8E6010010B504469E
:1012A0000021012000F03FF80021182000F03BF859
:1012B00000210B2000F037F80421192000F033F84A
:1012C00004210D2000F02FF804210E2000F02BF84F
:1012D00004210F2000F027F80421C84300F023F870
:1012E0000721162000F01FF80721152000F01BF839
:1012F0002046FFF795FF002010BD91210180704727
:10130000FFF79EBF10487047104A10B514680F4B86
:101310000F4A08331A60FFF79BFF0C48001D04605A
:1013200010BD704770474907090E002806DA00F023
:101330000F0000F1E02080F8141D704700F1E0205C
:1013400080F800147047000003F9004310050240C4
:101350000100000130B5FF4D044610280AD0112CC1
:1013600006D02846122C817806D0132C08D0FFDF37
:10137000AC7030BDFFDFFBE71129F9D0FFDFF7E7E5
:101380001129F5D0FFDFF3E770B506200DF016FD4B
:10139000044606200DF01AFD251A07200DF00EFD5B
:1013A000044607200DF012FDEA49201A2A18887811
:1013B00012280CD000231A4413280AD0002002441B
:1013C0000878022807D000201044C0B270BD012365
:1013D000F1E70120F3E70120F6E7DE4800B50079E8
:1013E000DC49420897B051F8050F89880CD01722C4
:1013F0008DF80020CDF80200ADF806100BA9684664
:101400000AF095FF17B000BD4022F1E702210DF070
:101410002ABD2DE9F04196B01D4690460E4607467E
:10142000FFF7F4FF04000BD02078222804D3A07F1C
:10143000C0F34010A84206D1082016B0BDE8F081E4
:1014400043F20200F9E745208DF80000ADF8027084
:101450003DB101208DF804008DF805608DF80680FF
:1014600002E000208DF804000BA968460AF05FFF37
:10147000A07F65F34510A0770020DEE730B5044675
:10148000A1F120000D460A284AD2DFE800F0050746
:101490000C1C2328353A3F44FFDF42E02078202807
:1014A0003FD1FFDF3DE0AB480178032939D0807898
:1014B000132836D02078242833D0252831D023286B
:1014C0002FD0FFDF2DE0207822282AD0232828D80B
:1014D000FFDF26E02078222823D0FFDF21E02078DC
:1014E00022281ED024281CD026281AD0272818D01D
:1014F000292816D0FFDF14E02078252811D0FFDF3F
:101500000FE0207825280CD0FFDF0AE0207825287E
:1015100007D0FFDF05E02078282802D0FFDF00E0B9
:10152000FFDF257030BD30B50B8840F67B444FF6A9
:10153000FF72022801D0934204D09D1FA54224D2FD
:10154000022802D04D88954203D04D88AD1FA54298
:101550001BD24C88A34218D88B88B3F5FA7F14D2DB
:10156000022802D0C888904205D0C88840F6774546
:101570000A38A84209D2C888904208D0944206D0BE
:101580005B1C6343B3EB800F01DB072030BD002001
:1015900030BD70B514460D46064611F0B3FA60B979
:1015A0000DB1A54201D90C2070BD002409E000BF97
:1015B00056F8240011F0A6FA08B1102070BD641C82
:1015C000E4B2AC42F4D3002070BDF0B50024059D18
:1015D00010B1A94203D851E009B90020F0BD09209B
:1015E000F0BD055D8DB107197E78112E3FD00FDC5F
:1015F0000A2E3CD2DFE806F03B1624242A2A2C2CA3
:101600003333025D72BB641CE4B28C42F9D3E4E76D
:101610001D2E2CDAA6F11206042E28D2DFE806F0E1
:1016200027271018022DDAD1BD781D70072D01D2A1
:101630006D0701D40A20F0BD157845F0010515E0CD
:10164000EE43F60707E0012D07D010E00620F0BDBD
:101650002E07A6F18056002EF5D06046F0BD157815
:10166000AE0701D50B20F0BD45F002051570055DF4
:10167000641C2C44E4B28C4202D9B0E74FF4485CBD
:101680008C42AED3A9E710B50278540809D00122E4
:1016900043F20223012C07D0022C0DD0032C13D1CE
:1016A0000FE00020087005E080790324B4EB901F60
:1016B0000AD10A70002010BD8079B2EB901F03D1CF
:1016C000F7E780798009F4D0184610BD214A917B54
:1016D00039B1D17B022908D0032908D043F2022076
:1016E00070470146101D01F082BB032100E001217B
:1016F00001700020704738B50C460546694601F078
:1017000076FB00280DD19DF80010207861F347008A
:10171000207055F8010FC4F80100A888A4F805004E
:10172000002038BD38B51378F0B102281CD00AA4C7
:101730006D46246800944C7905EB9414247864F386
:1017400047031370032814D003F0FE0010700868DC
:1017500004E00000C00100200302FF01C2F8010004
:101760008888A2F8050038BD23F0FE031370022814
:10177000E8D1D8B240F00100E8E730B50C4609786E
:1017800097B0222902D2082017B030BD28218DF849
:101790000010ADF80200132A03D03B2A01D0072025
:1017A000F2E78DF804200BA968460AF0C0FD050099
:1017B00003D121212046FFF761FE2846E4E700B56A
:1017C00097B023218DF80010ADF802001088ADF815
:1017D00004005088ADF80600D088ADF80A00908863
:1017E000ADF808000020ADF80C00ADF80E000BA914
:1017F00068460AF09CFD05E62DE9FF470220FA4EF7
:101800008DF804000027708AADF80600B84643F250
:1018100002094DE001A80DF090FA050006D0708A8B
:10182000A8B3A6F81280ADF806803FE0039CA07F25
:1018300001072DD504F124000090A28EBDF8080008
:10184000214604F1360301F0A6FF050005D04D4501
:101850002BD0112D3DD0FFDF3BE0A07F20F0080012
:10186000A077E07F810861F30000C10861F34100C7
:10187000E07794F8210000F01F0084F82000207821
:10188000282827D129212046FFF7F8FD22E015E07E
:1018900040070BD5BDF80800214604F10E02FFF702
:1018A0008EFF05000DD04D4510D100257F1CFFB2E5
:1018B00002200DF083FA401CB842ABD8052D12D09F
:1018C00008E0A07F20F00400A07703E0112D00D0F5
:1018D000FFDF0025BDF806007082052D05D02846E3
:1018E00004B0BDE8F087A6F812800020F8E72DE9E3
:1018F000F047040000D1FFDF2078BB4E20F00F003E
:10190000801C20F0F0007030207060680178091FA2
:101910001429E6D2DFE801F0F00A0B4FEF0B0CEFD1
:10192000EF36F00B0BF074F00B0BF0F0FFDFD8E7A5
:1019300087883846FFF76AFD050000D1FFDF607831
:10194000212140F008006070707C40F00400707449
:101950002846FFF793FD384607F0D0FA384603F0E3
:101960009AFF384605F025F83946022011F087F82D
:10197000A87F20F01000A877FFF73EFF0028B0D026
:10198000FFDFAEE785882846FFF740FD00B9FFDF9F
:1019900060688078012800D0FFDF60688179284680
:1019A00007F01CFC00289CD0617841F008016170B0
:1019B0006168C88095E786883046FFF727FD0500F7
:1019C00000D1FFDF6078314640F008006070606849
:1019D000C088288160680089688160684089A88122
:1019E000022011F04CF80020A875A87F00F0030039
:1019F00002289CD1FFF700FF002898D0FFDF70E796
:101A000080783C2803D0002502280AD000E0012578
:101A1000002720B13C2802D0022800D0FFDF17B1F8
:101A2000A0E00127F5E76078002D40F00800607025
:101A3000707C40F0080070747ED165680221B5F8B2
:101A40000480AD1C474638460DF004FA04460321D5
:101A500038460DF0FFF98246052138460DF0FAF9B7
:101A60008146042138460DF0F5F9074604B9FFDF39
:101A7000BAF1000F00D1FFDFB9F1000F00D1FFDF95
:101A800007B9FFDF22212046FFF7F8FC287901285B
:101A900033D00227A07F062167F30100A077288BAF
:101AA0002081688B6081A88BA08105F1120001F074
:101AB000D5F920B36879800700D5FFDF6979E07D2B
:101AC00061F34700E075D5F80600A0616889A0833E
:101AD000062105F10C0001F0C1F9D0B130794108BF
:101AE000607861F347006070D6F80500C4F8020022
:101AF000B6F8090016E042E046E00127CAE7E07DBB
:101B000020F0FE00801CE075D5F81200A061E88A84
:101B1000DDE7607820F0FE00801C6070E868C4F8A3
:101B20000200288AE0803148007884F82200A07FF3
:101B300000F00301404600E007E007F0D1F9012F73
:101B400003D0022F0ED0FFDFCBE63078032800D081
:101B5000FFDF0021084610F092FFBDE8F0470120AA
:101B600001F013B9B078132800D0FFDF002107205F
:101B700010F085FFBDE8F0471120FFF7EBBB2046D2
:101B8000BDE8F04702F0DAB8607840F00800607015
:101B9000A7E62DE9F047054600789146002702099F
:101BA000DFF844A00C463E46012A70D000214FF6D3
:101BB000FF70022A6CD0072A09D00A2A69D0FFDFF9
:101BC000A9F800600CB127806680002089E6D5F86E
:101BD00004C004F1080204F118089CF80060361FE4
:101BE000142E56D204E00000C00100201000002096
:101BF000DFE806F0984F4F454F4F0A4F4F3C5A4F82
:101C00004FC263FA4F4F50E811270926002C7CD0B1
:101C1000BCF80480A4F804806868807920729AF87F
:101C20001110404621F004018AF8111004210DF032
:101C30002CF9052140460DF028F9002140460DF011
:101C400024F9012140460DF020F9032140460DF012
:101C50001CF9022140460DF018F9062140460DF00E
:101C600014F9072140460DF010F9A9E701270926CC
:101C7000F4B3BCF80400A0806868807912E01227F1
:101C80001026BCF80400214601F0C9F898E7BFE02F
:101C9000E9E00EE11C27092654B3BCF80200A0803D
:101CA0006868007920728BE71B27092604B304209B
:101CB000207268684088A08082E79CF802003C2877
:101CC00026D0102718260CF1020C8CB1BCF80200AB
:101CD000A080BCF818006082BCF818002082BCF814
:101CE0001A00A082BCF81C00E0829CF8050000E00D
:101CF0000BE00CF10601FFF715FD9CF8040010B194
:101D00000120E07309E00220FBE7A9F800605CE72E
:101D10001B270926002CF8D021729AF8111021F007
:101D20000801B2E01D273726002CEED0A08069689C
:101D30000879491DFFF7F6FC686890F82B00A0753C
:101D40006868C0780428E07D13D020F00100E075B9
:101D500069681F22C97861F34200E0756968C97A31
:101D600061F3C700E075696840460C311CF0F6FA73
:101D700026E740F00100EAE71D273726002CC4D0F3
:101D8000A0806968481D0B7901461846FFF7CAFC18
:101D9000696804F10F0201F10C00CB7A0146184684
:101DA000FFF7C0FC6868807CA0756868C178E07D3A
:101DB00061F3420020F0F900E0751F2140461CF05D
:101DC00066FBFDE620271026002C9ED0A0806868C8
:101DD00004F10902407A20726968CB1C88781946A0
:101DE000FFF7A0FCECE6FFE704271026002C8CD0C0
:101DF000BCF80200A0806868808820816868C0887C
:101E0000608168680089A08168684089E081D7E6C0
:101E1000287A012803D0022814D0FFDFD0E61F273C
:101E20001026002CABD06888A08068892081A88902
:101E30006081E889A081288AE0819AF8111021F058
:101E4000200122E012271026688800F0E8FF002C0D
:101E500095D0687800F00700032889D19AF811100E
:101E600021F0020111E02A7A062A29D2DFE802F0E5
:101E70000310102121211B270926002CA5D0A080AA
:101E800021729AF8111021F001018AF8111097E6D9
:101E90001B270926002C98D0A080287A012806D07C
:101EA000032020729AF8111021F01001EDE70220B2
:101EB000F7E74A4621462846BDE8F04702F0B9B8A0
:101EC000FFDF7DE610B5F94896B08078132802D080
:101ED000082016B010BD22208DF800000BA968461E
:101EE0000AF025FA04460021072010F0C8FD20461C
:101EF000EFE700B5ED4897B08078122801D00820B0
:101F000079E41E208DF8000000208DF802008DF885
:101F100003000BA968460AF00AFA0028F0D1002154
:101F2000072010F0ACFD1120FFF714FA002062E446
:101F300000B5DE4897B00078012814D01B208DF83A
:101F4000000000208DF802000BA968460AF0EFF9A6
:101F5000002807D10021084610F091FD012000F073
:101F600014FF002047E4082045E42DE9F041CF4C60
:101F7000002740B102281DD0072842D0082800D0F1
:101F8000FFDFBDE8F081FFF7D3FF0028F9D106F0AD
:101F9000C2F80028F5D0017821F00F01891C21F04A
:101FA000F00120310170077206F095F8607C40F076
:101FB00001001DE08EB23046FFF728FA050000D17F
:101FC000FFDF28782128DCD006F0A5F890B1017851
:101FD00021F00F01891C21F0F00110310170022164
:101FE00001724680AF7506F076F8607C40F0020022
:101FF0006074C6E729463046BDE8F0411322FFF77A
:10200000BCBBA578122D03D0132D04D0FFDFB8E799
:10201000FFF76FFF01E0FFF755FF0028B1D106F091
:102020007AF80028ADD0017821F00F01891C21F049
:10203000F00120310170122D07D00221017206F04B
:102040004AF8607C40F01000D2E70121F6E72DE964
:10205000F04114460D00074600D1FFDF2878012823
:1020600003D0022821D0FFDF8BE73846FFF7CEF9F7
:10207000060000D1FFDF0220B075207820F00F00AD
:10208000801C20F0F00010302070607840F00800D4
:1020900060702868A0606868E060288920828348B2
:1020A000417C41F0200141746BE73846FFF7AEF9FF
:1020B000060000D1FFDF69884FF6FF70814209D129
:1020C000AA88824206D131463846BDE8F041132243
:1020D000FFF753BB814201D1A88898B1207820F046
:1020E0000F00801C20F0F00010302070607840F06D
:1020F000080060702868A0606868E0602889208215
:10210000002006E0782300223946022010F01AFC55
:102110000120B07535E770B5044696B00D46084607
:1021200010F0F0FC78BB00200121614E203C0C2C0B
:102130007AD2DFE804F0062950555E677360447E6A
:102140008A940021082010F073FC10B1112016B001
:1021500070BD24208DF80000D5F80200CDF80200F3
:10216000A8798DF806000BA968460AF0E0F804008B
:1021700073D1082300221146184610F0E3FB08280B
:102180006BD0FFDF69E003E0686810F0FDFC08B188
:102190001020DCE748208DF800002888ADF8020008
:1021A0006888ADF804000BA968460AF0C0F804007E
:1021B00053D1686888B3BDF8301001804DE04920E4
:1021C0008DF800002888ADF80200A87800F0010022
:1021D0008DF8040046E0286802F0CCF904463CE0A3
:1021E0004A2209E08DF802103CE000BF8DF80200A1
:1021F00038E0422200E052228DF800202A78D207EF
:10220000F4D0EFE738208DF800002888ADF8020000
:102210006888ADF8040025E006E015E0287828B1CC
:10222000A0F11B01E12902D3072416E01B20307026
:1022300012E04F208DF800000BA968460AF077F8ED
:1022400004000AD11B20307007E0FFF79DF808B1A9
:10225000082402E00AF050F80024204677E75020D6
:102260008DF800000BA968460AF061F8B6E730B5B2
:10227000054697B00C46084610F068FC10B11020D7
:1022800017B030BD203D0C2D2DD2DFE805F0062A19
:102290002A2A2C2C2A2C2A2A2A2A2088FFF7B6F848
:1022A00040B10078222808D20820E9E7C0010020C8
:1022B0001000002043F20200E2E725208DF8000024
:1022C0002088ADF802000BA968460AF030F8002813
:1022D000D6D1DDF83210C4F802109DF83610A17185
:1022E000CEE70620CCE70720CAE7FC487047FB4949
:1022F000091F08747047F948001F007C00F00100B6
:10230000704738B5F5481421001F1CF09EF80120D5
:1023100000F03BFD1120FFF71DF8F149FB20EF4CC9
:102320000870241F611D684605F0BFFF9DF800106E
:10233000207961F3470020F0010020710020A07394
:102340004FF46170A0810220E073FFF746F800B1FE
:10235000FFDF00F061FE01F0ACFC38BD10B50C46AB
:102360003E2120461CF071F8A07F20F00300A077EA
:10237000202020700020A07584F8230010BD704735
:102380007CB5054610F0BEFB08B110207CBDD34CD7
:10239000241F211D60680090A06801902846FFF767
:1023A000AAF90028F2D1FFF718F80028EED000991A
:1023B0006160BDF8041021819DF80610A1727CBDFA
:1023C00010B5044610F0C2FB08B1102010BDC3497F
:1023D0002246091F0879491D4008FFF7A3F900208C
:1023E00010BD2DE9F0479CB00D4604004FF00008E9
:1023F00011D00822FFF7CDF800281BD1002608E0F5
:1024000054F8260004A9FFF73EF9002812D1761CE3
:10241000F6B2AE42F4D32F460A2006AD0DF1440ABF
:102420008DF8180026465146284609F080FF20B155
:1024300043F203201CB0BDE8F0874046DFF89C82E1
:10244000A8F1040888F803002EB300244FF00B090C
:102450001DE000BF56F8240005A9FFF714F900B1EC
:10246000FFDF9DF81400A87056F8240050F8011FF3
:10247000C5F803108088A5F8070085F8009051463C
:10248000284609F054FF00B1FFDF641CE4B2BC42EF
:10249000E0D388F803700020CCE72DE9F0479EB028
:1024A0001546894604001ED00F4608222946FFF72C
:1024B00070F8002811D1002613E000BF54F8260060
:1024C00005A9103000F093FC002806D13FB157F861
:1024D000260010F017FB10B110201EB0ABE7761CE1
:1024E000F6B2AE42EAD30026A5F101081CE000BF17
:1024F00006F1010A0AF0FF0712E000BF54F82600B7
:10250000017C4A0854F827100B7CB2EB530F05D11D
:102510000622113011311BF0F5FEC0B17F1CFFB255
:10252000AF42EBD30AF0FF064645E1DBC8462F4633
:10253000342007AD0DF148098DF81C0026464946A8
:10254000284609F0F4FE28B143F20420C5E743F21F
:102550000520C2E796B300242CE000BF56F8240003
:10256000A91C103000F043FC00B1FFDF56F8240036
:10257000102250F8111FC5F803108088A5F8070035
:1025800056F8241005F109001BF0E8FEB8F1000F21
:1025900015D058F82410102205F119001BF0DEFEAA
:1025A000322028704946284609F0C1FE00B1FFDFFD
:1025B000641CE4B2BC42D1D3012206E004E005F180
:1025C000190001F0CBFFEBE700224946284600F056
:1025D00039FC002081E770B596B0044610F092FAFD
:1025E00018B9606810F0D9FA08B11020AFE560881A
:1025F0004AF2B811884206D8384D20786E462D1F11
:1026000018B1012804D00720A1E5FEF7E6FE1AE084
:102610006078022804D0032802D043F2022096E515
:10262000E87317208DF80000E97B0020CDF8020048
:10263000ADF80600022932D003292DD0FFDF0BA907
:10264000684609F074FE0028D0D1606801F079FF77
:10265000207870B101208DF80200F01C01F07EFF9F
:102660004C208DF800000BA9684609F060FE00B10F
:10267000FFDF6088A8B1A88180B2ADF802003020E9
:102680008DF800000BA9684609F051FE00B1FFDF8C
:102690002078A87300205AE58DF80700CFE7402086
:1026A000FAE74FF46170E6E710B5044610F04EFA11
:1026B00020B9606838B110F067FA08B1102010BD79
:1026C000606801F04BFF0548001F81896180C17B74
:1026D0006170807B2070002010BD0000C4010020CC
:1026E000100000202DE9F0419CB0054600208DF837
:1026F00064008DF860008DF830008DF868001E468B
:1027000014468846284610F048FA18B9204610F0BA
:1027100044FA10B110201CB033E455EA040018D07C
:102720001F270CAB19AA414628460097FEF74DFF1C
:102730000028F0D11AAB18AA314620460097FEF7C0
:1027400044FF0028E7D19DF86000C00703D00A20AD
:10275000E1E70720DFE701AF7DB11A208DF8040023
:102760008DF8068042462946F81C1BF0F7FD0DA99E
:1027700001A809F0DCFD0028CDD17CB120208DF826
:1027800004008DF8066032462146F81C1BF0E6FD79
:102790000DA901A809F0CBFD0028BCD1FF499DF887
:1027A000300048700020B6E72DE9F0439BB04FF0B1
:1027B0000008FBA104468DF83480D1E90001CDE981
:1027C0001901204610F09EF990B92078012803D114
:1027D000606810F097F958B9F04D4FF00109A87BE7
:1027E00050B1E87B022807D1606810F0D6F918B123
:1027F00010201BB0BDE8F0832878012801D0082004
:10280000F7E707200CF0E2FA18B9207848B1012860
:1028100007D000F0CEFA30B1687C10F00C0F08D170
:1028200003E01220E5E71320E3E7C10701D18007A9
:1028300001D51120DDE7608943F6E172A0F12001A6
:102840009142217807D301297ED100287CD1A1892A
:10285000002979D10FE0022901D0032901D1A02854
:1028600072D3012907D06978C90704D0A18900294A
:102870006AD0B42968D8217831B1012908D0022959
:1028800004D0032960D10AE0002609E0022607E00F
:1028900008B9A08908B1042609E0012607E003264B
:1028A000A87B50B1E87B022807D1606828B10DA948
:1028B0006068FEF7E8FE00289BD1207A30B101283D
:1028C00006D0022806D003286DD105E0002704E0D9
:1028D000012702E0022700E003270EB1022E0ED1ED
:1028E0006FB1E87880B36878800702D043F20120A6
:1028F0007FE7022E03D1022F55D0032F53D018208B
:102900008DF838006089ADF83A006089ADF83C0078
:102910008DF83E600DF13F00FEF7D8FE00B1FFDFFD
:102920009DF834008DF840002078012806D0A87B5F
:1029300068B1E87B02280AD1606840B1606850F84D
:10294000011FCDF8411000E02DE0808802E04046F4
:10295000CDF84180ADF845008DF84870A07BC0F3FC
:102960004002014662F35F01C0F3800041EA80004B
:1029700019A9085C8DF84700A8B169460EA809F0AE
:10298000D6FC0028B4D11B208DF838008DF83A9081
:1029900069460EA809F0CBFC0028A9D19DF80100DA
:1029A0001B2819D101E0072023E7052E09D2DFE813
:1029B00006F0030305050300032000E0022000F0F9
:1029C000E4F9012E0AD0A08940B10022830011460B
:1029D00010460FF0B7FF08B103200AE7002008E710
:1029E0002DE9FC4107460D460326084610F0D5F8B0
:1029F000002864D13846FEF709FD040005D0207890
:102A0000222805D20820BDE8FC8143F20200FAE743
:102A1000A07F00F0030C2DB129466046FEF783FD30
:102A20000600F0D15D48BCF1010F05D0BCF1020FEA
:102A300017D0FFDF3046E6E7A27D2946012A02D003
:102A4000407C800701D51120DDE729B9684600F0F8
:102A5000F0FB0028D7D16946384606F042FB06460F
:102A6000E8E7A17D022914D1407C800611D425B16C
:102A7000A07F40070BD4002100E00121384606F07A
:102A800078FB0600D6D1A075002DD3D002E0112628
:102A9000D0E7A5B12A4621463846FEF790FE064605
:102AA0001128C7D1A07F4107C4D4296844F80E1F5C
:102AB0006968616040F0040020740026BAE71020C5
:102AC000A1E770B50C460546FEF7A0FC010005D055
:102AD00022462846BDE87040FEF74FBE43F2020092
:102AE00070BD00B597B03F218DF800108DF8020041
:102AF0000BA9684609F01BFC17B000BD0123FEF7C7
:102B000088BC00231A461946FEF783BC30B597B03F
:102B100004460FF0F7FF10B1102017B030BD20466B
:102B200000F053F90028F8D11C4DA878112801D0E5
:102B30000820F2E700F03DF920B1687CC00603D51B
:102B40001120EAE71320E8E72078800701D5E8782C
:102B500018B31D208DF800002078022200F001003B
:102B60008DF802006088ADF80400A088ADF806007A
:102B70002078C0F3400102EA500001438DF80910AB
:102B800002A8FEF7A3FD00B1FFDF0BA9684609F01C
:102B9000CEFB0028C1D11E2006E01DE0C0010020B0
:102BA00007060504030201008DF8000001208DF8DE
:102BB000020000208DF803000BA9684609F0B7FB5E
:102BC0000028AAD1E08800F01CF90400A5D1122049
:102BD000FEF7C0FB2046A0E707209EE7F0B597B0C0
:102BE00015460C4607460FF0D8FF38B920460FF0BF
:102BF00089FF18B928460FF085FF10B1102017B0D3
:102C0000F0BD9E4E707C10F0180F01D1400701D529
:102C10001120F4E7204600F0D8F80028EFD129462B
:102C20000220FEF780FC0028E9D1B078112803D0FB
:102C3000122801D00820E2E72078C0F34001394390
:102C400011D0800700D577B906200CF0BFF840B14D
:102C50002078800701D5F07828B1B078122804D008
:102C600007E01220CBE70720C9E7FFF742F9002869
:102C7000C5D100F09EF8022801D21320BFE7212021
:102C80008DF800006088ADF80200A088ADF804005F
:102C90002078C0F340008DF806002078800716D415
:102CA0003878420808D0012A18D043F20221022ABB
:102CB00018D0032A18D115E0C00700D002208DF8E3
:102CC000070057F8010F0290B888ADF80C000DF11D
:102CD0000E00FEF7FBFC58B1032090E7C00705D0BB
:102CE0000320ECE7C00701D0084688E70120E6E7AB
:102CF0002888ADF810006888ADF81200A888ADF8F3
:102D00001400E888ADF816000020ADF81800ADF802
:102D10001A000BA9684609F00AFB00288BD1E0884D
:102D200000F06FF8040086D11320FEF713FB204655
:102D300065E730B5054697B00C4608460FF006FF2C
:102D400008B11020E9E62846FEF760FB38B10178AB
:102D5000222902D3807F800604D40820DDE643F2D6
:102D60000200DAE613208DF80000ADF802500BA93E
:102D7000684609F0DCFA0028E4D19DF932107F2979
:102D800001D02170C9E60520C7E630B53B4D0400EF
:102D900008D0012C04D0022C06D0032C04D0FFDF75
:102DA0002C7030BDFFDFFBE728780128F8D0FFDF6B
:102DB000F6E710B50DF027FE04460FF0FDF9241AD2
:102DC000FEF7E2FA201AC0B286E4418843F6FD73AA
:102DD0000A1F9A4209D28088042806D3B0F5804F92
:102DE00003D8884201D80020704707207047027836
:102DF000520804D0012A02D043F202207047FEF7A5
:102E000042BC10B548B183000022114607200FF0E4
:102E100099FD072801D003205EE400205CE470B532
:102E20000C0006460DD0FEF7F1FA050000D1FFDFD9
:102E3000A68028892081288960816889A081A88945
:102E4000E08170BD10B502F0010282703122027083
:102E500009F06DFA002800D0FFDF3DE410B5002333
:102E60001A4603E0845C2343521CD2B28A42F9D34F
:102E70000BB1002030E401202EE40000C00100204E
:102E80004FF0E0224FF400410020C2F880112049A9
:102E90000870204990020860704730B51C4D044608
:102EA0002878A04218BF002C02D0002818BFFFDFEE
:102EB0002878A04208BF30BD2C701749154A002061
:102EC000ECB1164DDFF858C0131F012C0DD0022CA9
:102ED0001CBFFFDF30BD086003200860CCF8005045
:102EE0004FF400001060186030BD086002200860D8
:102EF000CCF800504FF040701060186030BD086092
:102F000008604FF06070106030BD00B5FFDF00BD9D
:102F10001A00002008F5014000F5004028030020B9
:102F200014F50040094810B504680A4908480860CB
:102F30000EF0A3FA0848046010BD0849002008609C
:102F40004FF0E0210220C1F88002704710050240D6
:102F5000010000011805024014050240FC1F00405A
:102F60000F4A12680D498A420CD118470C4A126860
:102F70000A4B9A4206D101B50FF048FB06F0A9FFB3
:102F8000BDE801400749096809580847064807494C
:102F9000054A064B7047000000000000BEBAFECA9A
:102FA0009C0000200400002050120020501200203D
:102FB00018B1172802D20720704717200849088047
:102FC0000020704706480088704770B50C460546DB
:102FD00007F007FC21462846BDE8704008F002BD16
:102FE0004600002070477047704770477047704731
:102FF0007047704770470021016081807047010071
:1030000018FFFFFFDBE5B15100F001009100FFFF69
:1030100084000000A8CA2D00FE4800210160416024
:1030200070472DE9F743044692B091460120FFF71F
:103030005EF960680FF0A8FD58B160680FF0ADFD53
:1030400038B9607800F00300022802D10020FFF7B1
:103050004EF94D4648460FF055FD18B1102015B0F9
:10306000BDE8F08329460120FEF75DFA0028F6D17D
:1030700001258DF842504FF4C050ADF840000022B9
:1030800010A9284603F039FF0028E8D18DF84250F6
:103090004FF42850ADF8400000261C2168460796E2
:1030A0001BF0F5F99DF81C0007AF20F00F00401C45
:1030B00020F0F00010308DF81C0020788DF81D00F5
:1030C00061789DF81E000DF1400861F3420040F068
:1030D00001008DF81E009DF8000008AA40F00200D3
:1030E0008DF800002089ADF83000ADF832606089BD
:1030F000ADF834000B9760680E900AA9CDF82880CF
:10310000684603F0F9FC0028A9D1C24CBDF82000A4
:1031100008AA20808DF8425042F60120ADF8400008
:103120009DF81E000AA920F00600801C20F0010076
:103130008DF81E000220ADF83000ADF8340013A861
:103140000E90684603F0D8FC002888D1BDF8200016
:103150006080211D484600F032F9002887D18DF8A3
:10316000425042F6A620ADF840001C216846079662
:103170001BF08DF99DF81C00ADF8345020F00F00C5
:10318000401C20F0F00010308DF81C009DF81D0050
:1031900008AA20F0FF008DF81D009DF81E000AA966
:1031A00020F0060040F00100801C8DF81E009DF804
:1031B00000008DF8445040F002008DF80000CDE989
:1031C0000A8711A80E90ADF83050684603F094FCC1
:1031D000002899D1BDF82000E08000203FE73EB5EF
:1031E00004460820ADF8000020460FF08BFC08B123
:1031F00010203EBD21460120FEF795F90028F8D1A8
:103200002088ADF804006088ADF80600A088ADF80D
:103210000800E088ADF80A007E4801AB6A46808865
:10322000002104F065F8BDF800100829E1D0032062
:103230003EBD1FB50446002002900820ADF80800EE
:10324000CDF80CD020460FF05DFC10B1102004B07A
:1032500010BD704802AA81884FF6FF7004F02DFA65
:103260000028F4D1BDF80810082901D00320EEE7AA
:10327000BDF800102180BDF802106180BDF8041077
:10328000A180BDF80610E180E1E701B582B002201F
:10329000ADF800005F4802AB6A464088002104F0A8
:1032A00027F8BDF80010022900D003200EBD1CB580
:1032B000002100910221ADF8001001900FF046FCB2
:1032C00008B110201CBD53486A4641884FF6FF7074
:1032D00004F0F3F9BDF800100229F3D003201CBD5F
:1032E000FEB514460E460746FFF705F828B13046EE
:1032F0000FF008FC18B11020FEBD0F20FEBDF82C09
:1033000001D90C20FEBD38460FF0FCFB414D18BB27
:10331000288801A903F05FF90028F3D138788DF8E7
:103320000500288801A903F0C5FF0028EAD1009014
:103330009DF800009DF8051040F002008DF8000097
:10334000090703D040F008008DF80000288869467E
:1033500003F04EFF0028D5D1ADF808402888334649
:1033600002AA002103F0C4FFBDF80810A142C9D091
:103370000320FEBD7CB50546002000900190088822
:10338000ADF800000C46284601950FF0FDFB18B97A
:1033900020460FF0DBFB08B110207CBD15B1BDF855
:1033A000000050B11B486A4601884FF6FF7004F0D8
:1033B00084F9BDF8001021807CBD0C207CBD30B5A7
:1033C00093B0044600200D460090142101A81BF084
:1033D0005EF81C2108A81BF05AF89DF80000CDF8F3
:1033E00008D020F00F00401C20F0F00010308DF8C5
:1033F00000009DF8010020F0FF008DF801009DF80D
:10340000200040F002008DF8200001208DF84600D9
:1034100002E000001200002042F60420ADF8440053
:1034200011A801902088ADF83C006088ADF83E00FE
:10343000A088ADF84000E088ADF842009DF8020099
:1034400006AA20F00600801C20F001008DF8020082
:103450000820ADF80C00ADF810000FA8059001A9E8
:1034600008A803F049FB002803D1BDF81800288004
:10347000002013B030BD000010B504460FF042FB31
:1034800008B1102010BD2078C0F30210042807D81E
:103490006078072804D3A178102901D8814201D28D
:1034A000072010BDE078410706D421794A0703D4EC
:1034B000000701D4080701D5062010BD002010BD6B
:1034C00010B513785C08C37F64F30003C3771478E6
:1034D000A40864F34103C3771078C309887863F3C1
:1034E0004100887013781C094B7864F347134B70C4
:1034F0001378DB0863F3000088705078487110BDC2
:1035000010B5C4780B7864F300030B70C4786408BA
:1035100064F341030B70C478A40864F382030B7056
:10352000C478E40864F3C3030B700379117863F380
:103530000001117003795B0863F341011170037995
:103540009B0863F3820111700079C00860F3C30126
:10355000117010BD70B514460D46064604F0DBFD33
:1035600080B10178142221F00F01891C21F0F001B3
:10357000A03100F8081B21461AF035FFBDE8704065
:1035800004F0A9BD29463046BDE870401322FEF77D
:10359000F4B870B514460E46054604F0BCFD70B193
:1035A000017821F00F01891C21F0F0012031017018
:1035B000458021688160BDE8704004F08CBD3146D3
:1035C0002846BDE870401322FEF7D7B810B5FE4C70
:1035D00094F8300000280CD104F120014FF6FF725E
:1035E000A1F110000DF085F800B1FFDF012084F893
:1035F000300010BD2DE9F047064608A8894690E83E
:1036000030041F469046142128461AF040FF00213E
:10361000CAF80010B8F1000F03D0B9F1000F03D1C0
:1036200014E03878C00711D020680FF08FFAE8BB9B
:10363000B8F1000F07D120681230286020681430DC
:1036400068602068A8602168CAF800103878800790
:1036500028D560680FF098FA40BBB9F1000F2DD063
:10366000FEF743FE0168C6F8B4118188A6F8B811C8
:10367000807986F8BA01FFF7A9FFDFF84C8308F1DB
:103680002008C5F80C80626862B196F8B40106F2B1
:10369000B51140081032FEF745F810224146606827
:1036A0001AF05CFE3878400712D500E003E0A0680D
:1036B0000FF04CFA50B11020BDE8F0876068002888
:1036C000F9D0E8606068C6F8B001EBE7A06828614F
:1036D0000020F1E730B5054608780C4620F00F00D1
:1036E000401C20F0F001103121700020607095F82E
:1036F000230030B104280FD0052811D0062814D09B
:10370000FFDF20780121B1EB101F04D295F82000D3
:1037100000F01F00607030BD21F0F000203002E0AA
:1037200021F0F00030302070EBE721F0F000403065
:10373000F9E710B510B190F8A94044B1A24890F84B
:10374000354000205CB108601060186010BD00F1C9
:10375000A8040C6000F1D001F8301160F5E79A4C34
:1037600034340C60F0E700B58BB00723CDE90212CA
:103770008DF801300191944900236431059109933A
:1037800001468DF8103068460CF08BFF002800D001
:10379000FFDF0BB000BD30B597B00C462C251A9951
:1037A0008DF80050ADF80200B3B118680190586868
:1037B0000290ADF80C2010220DF10E001AF0CEFD93
:1037C0000BA9684608F0B3FD002803D1A17F41F0A2
:1037D0001001A17717B030BD00200190E8E72DE976
:1037E000F0470646008A8CB080B20D468146FDF750
:1037F0000DFE0446744F3078283FDFF8CC814FF03F
:10380000000A122873D2DFE800F072E93509367732
:103810007E98A8F3E7E6E5E4E35BE3E3A07F00F04E
:103820000300012806D0002148460BF01CFB0500D0
:1038300003D101E00121F7E7FFDF98F85C100906EA
:1038400002D5D8F860000BE0032105F121000EF04D
:1038500005FED5F821005D49B0FBF1F201FB120035
:10386000C5F8210070686866B068A86620782528C9
:1038700000D0FFDFECE0A07F00F00300012806D0BD
:10388000002148460BF0EFFA060003D101E00121C8
:10389000F7E7FFDF7078810702D52178252904D06A
:1038A00040F0010070700CB006E70220287096F816
:1038B0002000287106F121003136C5E90206F2E741
:1038C000A07F00F00300012806D0002148460BF03D
:1038D000CAFA040003D101E00121F7E7FFDF6078B5
:1038E000C10605D51320287041346C60DBE7DEE1AA
:1038F00040F008006070D6E73348082128380EF001
:10390000ADFD032016E02A208DF8000010220DF1F5
:10391000020071681AF022FD10220DF11200B16848
:103920001AF01CFD284968462C3908F000FD00B14A
:10393000FFDF042028706F60B5E7E07FC00600D588
:10394000FFDFB0680090B38806220321484605F0E7
:103950002EFB0028A7D0FFDFA5E704B9FFDF7168C1
:1039600021B1102204F124001AF0F8FC282120468D
:10397000FDF784FDA07F00F0030002280ED104F1C2
:103980002400002300901A4621464846FFF703FF13
:10399000112807D029212046FDF770FD307A84F8E0
:1039A000200080E7A07F000700D5FFDF14F81E0F7E
:1039B00040F008002070A4F816A0C4F818A0C4F8BD
:1039C0001CA0617808460AE02002002040420F0057
:1039D00030E068E196E08CE062E009E03FE061F30E
:1039E0008200410861F3C3006070307AE0705AE7EA
:1039F000A07F00F00300012806D0002148460BF00C
:103A000032FA040003D101E00121F7E7FFDF0221D0
:103A100004F175000EF022FD1020287004F5DA7014
:103A20006860B4F875002882FA486C346C61C5E9A6
:103A3000028038E7A07F00F00300012805D00021B4
:103A400048460BF010FA18B901E00121F8E7FFDF52
:103A50000CB0324621464846BDE8F0477AE504B945
:103A6000FFDF207821289CD93079012802D0022854
:103A70000AD103E0E07F40F01000E07798F85C1096
:103A800041F0010188F85C10324621464846FFF7B4
:103A900061FD0CB02046BDE8F0472321FDF7EEBCE8
:103AA000327901230321484605F090F878B11120BE
:103AB0002870327905F10800AA80031D00900321C7
:103AC000484605F000F9002891D0FFDFEBE6A07F23
:103AD00000F00300012806D0002148460BF0C3F98E
:103AE000040003D101E00121F7E7FFDF3079207006
:103AF000D9E60321484605F007FC002899D1122099
:103B00002870D0E6A07F00F00300012806D0002135
:103B100048460BF0A8F9050003D101E00121F7E7C1
:103B2000FFDF95F8740000F00300012878D1A07F32
:103B300000F00307E07FC0F3400616B1012F04D068
:103B40002BE095F89000C0072AD0D5F8AC1119B336
:103B500095F87320087C62F387000874E27FD5F83B
:103B6000AC1162F341000874D5F8AC1166F30000A3
:103B70000874AEB1D5F8AC01102204F124017835F7
:103B80001AF0ECFB287E40F001002876287820F01F
:103B9000010005F8780900E016B1022F04D02CE0EE
:103BA00095F87800C00726D0D5F8A81119B395F874
:103BB0007320087C62F387000874E27FD5F8A811AF
:103BC00062F341000874D5F8A81166F30000087488
:103BD0008EB1D5F8A801102204F1240178351AF02D
:103BE000BDFB287840F0010005F8180B287820F07C
:103BF000010005F89009022F51D0002000EB400091
:103C000005EBC00090F87800800709D595F86C00A6
:103C1000D5F8B021400805F16D011032FDF782FDA5
:103C2000052060F3070815F8740F00F0030060F337
:103C30000F28287960F31748287F60F31F687548BC
:103C40005C38027822F00F02921C22F0F00220323F
:103C50000270427822F00702D21C4270A0F8029053
:103C6000C0F8088004F0C1FB2078252805D0212861
:103C700007D0FFDF2078222803D922212046FDF734
:103C8000FDFBA07F00F0030001280AD00021484678
:103C90000BF0FBF800283FF412AEFFDF03E6012033
:103CA000ACE70121F3E7716881F801A0FBE5FFDFD4
:103CB000F9E570B5574C0025103C14F85C0F20F066
:103CC0008000207065600CF0B4FC5249A1F1100036
:103CD00004F01DFB04F82C5C062060724D487C301B
:103CE00020615030A0611030E06170BD70B50D46AC
:103CF000FDF78CFB040000D1FFDF4FF4DE71284696
:103D00001AF0C5FB43485430686104F1240028616F
:103D1000A07F00F00300012808D0022105F5907073
:103D20000CF088FC002800D0FFDF70BD0121F5E712
:103D30000A46014602F590700CF09CBC70B5054631
:103D400040689CB0017808290DD00B2903D00C29BC
:103D500036D101218171686886883046FDF756FBAF
:103D6000040035D133E046883046FDF74FFB0400B0
:103D700000D1FFDF2078212822D0282822D16868AE
:103D800002210C3001F0B8F9E0B168680821001D8B
:103D900001F0B2F9B0B12D208DF80000ADF802604D
:103DA000102204F1240101A81AF0D8FA0BA96846E0
:103DB00008F0BDFA00B1FFDF29212046FDF75EFBC8
:103DC0001CB070BD687840F008006870F8E7FFDF4D
:103DD000A07F00F00301022902D120F01000A0779B
:103DE000207821280AD06868817909B1807898B153
:103DF000A07F00F0030002285BD0FFDFA07F00F06F
:103E000003000228DCD1FDF7F7FC0028D8D0FFDF43
:103E1000D6E7000030020020687840F008006870A3
:103E2000E07FC10720D0800701D5062000E00520F3
:103E300084F823002078292818D02428DED13146A0
:103E400006200EF01CFE22212046FDF717FBA07F66
:103E500000F0030001282AD0002130460BF015F8AD
:103E60000028CBD0FFDFC9E70420E1E7A07F00F006
:103E70000300012806D0002130460AF0F4FF0500B7
:103E800003D101E00121F7E7FFDF25212046FDF7FF
:103E9000F5FA0F208DF8580016A905F590700CF072
:103EA000E0FB0228AAD00028A8D0FFDFA6E7012166
:103EB000D3E7687840F0080068709FE72DE9F04389
:103EC0008BB09946154688460646FDF79FFA0400D2
:103ED0004ED0207822284BD3232849D0E07FC0063B
:103EE00046D4A07F00F00300012806D00021304610
:103EF0000AF0B9FF070002D00BE00121F7E7A07F2D
:103F000000F00300012804D1012130460AF0A2FF8D
:103F1000074601AB02AA03A93846FFF70AFC03983B
:103F200000B9FFDF4FB1039807F5907787612078DC
:103F3000222806D0242804D007E0039900208861B5
:103F400003E025212046FDF799FA03980B214170E3
:103F500046628580C0E90289029901610199416147
:103F600004A90CF09EFB022802D0002800D0FFDF3D
:103F70000BB0BDE8F08330B587B00546FDF746FAD3
:103F8000017822292FD9807F00F00300012806D074
:103F9000002128460AF067FF040003D101E0012157
:103FA000F7E7FFDF227801230321284604F00EFE05
:103FB000002818D011208DF80400227803A8009062
:103FC000ADF8082004AB0321284604F07CFE00B1C4
:103FD000FFDF01A904F590700CF043FB022802D02A
:103FE000002800D0FFDF07B030BD10B586B0044612
:103FF000FDF70CFA0178222919D9807F00F003001F
:10400000012806D0002120460AF02DFF040003D12C
:1040100001E00121F7E7FFDF12208DF8000069467B
:1040200004F590700CF01DFB002800D0FFDF06B0F7
:1040300010BD2DE9F05F05460C460027007890463C
:1040400001093E46BB4604F1080A02297ED0072931
:1040500002D00A2909D142E068680178082905D010
:104060000B292CD00C292AD0FFDFC6E114271C26EF
:10407000002C6CD04088A080FDF7C8F95FEA0009E9
:1040800000D1FFDF99F817005246400809F11801E6
:10409000FDF748FB68688089208268684168C4F839
:1040A00012108068C4F81600A07E20F0060040F0D0
:1040B0000100A07699F81E0040F040014DE01A275B
:1040C0000A26002CD5D08088A080FDF79FF9050036
:1040D00000D1FFDF51462846FFF7FCFA8DE10CB115
:1040E000288BA080287A0E287ED006DC01287CD080
:1040F000022808D0032804D135E0102876D01128F2
:1041000075D0FFDF79E11E270926002CB1D0A088E9
:10411000FDF77CF95FEA000900D1FFDF287B00F0A2
:1041200003000128207A1BD020F001002072297B97
:10413000890861F341002072297BC90861F382007C
:104140002072297B090961F3C30001E04AE117E10C
:10415000207299F81E0040F0800189F81E104CE191
:1041600040F00100E2E713270D26002CAAD0A0881A
:10417000FDF74CF98146807F00F00300012806D04E
:104180000021A0880AF06FFE050003D101E00121A3
:10419000F7E7FFDF99F81E0000F00302012A59D06B
:1041A000A86E817801F003010129217A54D021F011
:1041B0000101217283789B0863F3410121728378A6
:1041C000DB0863F38201217283781B0963F3C30167
:1041D0002172037863F306112172437863F3C711E8
:1041E000217284F809B003E05EE0A4E08CE09CE07A
:1041F000C178A172012A32D04279E17A62F30001DA
:10420000E1724279520862F34101E1724279920807
:1042100062F38201E1724279D20862F3C301E17272
:104220000279217B62F3000121730279520862F363
:10423000410121730279920862F3820121730079AE
:10424000C00860F3C301217399F8000023285AD9EC
:10425000262168E0686EA4E741F00101A9E7027930
:10426000E17A62F30001E1720279520862F34101DE
:10427000E1720279920862F38201E1720279D20856
:1042800062F3C301E1724279217B62F30001217381
:104290004279520862F3410121734279920862F334
:1042A000820121734079CBE718271026002C67D0B4
:1042B000A088FDF7ABF88246807F00F0030001285C
:1042C00007D00021A0880AF0CEFD5FEA000903D1E3
:1042D00001E00121F6E7FFDFE868A06099F801003E
:1042E00040F0040189F8011099F80200800708D510
:1042F000012020739AF8000023287ED927215046F8
:1043000063E084F80CB078E015270F26C4B3A088CA
:10431000FDF77CF8814606225146E86808F06FF800
:104320000120A073AEE048464FE0162709263CB3B3
:10433000287B207261E0297BFE4802290CD01927D6
:104340000E26ECB101290DD003291AD004291BD067
:10435000052919D0FFDF23E01B270926BCB3012163
:10436000217205E001212172617A21F0030161725D
:1043700010F85C1F4A08520062F3060101700FE05A
:104380002BE00220207207E0687B052900F00F0077
:1043900040F0800020721BD0607A20F00300607231
:1043A000A088FDF733F805460078212825D023287A
:1043B00000D0FFDFA87F00F00300012810D000210B
:1043C000A0880AF062FD22212846FDF757F814E084
:1043D000607A20F00300401CE1E7A8F8006011E0DB
:1043E0000121EDE70CB16888A080287A03282BD042
:1043F00004280AD005284BD0FFDFA8F800600CB1D4
:10440000278066800020BDE8F09F15270F26002C2E
:10441000E3D0A088FCF7FAFF807F00F003000128BA
:1044200006D00021A0880AF01EFD050003D101E09E
:104430000121F7E7FFDFD5F821000622514607F0FA
:10444000DEFF84F80EB0D8E717270926002CC4D069
:10445000A088FCF7DBFF8146807F00F00300012885
:1044600006D00021A0880AF0FEFC050003D101E07F
:104470000121F7E7FFDFA878800701D5022000E0DF
:104480000120207299F800002328B6D927214AE795
:1044900019270E26002CA0D0A088FCF7B7FF5FEAF2
:1044A000000900D1FFDFC4F808B0A4F80CB084F80C
:1044B00008B0A07A40F00300A07299F81F1061F3D1
:1044C0008200A07299F81F1001EA510161F3C30044
:1044D000A072687A00F0030001288ED1607A40F063
:1044E0000400607299F81E00E97A00F003000128C8
:1044F00013D0607B61F300006073AA7A217B62F3C2
:1045000000012173EA7A520862F341006073A87ACD
:10451000400860F3410121736FE7207B61F30000E5
:104520002073AA7A617B62F300016173EA7A520810
:1045300062F341002073A87A400860F3410161737F
:104540005BE710B57B4C30B10146102204F120002E
:1045500019F004FF012084F8300010BD10B50446A6
:10456000FFF734F8734920461022BDE8104020318F
:1045700019F0F4BE70B56F4C06004FF0000514D072
:104580000EF0C0FA08B110250DE00621304607F004
:104590001DFF411C06D0206614F85C0F40F080001F
:1045A000207000E00725284670BD14F85C0F20F04D
:1045B0008000F5E7007810F00F0204D0012A05D042
:1045C000022A0CD110E0000909D10AE000090128F3
:1045D00007D0022805D0032803D0042801D00720E3
:1045E00070470870002070470620704705282AD2BF
:1045F000DFE800F003070F171F00087820F0FF0026
:104600001EE0087820F00F00401C20F0F000103071
:1046100016E0087820F00F00401C20F0F000203059
:104620000EE0087820F00F00401C20F0F000303041
:1046300006E0087820F00F00401C20F0F000403029
:10464000087000207047072070472DE9F041804630
:1046500088B00D46002708460EF09FFAA8B94046DC
:10466000FCF7D4FE040003D02078222815D104E002
:1046700043F2020008B0BDE8F08145B9A07F010611
:1046800003D500F00300022801D01020F2E7A07F3C
:10469000C10601D4010702D50DB10820EAE725497A
:1046A00091F85C10C90701D01120E3E7E17FC9064A
:1046B00001D50D20DEE700F00300022805D125B169
:1046C0002846FEF7D9FE0700D4D1A07F00F00300F2
:1046D000012806D0002140460AF0C5FB060002D0A2
:1046E0000CE00121F7E7A07F00F0030001280BD0C8
:1046F000002140460AF0AEFB060007D0A07F00F084
:104700000300022804D009E00121F2E70420B1E708
:1047100025B12A4631462046FEF7D2FE07AB1A469F
:1047200069463046FFF705F8009800B9FFDF0C2016
:10473000009901E020020020487006F59070C1F851
:104740002480486100200881A07F00F00300012838
:1047500028D0EDB302200871301D886170784009BF
:104760000877B078C0F340004877287800F001025D
:10477000887F62F301008877E27F62F382008877A6
:10478000E27F520862F3C3008877B27862F30410C4
:104790008877A878C87701F1210228462031FEF7F2
:1047A000AFFE22E001200871287800F00102087EA7
:1047B00062F3010008762A78520862F382000876D4
:1047C0002A78920862F3C30008762A78D20800E0BB
:1047D00007E062F30410087624212046FCF74EFE21
:1047E0000BE0032008710520087625212046FCF700
:1047F00045FEA07F20F08000A07701A900980BF073
:1048000050FF022801D000B1FFDF384632E72DE922
:10481000FF4FF94A0D4699B09A4607CA14AB0027D4
:1048200083E807001998FCF7F1FD060006D0307800
:10483000262806D008201DB0BDE8F08F43F2020004
:10484000F9E7B07F00F00309B9F1010F03D0B9F126
:10485000020F07D008E03DB91B98FEF70DFE0028B7
:10486000E9D101E01B9878BBB07F00F0030001287C
:1048700006D0002119980AF0F6FA040003D101E0ED
:104880000121F7E7FFDF852D25D007DCD5B1812D8C
:104890001BD0822D1BD0832D08D11AE0862D1CD071
:1048A000882D1CD0892D1CD08A2D1CD00F20207162
:1048B0000F281AD001208DF83400201D0E90207989
:1048C000A8B158E10020F2E70FE00120EFE7022055
:1048D000EDE70320EBE70520E9E70620E7E70820FE
:1048E000E5E70920E3E70A20E1E70720A3E7B9F1BC
:1048F000010F17D0D4E91950804602200190012001
:104900000090A87898F80210C0F3C000C1F3C0016D
:1049100008405FEA000B5DD050460EF0F3F8002827
:104920006CD12DE0D4E9198501200190022000907E
:10493000214630461B9AFEF7C3FD1B98007800F015
:104940000101A87861F30100A870F17F61F3820092
:10495000A870F17F490861F3C300A870A17861F3E2
:104960000410A870607840092870A078C0F3400057
:1049700068701B988078E870002068712871C0E723
:10498000DAF80C000EF0BEF8C0BBDAF81C000EF02E
:10499000B9F898BBDAF80C00A060DAF81C00E06007
:1049A00098F80100A17800F0010041EA4000A070F1
:1049B00098F80210C0B2C1F30011891E0840A0701F
:1049C000002084F82000009906F1170002290BD07E
:1049D00001210AE098F80110A07801F00101FD2200
:1049E00042EA41010840E2E7002104EB81018861CD
:1049F0000199701C022902D0012101E028E0002168
:104A000004EB81018861A87800F00300012849D1F6
:104A100098F8020000F00300012843D1B9F1010F1A
:104A200004D12A1D691D1B98FEF76AFD297998F8A3
:104A3000040001408DF82C10687998F8052010408A
:104A40008DF8300001432DD050460EF05BF808B1D0
:104A50001020F0E60AF1100004F5D47104F17C0294
:104A60000490B9F1020F3CD00090CDE90121002162
:104A70000BAB5A462046FEF7BDFD0028E9D104F5F0
:104A8000D67104F19402B9F1010F30D0049800906E
:104A9000CDE9012100210CAB5A462046FEF7AAFDC4
:104AA0000028D6D1A078800740D4A87898F80210C2
:104AB000C0F38000C1F38001084337D0297898F80B
:104AC000000014AAB9F1010F17D032F810204B00E2
:104AD000DA4012F0030718D0012F1ED0022F12D196
:104AE0001DE0CDF800A0CDE901210121C0E7CDF8FE
:104AF00000A0CDE901210121CDE732F811204300CA
:104B0000DA4002F00307032F07D0BBF1000F0DD0EE
:104B1000012906D0042904D008E00227F5E701277F
:104B2000F3E7012801D0042800D10427F07F40F0EA
:104B300001006BF34100F077A07881074FF003008C
:104B40000CD5A071BBF1000F15D100BF8DF85C0032
:104B500017AA31461998FEF71CFD0CE00221022F1E
:104B600018D0012F18D0042F22D00020A071F07F80
:104B700020F00100F07725213046FCF77FFC0DA9DD
:104B800004F590700BF06DFD10B1022800D0FFDF2E
:104B9000002050E6A171D9E7A1710D2104F1240094
:104BA00019F075FC607840F0020060700420CDE7D9
:104BB0000120A071DFE72DE9F04387B091468846D8
:104BC0000446FCF723FC070006D03878272806D0D7
:104BD000082007B0BDE8F08343F20200F9E7B87F90
:104BE00000F00300012809D0002120460AF03BF91B
:104BF000040006D104E0000004E801000121F4E70C
:104C0000FFDFA679012E08D0B8F1000F0FD048467B
:104C10000DF078FFB8B11020DBE7B9F1000F25D116
:104C2000B8F1000F09D0B8F1010F1FD120E0022E1A
:104C300005D0032E05D0FFDF28E00C2526E0012556
:104C400024E0022522E0B8F1020F03D0B8F1010FF1
:104C50000AD00BE0032E09D100251022494604F1A9
:104C6000210019F07BFB11E0022E01D00720B0E7F4
:104C70000025102104F1210019F0E7FB5FEA09008B
:104C800004D0062107F0A2FBC4F82100607825219A
:104C900040F0020060703846FCF7F0FB6078C10716
:104CA00013D020F00100607002208DF8000004F1A4
:104CB000210002908DF804506946FF300BF0D1FCC2
:104CC000022804D018B1FFDF01E084F82050002052
:104CD0007FE730B587B00D460446FCF797FB88B1F7
:104CE000807F00F0030001280FD0002120460AF049
:104CF000BAF804000ED028460DF004FF38B1102099
:104D000007B030BD43F20200FAE70121EEE7607818
:104D1000400701D40820F3E7294604F1410020228E
:104D2000054619F01BFB607840F010006070010729
:104D30000FD520F00800607013208DF80000694640
:104D400004F5907001950BF08CFC022801D000B1A5
:104D5000FFDF0020D4E770B592B00D460646FCF7A1
:104D600055FB18B10178272940D103E043F2020036
:104D700012B070BD807F00F00300012806D0002132
:104D800030460AF070F8040003D101E00121F7E792
:104D9000FFDFA079022829D1A078C00726D0002300
:104DA00002220321304603F011FF08B30C208DF8D6
:104DB00005000A9604A804F5907402220090069457
:104DC000ADF80C2005AB0321304603F07CFF00B1A9
:104DD000FFDF04208DF808008DF81C500BA901A8F6
:104DE0000BF05FFC00B1FFDF0020C1E70820BFE748
:104DF0001120BDE770B5064686B014460D4608463C
:104E00000DF080FE18B920460DF0A0FE10B1102064
:104E100006B070BDA6F57F40FF380ED03046FCF7D7
:104E2000F5FA38B1417822464B08811C1846FCF748
:104E300079FC07E043F20200EAE72046FDF7C0FAFA
:104E40000028E5D11021E01D0DF008FBE21D2946E8
:104E50006846FEF788FC102204F11700019919F04A
:104E60007DFA0020D4E72DE9F041044690B01546C4
:104E70008846002708460DF090FE18B928460DF028
:104E80008CFE18B1102010B0BDE8F0812046FCF770
:104E9000BDFA060003D03078272818D102E043F28B
:104EA0000200F0E7B07F00F00300012806D00021E7
:104EB000204609F0D8FF040003D101E00121F7E703
:104EC000FFDF6078400702D5A078800701D4082072
:104ED000D9E7B07F00F00300012818D0D4E9190108
:104EE000407800B1B5B1487810B1B8F1000F11D0D9
:104EF000C5B1EA1D02A8E168FEF735FC102205F1F4
:104F00001700039919F0FEF930B104270AE0D4E93B
:104F10001910E5E70720B6E71022E91D04F131007A
:104F200019F01CFAB8F1000F06D0102208F10701A1
:104F300004F1210019F012FA6078252140F00200F6
:104F400060703046FCF79AFA6078C10715D020F0FF
:104F50000100607002208DF8200004F121000A9009
:104F600010300B908DF8247008A9EF300BF079FB0E
:104F7000022804D018B1FFDF01E084F8207000207F
:104F800081E7F8B515460E460746FCF73FFA0400E0
:104F900004D02078222804D00820F8BD43F2020073
:104FA000F8BDA07F00F00300022802D043F2050004
:104FB000F8BD30460DF0A6FD18B928460DF0A2FD4B
:104FC00008B11020F8BD00953288B31C2146384640
:104FD000FEF7E1FB112814D00028F3D1297C4A0800
:104FE000E17F62F30001E1772A7C62F34101E1771E
:104FF000297C890884F82010A17F21F08001A17705
:10500000F8BDA17F0907FBD4D6F80200C4F836002A
:10501000D6F80600C4F83A003088A0861022294647
:1050200004F1240019F09AF9287C4108E07F61F32B
:105030008200E077297C61F3C300E077287C800858
:1050400084F82100A07F40F00800A0770020D3E77B
:1050500070B596B00D46064613B1072016B070BD68
:10506000FCF7D4F9040007D02078222802D3A07FCF
:10507000400604D40820F1E743F20200EEE7C5B190
:105080002D208DF80000ADF802601022294601A8FD
:1050900019F064F9287C4108E07F61F30000E077B3
:1050A000297C61F34100E077287C800884F82000A7
:1050B00004E02E208DF80000ADF802600BA96846D0
:1050C00007F035F9A17F21F04001A177C6E770B55F
:1050D0000D46FCF79BF9040005D028460DF036FD7F
:1050E00020B1102070BD43F2020070BD2946204659
:1050F000FEF7F0FA002070BD05E000BF10F8012BAC
:105100000AB100207047491E89B2F7D201207047CA
:10511000F0B50078059F1E4614460D46012800D0C4
:10512000FFDF0C2030803A203880002C08D0287A0D
:10513000052806D0287B012800D0FFDF17206081DA
:10514000F0BDA889FBE72DE9F04786B0144691F839
:105150000C900E9A0D46B9F1010F0BD0102100787A
:105160002E8A8846052807D0062833D0FFDF06B0F0
:10517000BDE8F0870221F2E7E8890C2100EB40004E
:1051800001EB4000188033201080002CEFD0E8891C
:10519000608100271AE00096688808F1020301AADE
:1051A000696900F096FE06EB0800801C07EB4701DA
:1051B00086B204EB4102BDF8040090810DF10601B6
:1051C00040460E320BF00EFB7F1CBFB26089B84226
:1051D000E1D8CCE734201080E889B9F1010F11D073
:1051E000122148430E301880002CC0D0E88960811D
:1051F0004846B9F1010F00D00220207300270DF1BD
:10520000040A1FE00621ECE70096688808F1020313
:1052100001AA696900F05DFE06EB0800801C86B2F9
:10522000B9F1010F12D007EBC70004EB4000BDF845
:105230000410C18110220AF10201103019F08EF819
:105240007F1CBFB26089B842DED890E707EB470108
:1052500004EB4102BDF80400D0810AF1020140468E
:1052600010320BF0BFFAEBE72DE9F0470E4688B09D
:1052700090F800C096F80C80378AF5890C201099B8
:1052800002F10C044FF0000ABCF1030F08D0BCF18E
:10529000040F3ED0BCF1070F7DD0FFDF08B067E7F9
:1052A00005EB850C00EB4C00188031200880002AAB
:1052B000F4D0A8F1060000F0FF09558125E018217F
:1052C00001A819F0E4F800977088434601AA7169B3
:1052D00000F0FFFDBDF804002080BDF80600E0806E
:1052E000BDF808002081A21C0DF10A0148460BF010
:1052F00079FAB9F1000F00D018B184F804A0A4F82D
:1053000002A007EB080087B20A346D1EADB2D6D2F8
:10531000C4E705EB850C00EB4C00188032200880B8
:10532000002ABBD0A8F1050000F0FF09558137E045
:1053300000977088434601AA716900F0CAFD9DF884
:105340000600BDF80410E1802179420860F30001F5
:1053500062F34101820862F38201C20862F3C30171
:10536000020962F30411420962F34511820962F3F2
:1053700086112171C0096071BDF8070020812246A5
:105380000DF1090148460BF02DFA18B184F802A07E
:10539000A4F800A000E007E007EB080087B20A3499
:1053A0006D1EADB2C4D279E7A8F1020084B205FB4C
:1053B00008F000F10E0CA3F800C035230B80002A82
:1053C000A6D055819481009783B270880E3271699E
:1053D00000F07FFD62E72DE9F84F1E460A9D0C465E
:1053E00081462AB1607A00F58070D080E089108112
:1053F00099F800000C274FF000084FF00E0A0D2816
:1054000073D2DFE800F09E070E1C28303846556A3C
:1054100073737300214648460095FFF779FEBDE897
:10542000F88F207B9146082802D0032800D0FFDFA8
:10543000378030200AE000BFA9F80A80EFE7207B20
:105440009146042800D0FFDF378031202880B9F151
:10545000000FF1D1E3E7207B9146042800D0FFDF65
:1054600037803220F2E7207B9146022800D0FFDF10
:1054700037803320EAE7207B1746022800D0FFDF81
:105480003420A6F800A02880002FC8D0A7F80A80F2
:10549000C5E7207B1746042800D0FFDF3520A6F89B
:1054A00000A02880002FBAD04046A7F80A8012E05A
:1054B000207B1746052802D0062800D0FFDF1020E9
:1054C000308036202880002FA9D0E0897881A7F885
:1054D0000E80B9F80200B881A1E7207B9146072829
:1054E00000D0FFDF37803720B0E72AE04FF012000E
:1054F00018804FF038001700288090D0E08978811C
:10550000A7F80E80A7F8108099F800000A2805D0A7
:105510000B2809D00C280DD0FFDF80E7207B0C285A
:1055200000D0FFDF01200AE0207B0D2800D0FFDF44
:10553000042004E0207B0E2800D0FFDF0520387314
:105540006DE7FFDF6BE770B50C460546FBF75EFFC6
:1055500020B10078222804D2082070BD43F2020056
:1055600070BD0521284609F07EFC206008B10020AE
:1055700070BD032070BDFFB585B00746089814467E
:105580000D46022628B908A93846FFF7DCFF002897
:1055900040D108980121801D04F0C6FDADF8080037
:1055A00002464DB100233146384603F00FFB98B355
:1055B0000898007880BB05E02078092820D00F28C3
:1055C0002BD0FFDF03A8009004ABBDF808203146C4
:1055D000384603F078FB00281CD1089802A9801DEA
:1055E000C4E90107DDE90332204604F0AAFD40B317
:1055F000072824D2DFE800F01A182323211C1E00FC
:10560000072600233146384603F0E0FA0028D9D1B6
:1056100043F2040009B0F0BD06E0002331463846ED
:1056200003F0D4FA0028CDD11120F3E70020F1E7F0
:105630000820EFE743F20300ECE70720EAE7032046
:10564000E8E703980090BDF8083004223146384658
:1056500003F0ADFC0028DDD1002DDBD008990D70E2
:10566000D8E710B588B01C46AAB104238DF80030E5
:105670001388ADF80C305288ADF80E208A788DF87A
:1056800012200988ADF8101000236A462146FFF762
:1056900072FF08B010BD1020FBE770B50D46052164
:1056A00009F0E1FB040000D1FFDF2946A01DBDE8A1
:1056B000704004F022BD70B596B00C460646FFF768
:1056C000ECFF05462146304601F03AFE0121304606
:1056D00001F054FE06F014FE002827D0002D25D13D
:1056E0003046FBF793FE050000D1FFDF95F822005E
:1056F0001B281BD9172C19D93A208DF80000ADF8BA
:10570000026095F82200211D884201D9241D00E085
:105710000446ADF8044040F64800ADF806000BA979
:10572000684606F004FE002800D0FFDF16B070BD0A
:105730002DE9F8430546007800260C4612287BD256
:10574000DFE800F0896464433B6637371337373747
:105750000937373737372879001FC0B2022801D000
:1057600010281FD104BBFFDF1EE004B9FFDF6088F3
:10577000052109F078FB0078032805D004280AD019
:10578000072811D0FFDF0DE02879801FC0B2022862
:105790000AD048B106E02879401FC0B2022803D0E1
:1057A000102801D0072657E0607840F008006070AC
:1057B00052E0002CF8D1FFDFF6E704B9FFDF2879CB
:1057C0000128F1D16088172142E0A888052180B224
:1057D000804609F048FB074604B1FFDF07B9FFDF49
:1057E0004146B81D04F063FC02F095FC040008D0AB
:1057F000607840F008006070A4F8028002F06BFC52
:105800002BE013214046FDF75CF937E0FFDF23E092
:1058100004B9FFDF6088052109F025FB070000D1EE
:10582000FFDF6946B81D04F049FC00B1FFDFA9881D
:10583000172902D2172201E00DE00A46BDF8000048
:10584000824201D9014602E0172900D2172160885F
:10585000FFF731FFA8E7FFDF84B1607800070DD5BF
:105860002078182220F00F00C01C20F0F0009030AB
:105870002070294604F1080018F0B5FD3046BDE857
:10588000F88300200870881D04F005BC0A46014614
:10589000901D04F012BC70B50546052109F0E3FA2D
:1058A000040000D1FFDF2946A01DBDE8704004F0D0
:1058B000FEBB2DE9F74F90B04FF0000AADF830A0D5
:1058C000ADF804A047880C4605460521384609F086
:1058D000CAFA060000D1FFDF24B1A780A4F806A011
:1058E000A4F808A0297A04F110003827C91E4FF047
:1058F0000C0B4FF001084FF0120902900F297DD2D6
:10590000DFE801F0F1F0EF7F08D2888D9F3DDBF2F8
:10591000EDB6B6003078022800D0FFDFA8890BEB87
:10592000C001ADF804103021ADF83010002C25D0A6
:105930006081B5F80E8000271DE004EBC7093179BE
:1059400089F80E107188A9F80C10CDF800806888CD
:10595000042305AA296900F0BCFABDF81410A9F8BF
:10596000101008F10400BDF816107F1C1FFA80F813
:10597000A9F81210BFB26089B842DED808E13078C9
:10598000022800D0FFDFE9890BEBC100ADF804006D
:105990003020ADF8300095F80CB0002CABF10400CD
:1059A000C0B20F90EAD06181B5F81090002722E0D4
:1059B000CDF8009068885B4603AA696900F089FA0F
:1059C00009EB0B001FFA80F904EBC70808F10C0281
:1059D00004A90F980AF006FF18B188F80EA0A8F8DD
:1059E0000CA0BDF80C10A8F81010BDF80E107F1C0C
:1059F000A8F81210BFB26089B84200E0C7E0D7D85B
:105A0000C6E00CA8009001AB224629463046FFF7BD
:105A10009AFBBDE03078082805D0FFDF03E030783E
:105A2000082800D0FFDFE8891030ADF804003620E8
:105A3000ADF83000002C3FD0A98961817188A18127
:105A400027E03078092800D0FFDFA88900F10C0199
:105A5000ADF804103721ADF83010002C2CD0608147
:105A6000E8890090AB89688804F10C02296955E047
:105A7000E8893921103080B2ADF80400ADF830105B
:105A8000002C72D0A9896181287A10280AD00221BD
:105A90002173E989E181288A0090EB896888696926
:105AA000029A3BE00121F3E70CA8009001AB2246EB
:105AB00029463046FFF7D8FB6AE030780A2800D044
:105AC000FFDFADF80490ADF830704CB3A989618167
:105AD000A4F810A0A4F80EA084F80C8058E020E0F0
:105AE00002E030E038E041E030780B2800D0FFDF02
:105AF000288AADF830701230ADF8040084B104216A
:105B00002173A9896181E989E181298A2182688AD1
:105B100000902B8A688804F11202696900F0D9F9B3
:105B200036E030780C2800D0FFDFADF80490ADF8F7
:105B3000307044B305212173A4F80AA0A4F80EA084
:105B4000A4F810A024E00CA8009001AB224629463E
:105B50003046FFF7DDFA1BE00CA8009001AB2246AF
:105B600029463046FFF737FC12E00DE00B203B21C1
:105B7000ADF80400ADF8301034B1A4F80680A4F8F4
:105B800008A084F80AA003E01299088014E0FFDF5F
:105B90001299BDF80400088074B1BDF8300020806F
:105BA000BDF804006080287A032805D0102803D0AF
:105BB000112801D086F800A013B00020BDE8F08FB6
:105BC0002DE9FC4156880F46804615460521304692
:105BD00009F049F9040000D1FFDFA41DCDE90064FC
:105BE0002B463A464046696804F05FFCBDE8FC81FC
:105BF00070B50D46052109F036F9040000D1FFDF2C
:105C00002946A01DBDE8704004F063BA70B50D468A
:105C1000052109F028F9040000D1FFDF2946A01D65
:105C2000BDE8704004F088BA2DE9F0438DB00D4610
:105C30001446814607A9FFF786FC002814D14FF6C9
:105C4000FF7601274FF420588CB103208DF8000017
:105C50001020ADF8140008A8069008AA204605A94F
:105C60000AF0DFFD78B107200DB0BDE8F083082011
:105C7000ADF80C508DF812708DF80000ADF80E6084
:105C8000ADF810800CE00798A1780171218841805F
:105C90008DF81270ADF80C50ADF81080ADF80E60B4
:105CA0006A4602214846079BFFF765FCDCE708B51A
:105CB00001228DF8022042F60202ADF800200A46C9
:105CC00003236946FFF7CDFC08BD08B501228DF816
:105CD000022042F60302ADF800200A46042369467A
:105CE000FFF7BFFC08BD00B587B079B102228DF87F
:105CF00000200A88ADF80C204988ADF80E1000236A
:105D00006A460521FFF737FC07B000BD1020FBE70E
:105D100009B10723A5E40720704770B588B00D4688
:105D20001446064607A9FFF70EFC00280ED17CB1E9
:105D30000620ADF80C508DF80000ADF80E40079B22
:105D40006A4608215C803046FFF715FC08B070BD3C
:105D500005208DF80000ADF80C50F0E700B587B0D5
:105D600059B107238DF80030ADF80C2004910023C1
:105D70006A460921FFF7FFFBC6E71020C4E770B5AC
:105D800088B00C460646002507A9FFF7DCFB002873
:105D9000DCD107980121801D04F0C6F99CB121785F
:105DA000062921D2DFE801F0200505160318801E20
:105DB00080B2C01EE28880B20AB1A3681BB18242E1
:105DC00003D90C20C2E71020C0E7042904D0A08822
:105DD00050B901E00620B9E7012913D0022905D006
:105DE00004291CD005292AD00720AFE709208DF807
:105DF00000006088ADF80C00E088ADF80E00A068E7
:105E0000049023E00C208DF800006088ADF80C00B1
:105E1000E088ADF80E00A0680A25049016E00D2079
:105E20008DF800006088ADF80C00A088ADF80E0079
:105E3000E088ADF81000A0680B25059006E00E2064
:105E40008DF8000060788DF80C000C256A46294614
:105E50003046079BFFF78FFB78E700B587B00F222E
:105E60008DF80020ADF80C1000236A461946FFF7A4
:105E700082FB49E700B587B071B102228DF800209E
:105E80000A88ADF80C204988ADF80E1000236A4648
:105E90000621FFF770FB37E7102035E770B588B0B3
:105EA000064601200D46ADF80C108DF800000146A5
:105EB00000236A463046FFF75EFB040008D12946FE
:105EC000304601F02EFA0021304601F057FA204604
:105ED0003CE7F8B51C4615460E46069F09F026F924
:105EE0002346FF1DBCB231462A46009408F03EFD11
:105EF000F8BD000018B18178012938D101E01020E7
:105F00007047018842F60112881A914231D018DC9C
:105F100042F60102A1EB020091422AD00CDC41B30F
:105F2000B1F5C05F25D06FF4C050081821D0A0F59E
:105F30007060FF381BD11CE001281AD002280AD15A
:105F400017E0B0F5807F14D008DC012811D00228BA
:105F50000FD003280DD0FF2809D10AE0B0F5817FCA
:105F600007D0A0F58070033803D0012801D00020AD
:105F700070470F2070470B2826D008DC1BD2DFE8C3
:105F800000F01C2025251A25292325271E0011286D
:105F90001CD008DC0C2817D00D281DD00F2815D0D8
:105FA000102808D110E0822809D0842810D0852834
:105FB00010D0872812D0032070470020704705209A
:105FC000704743F203007047072070470F20704767
:105FD00004207047062070470C2070474FF4505043
:105FE000704708280DD2DFE800F00406040C0C0806
:105FF0000C0A0020704711207047072070470820C6
:1060000070470320704738B50C46050041D06946FB
:10601000FEF7D0FA002819D19DF80010607861F3DE
:10602000020060706946681CFEF7C4FA00280DD1B2
:106030009DF80010607861F3C5006070A978C1F325
:106040004101012903D0022905D0072038BD21785C
:1060500021F0200102E0217841F020012170410768
:1060600004D0A978C90861F386106070607810F0D8
:10607000380F07D0A978090961F3C710607010F0D4
:10608000380F02D16078400603D5207840F04000F8
:106090002070002038BD70B50446002008801546E9
:1060A0006068FFF7B0FF002816D12089A1898842D7
:1060B00011D860688078C0070AD0B1F5007F0AD88F
:1060C00040F20120B1FBF0F200FB1210288007E043
:1060D000B1F5FF7F01D90C2070BD01F201212980AB
:1060E000002070BD10B50478137864F300031370BA
:1060F0000478640864F3410313700478A40864F31B
:10610000820313700478E40864F3C3031370047803
:10611000240964F3041313700478640964F34513C9
:1061200013700078800960F38613137031B108781A
:10613000C10701D1800701D5012000E0002060F3F4
:10614000C713137010BD4278530702D002F0070343
:1061500006E012F0380F02D0C2F3C20300E00123C0
:106160004A7863F302024A70407810F0380F02D088
:10617000C0F3C20005E0430702D000F0070000E0D2
:10618000012060F3C5024A7070472DE9F04796B0D0
:106190000D00804613D0B8F1000F14D0122128460C
:1061A00018F053F906AAFF21012005F0EBFE0024A8
:1061B000264637464FF420596FF4205A78E01020D5
:1061C00016B0BDE8F0870720FAE700BF9DF822006F
:1061D00001280AD1BDF8200048450BD010EB0A0079
:1061E0000AD001280CD002280CD0042C0ED0052C8B
:1061F0000FD10DE0012400E00224BDF81E6008E08C
:10620000032406E00424BDF81E7002E0052400E02B
:106210000624BDF81E1041454AD12C74D6B30DF1A9
:1062200040094FF0000811AACDF81490CDF808806D
:10623000CDE903824FF0070ACDE900A810234246BA
:10624000FF21304605F04CFF10BBBDF840002A4648
:10625000C0B211A90AF0C6FAD0B9AE81D7B103A96C
:106260000BAE4046CDF8088081E84102CDE900A898
:1062700013230022FF21384605F032FF40B9BDF854
:106280004000F11CC01EC0B22A1D0AF0ABFA10B1CA
:10629000032095E70AE0BDF82D00E881062C05D122
:1062A0009DF82200A872BDF820002881002087E711
:1062B00006A805F06FFE002888D0FFF75CFE7FE798
:1062C0002DE9F8439846DDE9087614460D0081462D
:1062D00000D1FFDF0CB1012100E0002105F1080031
:1062E00004F02CFD3080024600232146484602F08F
:1062F0006DFC40B10097328843462146484602F083
:10630000E2FCBDE8F883072C01D01120F9E743F245
:106310000400F6E72DE9F0438DB00E46DDE9149850
:1063200005461C461746142106A818F0B0F80120AF
:1063300002218DF81C108DF818008DF81D80ADF825
:10634000207064B1A178C90709D08DF82200E088D7
:10635000ADF82600A088ADF82400A0680A9001F0EE
:10636000DAFE040023D065800BA904A8CDE9000162
:106370000CAB002231462846FFF7A2FF002813D1BC
:10638000049808368DE871000BAA494606A80C9BB4
:1063900005F0A5F806466078000701D501F09BFEE0
:1063A0005EB13046FFF71DFE0DB0BDE8F08313214E
:1063B0002846FCF786FB0320F6E704980090BDF81A
:1063C0002C3004220021284602F0F1FDECE7F0B564
:1063D0008DB000240746099406A80A94CDE904402C
:1063E0000725CDE90054079408940E4602940394BF
:1063F00010232246384605F073FE80B90BA805909D
:1064000007A90294CDE90341CDE90054BDF8183045
:1064100000223146384605F046FC002801D0FFF73F
:10642000AAFD0DB0F0BD05F0EBBA2DE9FC4705461D
:10643000002600780C46B0460D2871D2DFE800F047
:10644000B2070EAA30C853537188A68C970004B1C6
:10645000FFDFA88880B201F0D2FFA4E0A888042161
:1064600080B2814608F0FFFC074604B1FFDF07B9A0
:10647000FFDF494607F1080004F0F9FB01F04BFE8D
:10648000040008D0607840F008006070A4F8029022
:1064900001F021FE88E013214846FCF712FB97E04B
:1064A00004B9FFDF6088042108F0DDFC070000D19B
:1064B000FFDFE888ADF80000002038809DF800007C
:1064C000010704D5C00602D5A888388005E09DF8EC
:1064D0000100400667D5A88878806078022640F0E1
:1064E000080060705FE0E888ADF8000004B9FFDFE5
:1064F0009DF80100000604D52878072806D0062854
:1065000028D0607840F0080060704CE0608804217A
:1065100008F0A9FC060000D1FFDFA888708019E010
:1065200040E004B9FFDF6088042108F09CFC07000C
:1065300000D1FFDF07F1080005F09AFA90F0010F93
:1065400002D1E87900062ED560880226B880D8E707
:1065500004B9FFDF0226D4E704B9FFDF0226618811
:106560000122204601F08FFF4FF00108C9E7A889FA
:1065700087B204B1FFDF686800902889ADF8040095
:1065800001226946384601F099FF0CE0002CB8D191
:10659000FFDFB6E704B9FFDF022660880021FFF7BE
:1065A00035FBAEE7FFDF9CB16078000710D5B8F18E
:1065B000000F0DD12078142220F00F00001D20F0D4
:1065C000F00080302070294604F1080017F00BFF1E
:1065D0003046BDE8FC873EB50C0008D06B4601AAEA
:1065E000002105F0FCFD20B1FFF7C5FC3EBD1020E9
:1065F0003EBD00202080A0709DF8050002A900F09B
:106600000700FDF7F3FF50B99DF8080020709DF8D2
:10661000050002A9C0F3C200FDF7E8FF08B103209E
:106620003EBD9DF8080060709DF80500C109A07886
:1066300061F30410A0709DF80510890961F3C3008F
:10664000A0709DF80410890601D5022100E0012107
:1066500061F342009DF8001061F30000A07000207B
:106660003EBD70B5144606460D4651EA040005D0FD
:1066700075B108460CF088FA78B901E0072070BDC2
:106680002946304605F006FE10B1BDE8704072E4C0
:1066900054B120460CF078FA08B1102070BD2146A4
:1066A0003046BDE8704096E7002070BD2DE9FE4FF2
:1066B00005460C46007A0A31009104F10801029166
:1066C000904600270C31821E3E464FF0020B4FF0E1
:1066D000010A0191092A75D2DFE802F0F3F205748C
:1066E000252577B6F4006888042108F0BCFB060075
:1066F00000D1FFDF308810B152270726E9E051278B
:106700001026002C7ED06888A08084F806A0A88976
:1067100000220099FFF7A5FF002874D1A8892081E5
:10672000288AE081F8E0B5F81290072825D1E87BA7
:10673000000622D5512709F1140086B2002CE1D0C1
:10674000A88900220099FFF78CFF00287AD1688879
:10675000A08084F806B0A889208184F80EA0288A39
:106760002082A4F81290A88A009068884B46A969F4
:10677000DDF8042001F0C4FACEE0502709F1120040
:1067800086B2002C3ED0A88900220299FFF769FF4B
:10679000002857D16888A080A889E080287A072837
:1067A00011D002202073288AE081E87B4B46C00983
:1067B0006073A4F81090A88A0090688804F112020F
:1067C000A969D7E7A7E00120ECE76888042108F071
:1067D0004AFBB5F812A05FEA000900D1FFDF09F11A
:1067E000080005F045F990F0010F02D1E87B0006A2
:1067F00027D50AF11400512786B2002C7FD0688873
:10680000A08001E070E01DE0A88900220099FFF758
:1068100028FF002816D184F806B0A889208104201A
:10682000A073288A2082A4F812A0A88A0090688801
:106830005346A969019A01F063FAA989A9F80210DF
:106840006AE00320BDE8FE8F6888FAF7DFFD824624
:106850006888042108F007FB8146BAF1000F00D1D7
:10686000FFDFB9F1000F00D1FFDFB9F80400A0F598
:106870007F41FF3902D05127142601E0502712260C
:1068800094B36888A080502F06D084F806B0287B87
:10689000029901F045FA3FE0287BA11D01F040FA82
:1068A00000219AF82300CDE900010B46B9F8022037
:1068B00068884946FFF72EFD0028C3D12CE001E08F
:1068C00013E01FE0FE49A889C988814205D15427F9
:1068D00006264CB16888A0801EE053270CE068882B
:1068E000A080A889E08017E009E06888042108F00A
:1068F000BAFA00B9FFDF55270826002CEFD1A8F817
:1069000000600EE056270726002CF8D0A889A0804A
:106910000020A07100E0FFDFA8F800600CB1278024
:10692000668000208EE7E64900200870704730B589
:1069300087B00C4608F060FA0546FF2800D1FFDF5B
:106940000020208060804FF6FF70A080294604F16F
:10695000080004F073F902AA2946012005F012FB91
:106960001AE000BF9DF80B00000715D5BDF80E001A
:106970002946FFF72CFD9DF80B00FF2340F0100087
:106980008DF80B00BDF80B00ADF80400BDF80E004B
:106990002946019A05F04CFC02A805F0FBFA0028F4
:1069A000E0D007B030BD0A46014602F1080004F00D
:1069B00064B970B50546042108F055FA040000D109
:1069C000FFDF294604F10800BDE8704004F04FB92C
:1069D000F0B58FB00C460746FAF718FD060005D053
:1069E0003078222805D208200FB0F0BD43F2020013
:1069F000FAE70CB1A08870B101208DF81C000320CB
:106A00008DF8200000208DF8210034B1A088ADF869
:106A10002800206803E00920E6E7ADF82800099087
:106A200001F079FB050007D06F800421384608F09B
:106A30001AFA040007D105E013213846FCF741F8A3
:106A40000320D1E7FFDF06A904A8CDE900010CABC4
:106A5000002221463846FFF733FC0028C4D104F158
:106A60000800049903908DE8A20096F8231006AA66
:106A700007A80C9B04F033FD06466878000701D593
:106A800001F029FB1EB13046FFF7ABFAACE70498E2
:106A90000090BDF8183004220021384602F087FA31
:106AA0004FF6FF71A1809FE72DE9FF4F87B0984611
:106AB000DDE9159793467E88DDF850A03046FAF759
:106AC000A5FC05460421304608F0CDF9044605B979
:106AD000FFDF04B9FFDF0834CDE90464CDE9029794
:106AE000CDE9008ADDE9070295F823105B4604F042
:106AF00035F90BB0BDE8F08F2DE9F04F9BB004469F
:106B00004FF000086E48ADF85880ADF83080ADF811
:106B10005480A0F80480ADF81880ADF81C80ADF862
:106B20002480ADF82080007816460D46474601289F
:106B300008D0022806D0032804D0042802D0082058
:106B40001BB0D7E720460BF0DDFFD0BB28460BF08B
:106B5000D9FFB0BB60680CF020F890BB606848B10A
:106B600060892189884202D8B1F5007F01D90C20C3
:106B7000E6E780460BAA07A92846FFF78CFA00280B
:106B8000DED168688078C0F34100022808D19DF802
:106B90001D0010F0380F03D028690BF0F5FF80B905
:106BA00006A92069FFF72FFA0028C9D1206950B142
:106BB000607880079DF8190000F0380002D5E8B32E
:106BC00001E011E0D0BB9DF8180080060ED59DF8BD
:106BD000190010F0380F03D060680BF0D5FF18B91A
:106BE00060680BF0DAFF08B11020A9E708A9606916
:106BF000FFF709FA0028A3D1606940B19DF8210090
:106C000000F0070101293BD110F0380F38D009A955
:106C1000A069FFF7F8F9002892D19DF820008006BE
:106C20002ED49DF8240080062AD4A06950B19DF886
:106C3000250000F00701012922D100E020E010F03A
:106C4000380F1DD0E06818B10078C8B11C2817D2E1
:106C50000FAA611C2046FFF745FA0120B94660F3F0
:106C60000F27BA4607468DF8520042F60300ADF8EA
:106C700050000DF13F0218A9286809F0D2FD08B1B3
:106C800007205DE79DF8600017A9CDF80090C01CB3
:106C9000CDE9019100F0FF0B00230BF201225146D8
:106CA00014A805F0B4F8E8BBBDF85C000E900449E8
:106CB0002A892869091D0092CDE901016B8901E04B
:106CC0001C030020BDF82C202868079905F09FF8C8
:106CD00001007DD120784FF0020AC10601D4800660
:106CE0002BD5ADF80C90606950B908A907A8FFF73B
:106CF0002AFA9DF8210020F00700401C8DF82100A1
:106D00009DF820008DF8527040F0C8008DF82000EA
:106D100042F60210ADF850000CA903AA0023CDF8EA
:106D200000A000E021E0CDE9012140F2032214A8F7
:106D3000089905F06CF801004AD1FE484D465B46C3
:106D40008088ADF83D000FA8CDF80890CDE90390FC
:106D5000CDF814904FF00709CDE900950022FF21EE
:106D6000BDF85C0004F09FFF10B1FFF704F9E7E6FF
:106D70009DF83C00000625D52946012060F30F212F
:106D80008DF852704FF42450ADF85000ADF810500B
:106D900062789DF81000002362F300008DF8100067
:106DA0006278CDF800A0520862F341008DF810001F
:106DB00004AACDE9012540F2032214A805F027F822
:106DC000010005D1606850B3206970B906A900E0E0
:106DD0007EE007A8FFF7B7F96078800705D49DF833
:106DE000190020F038008DF819008DF8527042F625
:106DF0000110ADF85000208940F20121B0FBF1F202
:106E000001FB1202606815ABCDF80080CDE90103EB
:106E1000002314A8069904F0FAFF010058D1207845
:106E2000C00729D0ADF80C50A06950B909A907A82E
:106E3000FFF789F99DF8250020F00700401C8DF828
:106E400025009DF824008DF8527040F040008DF828
:106E5000240042F60310ADF8500016A903AACDF89D
:106E600000A0CDE90121002340F2032214A80999D2
:106E700004F0CDFF01002BD1E06868B32946012062
:106E800060F30F218DF8527042F60410ADF85000F7
:106E9000E068002302788DF8102040788DF811000A
:106EA000E06804AA4088ADF81200E06800798DF827
:106EB0001400E068C088ADF81500CDF80090CDE969
:106EC00001254FF4027214A804F0A1FF010003D0C1
:106ED0000E9800F038FF33E696480321017056B152
:106EE00080883080BDF854007080BDF83000B080DC
:106EF000BDF85800F080002022E670B501258AB068
:106F000016460B46012802D0022816D104E08DF85F
:106F10000E504FF4205003E08DF80E5042F6010061
:106F2000ADF80C0063B10024601C60F30F2404AAC8
:106F300008A9184609F075FC20B107200AB070BDF9
:106F40001020FBE704A99DF820207A48CDE9002114
:106F5000801C02900023214603A802F2012204F0C3
:106F600056FF10B1FFF707F8E8E772480EB1418805
:106F7000318005700020E1E770B594B00446012629
:106F80008DF83E6041F60100ADF83C0012AA0FA951
:106F90003046FFF7B2FF002848D12078654CC00783
:106FA0004FF0000544D01C2102A817F070FA9DF89C
:106FB00008008DF83E6040F020008DF8080042F691
:106FC0000520ADF83C000E959DF83A00119520F093
:106FD0000600801C8DF83A009DF838006A4620F0C3
:106FE000FF008DF838009DF8390009A920F0FF0056
:106FF0008DF839000420ADF82C00ADF830000EA853
:107000000A9011A80D900FA80990ADF82E5002A873
:10701000FFF772FD002809D1BDF80000E080BDF83F
:1070200004002081401C60812570002014B070BDD8
:10703000E5802581BDF84800F4E72DE9F74F3D498B
:10704000A2B04FF000080A78012A04D0022A02D028
:10705000082025B04EE54A88824201D00620F8E794
:1070600023988A46824201D10720F2E701208DF859
:10707000760042F6020B0024ADF874B0ADF84C0077
:107080004FF6FF702146621C62F30F21ADF84E00EF
:10709000ADF8560007918DF87A40FF20ADF87840A2
:1070A0001EA98DF85400149113A804F097FF002531
:1070B0002E462F460DF128090EAB4FF6FF72072121
:1070C00013A804F08EFF78B182285FD1A5B39EB3D8
:1070D0009DF86600ADF86C508DF81840ADF86E6004
:1070E0001BAC012866D06DE09DF83E002FB301284F
:1070F0005BD1BDF83C10594521D11AA8CDE90490C7
:107100000720CDE9000402940394BDF83A0010234F
:107110000022FF2104F0E4FFC0BBBDF86800042892
:1071200001D006284CD1BDF82810239881423CD1CB
:107130000F208EE71C0300203AE0012835D1BDF86E
:107140003C00B0F5205F03D042F6010188422CD10B
:10715000BAF80210BDF83A00814201D1012700E0DF
:10716000002705B19EB1239988421ED11AA9CDE905
:1071700004910721CDE900140546029403941023DD
:107180000022FF2104F0ACFF00B902E02DE04646EA
:107190000BE0BDF86800022801D0102810D1C0B261
:1071A00019AA0AA909F01EFB50B9BDF83A8083E775
:1071B00005204EE706A919A8221D09F032FB08B1E7
:1071C000032046E79DF818000023001DC2B28DF889
:1071D000182024980092CDE901401DA8079904F0D9
:1071E00016FE10B902228AF80020FEF7C4FE30E72E
:1071F00010B50B46401E88B084B206AA002118467E
:10720000FEF770FF07A906AACDE904210020072197
:10721000CDE900100290039002460123FF21204691
:1072200004F041FD0446BDF81C00012800D0FFDF3A
:107230002046FEF7A0FE08B010BDF0B5F84F04469A
:1072400087B038780E46032804D0042802D00820DE
:1072500007B0F0BD04AA03A92046FEF71CFF0500F5
:10726000F6D160688078C0F3410002280AD19DF809
:107270000D0010F0380F05D020690BF085FC08B127
:107280001020E5E7208905AA21698DE807006389B8
:10729000BDF810202068039904F0B9FD10B1FEF785
:1072A0006AFED5E716B1BDF81400308004203870AE
:1072B0002846CDE738B50C00054608D000236A46BD
:1072C000FF2104F08CFF20B1FEF755FE38BD1020E1
:1072D00038BD69462046FEF796FE0028F8D1A07812
:1072E000FF2100F001032846009A04F0A1FFEBE71C
:1072F00030B587B0144600220DF10C0C06AD029299
:107300008CE82C000723CDE900320A462388FF21B0
:1073100004F0C9FCBDF818102180FEF72CFE07B060
:1073200030BD70B50D46042107F09DFD040000D16D
:10733000FFDF294604F10800BDE8704003F0BEBC41
:1073400070B50D46042107F08EFD040000D1FFDF6B
:10735000294604F10800BDE8704003F0D2BC70B5C6
:107360000D46042107F07FFD040000D1FFDF294610
:1073700004F10800BDE8704003F0E0BC70B50D46B4
:10738000042107F070FD040000D1FFDF294604F15D
:107390000800BDE8704003F0DBBC0121FEF736BCFD
:1073A0002DE9F04196B04FF000050C008046ADF895
:1073B00018501CD0E06828B1A068C0B10188ADF8B1
:1073C000181005804046FAF721F8070011D03878E8
:1073D000222861D3404607F00FFD0146A07801281E
:1073E0000AD0022808D0072016B0BDE8F08110208E
:1073F000FAE743F20200F7E7208830B1401C80B280
:1074000007AA04F0BFFD50BB02E043F20300EBE724
:1074100007A804F0BFFD9DF826204FF45051012A23
:1074200009D1BDF82420A2F52453023B03D18228C0
:1074300001D0A0B901E00846D6E7E068B0B106A9DE
:10744000CDE904010720CDE9000502950395A28846
:107450002088BDF81830FF2104F025FC10B1FEF79C
:107460008AFDC1E7A168BDF8180008809DF81F00DB
:10747000C00602D543F20140B6E70B9818B1BDF83B
:107480002800022801D00320AEE70B98A1780078ED
:10749000012903D0800706D40820A5E7C007FBD048
:1074A0000726022001E0012603208DF83C009DF80C
:1074B000200010F0380F00D1FFDF9DF8200059495F
:1074C000C0F3C200084497F8231010F8010C88425A
:1074D00001D90F2088E72088ADF8400004214046FC
:1074E00007F0C1FC040000D1FFDF0DA90CA8CDE915
:1074F00000010EAB324621464046FEF7E1FE002871
:1075000085D108340C9903948DE822010DAA072136
:107510000FA80E9B03F0E3FF10B1FEF762FD63E7D7
:107520000C980090BDF8343004223146404601F0FA
:107530003EFD59E770B5064615460C460846FEF76F
:10754000D9FC002805D12A4621463046BDE87040C6
:10755000D3E470BD71E570B51E4614460D0009D028
:1075600044B1616831B138B12D494988814203D0B5
:10757000072070BD102070BD2068FEF7BBFC0028FE
:10758000F9D1324621462846BDE87040FFF7B4BA2B
:1075900070B515460C0006D038B121498988814262
:1075A00003D0072070BD102070BD2068FEF7A2FC3C
:1075B0000028F9D129462046BDE870403DE670B567
:1075C000054686B00E46144610460BF0BFFA30BB97
:1075D00060680BF0E2FA10BBA5F57F40FF3803D0DE
:1075E0002846F9F713FFA0B1284607F005FC054629
:1075F00030466946FEF7C9FD00280CD19DF81010F1
:107600000F2008293FD2DFE801F008060606060F22
:107610000F0843F2020006B070BD0320FBE743E011
:107620001C0300200EE801009DF80210012908D17A
:10763000BDF80010B1F5C05FEDD06FF4C052D1427B
:10764000E9D09DF8061001290BD1BDF80410A1F571
:107650002851062905D2DFE801F0030304030303E0
:10766000D9E79DF80A1001290ED1BDF80810B1F52F
:10767000245FD0D0A1F524510239CCD00129CAD041
:10768000022901D1C7E7FFDF606878B9002305AAA6
:107690002946304604F0A3FD10B1FEF76CFCBAE7B2
:1076A0009DF81400800601D41020B4E761882246BA
:1076B00030466368FFF71CFEADE72DE9F043044652
:1076C00089B08946154610460BF040FA18B11020D3
:1076D00009B0BDE8F083204607F08EFB4FF6FF7738
:1076E0000646BC4201D0FF2E09D00146002307AA5E
:1076F000484604F074FD28B1FEF73DFCE8E743F28C
:107700000200E5E79DF81C00C00602D543F20140E7
:10771000DEE7002406A8CDE904404FF00708CDE9D4
:107720000084029403946A883B463146484604F03C
:10773000D7FC070014D168680BF008FA68B96868CC
:107740000294CDE903400594CDE900842B886A8832
:107750003146484604F0C4FC0746BDF818002880AE
:107760003846C9E739B1FA4B0A881B899A4202D8D0
:1077700043F20300704713E610B586B0F44C0423BF
:10778000ADF81430E38843B124898C4201D2914290
:1077900005D943F2030006B010BD0620FBE7ADF8A3
:1077A0001010002100910191ADF8003002218DF8F8
:1077B000021005A9029104A90391ADF812206946AF
:1077C000FFF7EEFDE7E72DE9FC4781460F46084647
:1077D0000BF098F988BB4846F9F718FE5FEA0008F5
:1077E0000AD098F80000222829D30421484607F03F
:1077F0003AFB060005D103E043F20200BDE8FC8736
:10780000FFDF06F1080003F060FA0546387801282A
:1078100003D0022804D00720F0E7A8070FD502E024
:1078200015F0340F0BD0B8793C1DC00709D0E088A3
:1078300038B1A0680BF066F918B11020DEE7082017
:10784000DCE73A782088002128B3A0F20113072151
:10785000112B18D20CD2DFE803F00B090D0B1D0B16
:10786000121D100B0B1D1D1D1D0B1D00022A11D119
:107870000846C3E7012AFBD00CE0EA0600E0AA06AE
:10788000002AF5DA06E0A0F5C0721F2A02D97D3A77
:10789000022AEDD8C1B298F82300CDE90001728820
:1078A000234631464846FEF735FDA7E72DE9FF4F51
:1078B0008DB01E4615460C464FF000080F460D9839
:1078C000F9F7A4FD30B10078222806D2082011B0C3
:1078D000BDE8F08F43F20200F9E7B00801D00720BD
:1078E000F5E7032E00D100260D9807F085FA4FF634
:1078F000FF7A0690CCB1022D74D320460BF04DF9DF
:1079000030B904EB0509A9F101000BF046F908B103
:107910001020DCE7AD1EAAB22146504604F080FDDF
:1079200039F8021C88425DD1ADB28948B10702D551
:107930000189491C00E001211FFA81F9F10701D0FA
:10794000068900E0564607AA4846069904F01AFB45
:107950004FF0070B4FF0000A0BE07888102841D851
:1079600008F1040108441FFA80F8A8453AD804EB4E
:1079700008077FB339884945EFD353E09DF81F10BE
:107980000A074FD544B304EB080708F104027B88CB
:107990001FFA82F8102B25D803EB0802AA4221D83F
:1079A0003A8890421ED1C8061ED50DF10C090CAACA
:1079B00004EB08015046CDF808A089E80700CDE99E
:1079C00000BA38880022069904F06DF928B1FEF754
:1079D000D2FA7CE726E005E00CE07888BDF83010AC
:1079E000884201D00B2072E7798801EB08001FFA6A
:1079F00080F806E0C90604D50699FEF7E8FC0028E1
:107A000087D19DF81F00FF2320F010008DF81F0084
:107A1000BDF81F00ADF80000BDF82200009A0699DD
:107A200004F006FC07A804F0B5FA18B9BDF8220066
:107A3000B042A3D904210D9807F015FA040000D133
:107A4000FFDF22885AB1CDE900BA5546002321460E
:107A50000D98FEF75FFC0028BBD1258037E700209A
:107A600035E72DE9F04F8DB01E4617000D464FF05B
:107A700000041BD0B10802D007200DB028E7032E68
:107A800000D1002607F0B8F98046FF2805D07DB167
:107A900028460BF079F848B902E043F20200ECE71F
:107AA0003988681E08440BF06FF808B11020E4E72D
:107AB0002749B00701D5488900E00120F2074FF6B9
:107AC000FF7902D04989491E00E049468EB207AAD3
:107AD000414604F057FA4FF0000B4FF0070A3EE022
:107AE0009DF81F0000073AD506A9CDE904B1CDF8ED
:107AF00008B0CDF80CB04B4600224146CDE900ABB2
:107B0000604604F0EDFA08BB25B3BDF818103A88BA
:107B100021442819091D8A4234D3BDF8222020F8B7
:107B2000022BBDF8182020F8022B06AA0592CDF8EA
:107B300008B0CDE903B0CDE900ABBDF82200BDF837
:107B400018300022414604F0CBFA18B1032094E724
:107B50001C030020BDF818002044001D84B207A8B3
:107B600004F018FA20B1822806D0FEF704FA84E760
:107B7000BDF822C0B445B3D934B175B13988A01C61
:107B8000814203D20C2078E7052076E72246294679
:107B9000484604F045FC29190880A41C3C800020BC
:107BA0006BE710B504460AF0D1FF08B1102010BDF4
:107BB0006A4840892080002010BD2DE9F041A4B022
:107BC0000C4606464FF00008142105A816F05FFC8D
:107BD00001208DF818008DF8140000278DF8197019
:107BE000ADF81C403046F9F711FC30B1007822287E
:107BF00006D2082024B0BDE8F08143F20200F9E784
:107C00000421304607F02FF9050000D1FFDF0AA953
:107C100004A8CDE9000116AB002229463046FEF744
:107C20004FFB0028E6D104980835CDE90007CDE9DF
:107C300002650AAA072105A8169B03F050FC10B1A3
:107C4000FEF7CFF9D6E704980090BDF8283004225B
:107C50004146304601F0ABF900B1FFDF2146304626
:107C6000FDF7C6FF17A9284603F01EF800B1FFDF95
:107C7000BDF85C00172801D2172100E00146A1429F
:107C800004D8172801D2172400E0044621463046C4
:107C9000FFF756FB054621463046FDF7FEFC414600
:107CA000304601F031FB00B9FFDF04F029FB28B3B7
:107CB00025BB3046F9F7AAFB050000D1FFDF95F898
:107CC00022001B281AD9172C18D93A208DF82C001D
:107CD000ADF82E6095F82200211D884201D9241D9F
:107CE00000E00446ADF8304040F64800ADF8320000
:107CF00018A90BA804F01BFB00B1FFDF002079E7F7
:107D0000F8B51C4615460E46069F07F00FFA2346A7
:107D1000FF1DBCB231462A46009406F027FEF8BD8E
:107D200070B50C4605460E21204616F08EFB00204D
:107D300020802DB1012D01D0FFDF70BD062000E0B5
:107D40000520A07170BD10B50C4604F0E8F800B134
:107D5000FFDF2046BDE81040FEF70DB91C030020F0
:107D600010B50446007896B0022805D0012803D04B
:107D700043F2050016B010BDA17889290AD06078B9
:107D8000892807D021B1032902D808B1032801D9D5
:107D90000720EFE74E208DF800002078022801D060
:107DA000012000E000208DF80200607800F0DBFD8B
:107DB000C01D8DF80300A078012815D000F0D3FD78
:107DC00010F101008DF80400607800F0CCFD8DF812
:107DD0000500A07800F0C7FD8DF806009DF805208D
:107DE0000621102A04D005E0022000F0BCFDE9E7DE
:107DF0008DF80510102801D18DF806102078012883
:107E000004D19DF80300401C8DF80300FBF7DAF85D
:107E1000001DADF808000BA9684604F088FA00B10F
:107E2000FFDF0020A6E72DE9FF4F91B09B461546E6
:107E30000600FE49D1E900010396CDE90C01507A14
:107E4000117A0844C7B222D05FF000044FF0000955
:107E5000CDF81C900520ADF81C001F20ADF81E00C9
:107E6000F3A00690CDF81490F01D8DF814904FF00B
:107E7000010A20F007008DF815A0B04200D0FFDF06
:107E800028880399401C1FFA80F814B107E00124E8
:107E9000DCE708F0FF0008F04BFC00B1FFDF0399BE
:107EA0003A4601EB0810C01C20F00301D5F81880F9
:107EB00003913CB981F800901FFA88F003F0BAFEF4
:107EC00000B1FFDF0399234601EB08000390A87A75
:107ED000297A3A460844C1B203A800F092FD0398FB
:107EE000C01C20F003000390697A00912B7AAA7AD3
:107EF00004B1002002A906F092FE00B1FFDFBDF838
:107F0000081003980DF1780808443A4698E88A006A
:107F1000C01C20F00300CDE90270CDE9001304B1CC
:107F200000205B4608A907F005F800B1FFDF0899BB
:107F300003980844C01D20F0070003901299821B8B
:107F4000002C0A603CD1BD4ABB491160111D401E86
:107F5000086001232C220EA9B94806F0E1FD00F0CB
:107F600010FD00211E22084602F08EF8FAF7C9F92A
:107F700000F079FF04F0BCF9FEF7D5FCE8680CAA24
:107F8000214620B1FBF74DF830B1FFDF04E005A832
:107F9000FBF747F800B1FFDF05F11400FEF7ECFF37
:107FA00000B1FFDF4FF49671A64816F070FAA548AD
:107FB000022180F829A180F82A11062180F82B11CE
:107FC00015B0BDE8F08F10B59E4CA078092800D3FD
:107FD000FFDF207804EB401010F8041F21F0FF01B0
:107FE0000170417821F00701C91C21F0180141708E
:107FF0000121E17010BD2DE9F04105460C46002736
:108000000078052190463E46B1EB101F00D0FFDFFF
:10801000287A58B1012810D0FFDF00BFA8F800600F
:108020000CB1278066800020BDE8F0810227092678
:108030007CB1A889A080A87B09E00327142644B15D
:108040006888A0802869E060A88A2082287B207246
:10805000E4E7A8F80060E6E700B597B051218DF895
:10806000001000780BA900F001008DF802006846AE
:1080700004F05DF917B000BD00B5017897B001F0CC
:1080800001018DF80210417801F001018DF8031013
:108090000178C1F340018DF804104178C1F340012B
:1080A0008DF80510017889088DF806104178890847
:1080B0008DF8071081788DF80810C1788DF80910B7
:1080C00000798DF80A004B208DF800000BA9684656
:1080D00004F02DF9CEE770B55A4CE078002819D09D
:1080E0002078002504EB4010407900F007000119CA
:1080F00091F82801401E81F828012078401CC0B268
:108100002070092800D12570A078401CA0700AF0CA
:1081100094F8E57070BD4B4890F82B01002800D012
:1081200051E770472DE9F043464D9BB05FF00006E4
:10813000D5F8240168B1FFF7EEFF002874D02022A3
:10814000D5F8241116F04FF9FFF7C5FFC5F82461E3
:10815000EEE795F82901002866D0FFF734FF0446C2
:10816000374806F00EFD606000B9FFDF606804F07C
:108170002BF988B12046F9F7BAFB6078010706D5DC
:1081800020F00700401C6070FFF7A5FFD0E72C48E7
:10819000616806F0FFFCCBE72948616806F0FAFC4D
:1081A00001A800F0BBFC00286DD10321BDF804003C
:1081B00006F059FE8046BDF8040006F0B7FF0746FA
:1081C000B8F1000F00D1FFDFD8F8040010B100783B
:1081D000FF2858D0FFF7F7FE0446384606F069FB43
:1081E000606000B9FFDF606800F104090671BDF846
:1081F00004006080204600F02EFF384606F029FC7F
:1082000000B9FFDF47208DF81000BDF80400ADF87D
:10821000120004A805F0B4FF10A804F038FB607841
:10822000010713D4C0060FE02DE0000014E80100A0
:108230006E52463578000000000000200006024023
:10824000840500205804002006D408E020F0070030
:10825000801C6070FFF73FFFC8F8049068E7D8F80B
:10826000040038B10178491C11F0FF0101708DD173
:10827000FFDF5DE700221146384600F072FB002860
:1082800084D1FFDF54E71BB0BDE8F08310B5FE4C8E
:10829000A0600868E060AFF2731001F080FE6070CB
:1082A00010BDF94900200870704730B505464FF001
:1082B00080500C46D0F8A41097B0491C05D1D0F8D6
:1082C000A810C9430904090C08D050F8A01F01F0F8
:1082D000010129704168216080680EE02B208DF833
:1082E00000000BA9684604F022F800B1FFDF01206E
:1082F00028700C982060BDF83400A08028780028F1
:1083000003D0607940F0C000607117B030BDF0B5A7
:108310004FF080540746D4F8800097B00D462B26C6
:10832000401C0BD1D4F88400401C07D1D4F888003D
:10833000401C03D1D4F88C00401C0BD0D4F8800032
:108340003860D4F884007860D4F88800B860D4F835
:108350008C0016E08DF82C6069460BA803F0E7FF4F
:1083600000B1FFDF01983860029878608DF82C60CA
:1083700069460BA803F0DBFF00B1FFDF0198B8608E
:108380000298F860D4F89000401C0BD1D4F8940007
:10839000401C07D1D4F89800401C03D1D4F89C00AD
:1083A000401C08D054F8900F286060686860A0688E
:1083B000A860E06816E08DF800600BA9684603F03D
:1083C000B6FF00B1FFDF0C9828600D9868608DF84B
:1083D00000600BA9684603F0AAFF00B1FFDF0C980C
:1083E000A8600D98E86017B0F0BD30B5A74C054601
:1083F000D4F8240100B1FFDFC4F8245130BD3EB5EC
:108400000546032106F02FFD0446284606F08EFEA1
:10841000054604B9FFDF606818B10078FF2800D175
:10842000FFDF01AA6946284600F09BFA60B9FFDF2A
:108430000AE0002202A9284600F093FA00B9FFDF03
:108440009DF8080000B1FFDF9DF80000411E8DF887
:108450000010EED260680199884201D1002060606E
:108460008A4C94F82A01022800D3FFDF94F82A01ED
:10847000401CC0B284F82A01012803D18248407808
:1084800001F0ACFD3EBD70B50446A1F57F40164637
:108490000D46FF3800D1FFDF012E01D0FFDF70BD98
:1084A000207820F00F00401D20F0F00050302070A8
:1084B00000202072A5810120A07370BD70B5154603
:1084C0000C460646FFF727FE90B1017821F00F0118
:1084D000491D21F0F00150310170468001210172E7
:1084E00021680161A18881820573BDE87040F2E5D1
:1084F0003046BDE870401321FAF7E3BA70B505467F
:108500000C4608460AF022FB08B1102070BD284630
:10851000F8F77CFF28B1284600F0E7FE2070002025
:1085200070BD43F2020070BD2DE9F04F044656487D
:10853000894687B0017811B1082007B041E552485B
:108540005349416020460AF001FB002875D1484696
:108550000AF0FCFA002870D1637A217A5818FF28B3
:108560007DD82088FE287AD800B90A202080A0690A
:1085700008B94FF4B060A0616068A0B14578827816
:1085800005EB45052A440578067905EB450502EB20
:1085900045024579C07805EB450505EB8605C0EB3E
:1085A000C000284409E003EB430001EB410200EB6B
:1085B0004202C1EBC10505EB830086B2C3EBC300E9
:1085C0001044C1EBC1021044084487B2208AFAF774
:1085D000EFFC0028B1D1FAF7F5FC001D78430590B7
:1085E000FAF7F0FC001D00FB06F8E168A06900F056
:1085F00041FA5FEA000AA0D1A17A607A81422ED8BE
:108600004FF0120B08280ED8207A01280BD808F05A
:10861000FAF9054609F0D0FD2A1A217A607A521E2D
:108620000B189A4201DA584687E765688B46009036
:10863000BDB128460AF0B1FA08B110207DE7A9784B
:10864000687808442978421800985844904206D126
:108650006A7929791144EA781144884201D00720C7
:108660006BE7CDF80080CDE90176224603A9002012
:10867000059BFFF7D8FB044D039AD9F800306868D2
:108680001118994209D805E01C0000205804002068
:1086900048130020B2F5803F03D30420C9F800102E
:1086A0004BE7CDF80080CDE90176224604A9059B71
:1086B000FFF7B9FBDDE90301884200D0FFDF049832
:1086C000696808446860C9F80000FF490120287003
:1086D0000870504631E72DE9F04707460C4608463A
:1086E0000AF034FA40B938460AF04EFA20B9F81CBC
:1086F00020F00300B84202D01020BDE8F087F34814
:108700004FF00008817889B14178824600EB41152D
:10871000B4F8009015F8040F234600F00F00002273
:10872000294600F037FA060004D013E0A4F80080D0
:108730000520E2E797B12188494501D90C260DE0D3
:108740002878234600F00F003A46294600F022FA26
:10875000060005D00C2E01D0A4F800803046CCE7EE
:108760009AF801005446401CC0B28AF8010009285A
:1087700001D184F80180A078401EA070687800F0D4
:10878000070101290BD0022903D0032918D0FFDFEC
:10879000E4E7C006E2D46888FFF731FEDEE7CC48A4
:1087A000696806F0F7F994F82901401CC0B284F812
:1087B00029010128D2D1C748407801F00FFCCDE74C
:1087C00094F82B01401C8AF82B01C7E770B50D46C1
:1087D00004460AF097F918B928460AF0B7F908B123
:1087E000102070BD29462046BDE8704007F0D7BF75
:1087F00070B5044615460E4608460AF083F918B9C6
:1088000028460AF0A3F908B1102070BD022C03D04D
:10881000102C01D0092070BD2A463146204607F0B1
:10882000E1FF0028F7D0052070BD70B514460D4655
:1088300006460AF067F938B928460AF087F918B9E8
:1088400020460AF0A1F908B1102070BD2246294641
:10885000304607F0E6FF0028F7D0072070BD10B5BE
:1088600096B004460AF072F910B1102016B010BD8F
:108870000F208DF800000BA9684603F058FD002872
:10888000F4D19DF834002070BDF836006080BDF84A
:108890003800A0800020E9E770B505460C46084680
:1088A0000AF072F920B93CB120680AF04FF908B11A
:1088B000102070BDA08828B121462846BDE8704030
:1088C000FEF786B8092070BD70B504460D4608460F
:1088D0000AF018F930B9601E1E2814D828460AF08C
:1088E00011F908B1102070BD032C01D9072070BD0B
:1088F00004B9FFDF784800EB840050F8041C2846D8
:10890000BDE870400847A4F120001F28EED8294692
:108910002046BDE87040F9F7FEBB70B504460D4631
:1089200008460AF013F930B9601E1E280FD82846F1
:108930000AF0E8F808B1102070BD012C03D0022C19
:1089400001D0032C01D1062070BD072070BDA4F119
:1089500020001F28F9D829462046BDE87040F9F7C5
:1089600086BC05F042BE892805D0032805D0022820
:1089700005D0012070471020704706207047032063
:10898000704710B596B003F0C3FC52484178806838
:1089900003F0BCFE4F4801240C300178012916D1A8
:1089A0003E218DF80010C0788DF8020010B101282A
:1089B00003D005E08DF8024002E000208DF80200AF
:1089C000684605F0DDFB10B10BA803F060FF022044
:1089D0008DF82C008DF82D008DF82E000BA8FFF7D8
:1089E000BFF900B1FFDF8DF82C4003208DF82D007A
:1089F0008DF82E000BA8FFF7B3F9002800D0FFDF99
:108A000034E72DE9F0410646022012B101EB4200A5
:108A1000401DC7B23068C01C20F0030232601BBB8F
:108A20002A483B460921243809F05DFF002408E06C
:108A3000092C11D2DFE804F005070509090B0B0525
:108A40000500264804E0264802E0264800E02648C3
:108A500009F068FF054600E0FFDFA54200D0FFDF18
:108A6000641CE4B2092CE3D3306800EB07103060DB
:108A7000BDE8F08138B50C00054604D008460AF080
:108A800041F800BB02E0F62844D345E060680AF0F4
:108A900039F8C0B9607800F00300012803D002283B
:108AA00001D0072038BD69462046FBF783FD00282A
:108AB000F8D1607800F0030002281CD19DF8000076
:108AC000C8B1606812E014E00800002058040020DB
:108AD000840500201C00002034E801006B1F00000A
:108AE000058F0000CB2F0000E50401000AF04CF8D0
:108AF00008B1102038BD6089F8280BD8218981423F
:108B000008D8617801F00301012905D1D73080B27E
:108B1000A84201D9092038BD002038BD2DE9F04315
:108B200097B0814646208DF82C0069460BA803F0CB
:108B3000FEFB00B1FFDF43F2040600246D46DFF8C0
:108B400084801FE02F19B87DC10706D0400704D4E8
:108B500005EB4400C08800F0B9FB98F82A0178B111
:108B6000B87D80070CD505EB4400C08800F037FACB
:108B700030B105EB44000026C188A9F8001005E0DB
:108B8000641CE4B29DF80400A042DBD817B0304664
:108B9000BDE8F0832DE9F041044600201880601EF6
:108BA0001D4616460F46052800D3FFDF06482A4615
:108BB00000EB8400314650F8043C3846BDE8F041F3
:108BC00018470000580400201CE801002DE9F04778
:108BD0008A46984615460646032106F044F904469F
:108BE000304606F0B5FA0C35AFB2002581462E4668
:108BF00004B9FFDFB9F1000F00D1FFDF04EB8A00F9
:108C00000189B94200D30125218CB94202D2BAF1BF
:108C1000060F00D3012638EA050104D0817A41F01D
:108C2000020181720BE038EA060108D0817A41F036
:108C30000401817214F8220F40F00400207005EA4C
:108C40000600BDE8F0872DE9F0478246DDE90846D9
:108C5000174604F10C0099460D461FFA80F80023D0
:108C6000224639465046FFF7B1FF60B1A8780006AA
:108C70001BD426F8044C26F8029C504606F068FAED
:108C8000060008D106E0072F01D01120D9E743F2F2
:108C90000400D6E7FFDF241D3046A1B205F0A4FB97
:108CA00000B9FFDF504603F095FC05EB8700062F67
:108CB0000289A2EB0801018103D2298CA1EB0800F3
:108CC00028840020BDE72DE9F8431D4617460E46CF
:108CD000DDF8208006F03CFA040019D03F1DB9B23F
:108CE00005F032FB2860B0B1067120466A4629685B
:108CF00005F0EEFD009800210A460180817003F026
:108D000029FD0098C01DC8F800000020BDE8F883C8
:108D100043F20200FAE7072E01D01120F6E743F2F2
:108D20000400F3E72DE9F04F0F46054687B01646DD
:108D30005088032106F097F8040000D1FFDF4FF0C0
:108D400000098DF80890A078400600D1FFDF042FBD
:108D500053D3297841F30000401C06D162786B7828
:108D60009A424AD12278120747D04FF0010B4FF0B8
:108D70000208142939DA4FF6FF7A012933D0122973
:108D800002D0132931D11CE00C2F2ED1A17801F093
:108D90007F01012929D0207820F00F00401C20708D
:108DA000687860708DF808B0A888ADF80A00E88887
:108DB000ADF80C002889ADF80E006889ADF81000F8
:108DC00016E0062F11D1207820F00F002070718856
:108DD000012009F054FE8DF80880ADF80AA0A8889B
:108DE000ADF80C0004E0062F0AD09DF80810B9B1C8
:108DF0007088324602A9F9F72AF907B0BDE8F08F6A
:108E0000207820F00F0020707188012009F037FED3
:108E10008DF80880A888ADF80A00ADF80CA0E7E747
:108E20000028EAD0768805A8009006AB0622042127
:108E30003046FFF748FF00B1FFDF05980523042205
:108E400080F800B069784170A0F80280A0F8049022
:108E50000621CDE9001021463046FFF7F4FE002838
:108E6000CBD0FFDFC9E710B5FAF7ACF80021FF4B14
:108E70000A4600BF23F81120491C0829FAD3FB4AEF
:108E800000F10C01103240001180518018309080A8
:108E90004D20D08011815181C1EBC100908110BD66
:108EA00070B50C46897821F0FF01A170217821F07E
:108EB0000F012170012161700021616006F048F905
:108EC000050000D1FFDF284605F03CFAE7491031E4
:108ED0008989401A20852046BDE8704000F014BB07
:108EE00070B50D46032105F0BEFF040000D1FFDF81
:108EF000A07865F30600A07070BD704701460120A0
:108F000009F0BDBD3EB58DB20321284605F0ABFF8B
:108F1000040000D1FFDF2078002220F00F00207035
:108F200002208DF800004FF6FF70ADF80200ADF89A
:108F3000040069462846F9F78AF83EBD2DE9F84F46
:108F400005460C4600270078012192463E46B1EBCB
:108F5000101F00D0FFDF287A032809D0FFDF00BFF1
:108F6000AAF800600CB1278066800020BDE8F88F69
:108F7000B5F80C80702708F10A0086B2A4B16888A1
:108F8000A08068892081A4F806806888D5F80490BC
:108F900004F10A0506F0CAF82A4607254946434661
:108FA000009505F0E3FCDBE7AAF80060DDE72DE9BA
:108FB000FC410F461C46164680460321089D05F0DD
:108FC00052FF010008D033463A464046CDE90045FD
:108FD000FFF739FEBDE8FC8143F20200FAE7F8B57D
:108FE0000646A0F57F40FF3816D0304606F09EF8C2
:108FF000040000D1FFDF204605F05BFC050000D136
:10900000FFDF204629466A4605F062FC009CB4F862
:109010000500E41C052801D00120F8BD03213046DD
:1090200005F021FF050000D1FFDF2079122807D1CC
:1090300020880C2804D1A87800F07F00022806D0F0
:109040000023062204213046FFF7C0FDF8BD0023AF
:1090500006220521F7E7F8B50446408806F066F8D1
:10906000050000D1FFDF6A462846616800F0CCF9B0
:1090700002460098121F30F8031F458891421DD107
:10908000042D1CD0052D27D0062D1DD0402D15D325
:109090000E46284600F0D4F908280FD0207820F09A
:1090A0000F00401C20F0F0001030207003202072D0
:1090B0006581A681607840F008006070F8BD2246A6
:1090C000001D00F0C9F9F8BD636864880A46011DF7
:1090D0002046FAF7F3FEF8BD2246001DFFF722FEF8
:1090E000F8BD7FB50D460646032105F0BCFE040021
:1090F0003AD0207800F00F00012838D002A8009064
:1091000003AB0C2205213046FFF7DDFD002829D1F5
:10911000029812210523017061781A46891C41705A
:1091200008214180298881806988C180A9880181BE
:10913000E98841810C21CDE9001021463046FFF736
:1091400082FD00B1FFDFF02300223146012009F04B
:10915000F9FB207820F00F00401C20706078801C04
:109160006070002004B070BD43F20200FAE71120E5
:10917000F8E77FB50D460646032105F074FE0400AE
:1091800006D0207800F00F00012804D00820E9E77D
:1091900043F20200E6E702A8009003AB0622052195
:1091A0003046FFF790FD0028DCD1029813210523FB
:1091B0000170617841700221418085800621CDE9EE
:1091C00000101A4621463046FFF73DFD00B1FFDF93
:1091D000207820F00F0020700020C3E72DE9F84F21
:1091E0000F468346032105F03EFE0546584605F02E
:1091F000AFFF80464FF0000A05B9FFDFB8F1000F5E
:1092000058D1FFDF56E040466946002205F0EDF9EF
:109210009DF800408146082C00D3FFDF05EB840653
:1092200009F108003189062C0144318102D2298CD0
:1092300008442884072C03D10AF1010000F0FF0A3A
:10924000B07AC0070DD02146284600F0DFF840B9BB
:10925000B07A20F00100B072584684B3032C2FD0AE
:10926000FFDFB07A81070AD502E00000B4050020D4
:1092700020F00200B0722146584600F0D8F8062CC3
:1092800018D895F82200410714D520F0040085F87D
:109290002200002405EB8400817A4A0706D521F0DC
:1092A000040181722146584600F0C1F8641CE4B202
:1092B000062CEFD37F1EFFB2A5D2504656E602E041
:1092C000FAF793FECDE7FEF768F8CAE710B5032179
:1092D00005F0C9FD040000D1FFDF204600F014F9BD
:1092E000A07840F08000A07010BD10B5032105F0FB
:1092F000BAFD040000D1FFDFF9F764FE218D0C30C8
:10930000B1FBF0F0C0B210BD70B50D46032105F001
:10931000AAFD040000D1FFDF062D00D9FFDF29469A
:10932000204600F073F8002805D004EB85018A7A06
:1093300042F001028A7270BD10B50446402801D285
:10934000072010BD00F07CF8082802D04FF44450EC
:1093500010BD0021774802E0491C082903D230F8EB
:109360001120002AF8D1082903D020F8114000204C
:1093700010BD042010BD10B5402801D2072010BD3B
:1093800000F05EF8082805D06A4A002122F8101083
:10939000084610BD052010BD2DE9FE4315460C0002
:1093A000804606D02DB16088402804D20720BDE851
:1093B000FE831020FBE7218811B300F041F8082854
:1093C00020D002A80090228801AB07214046FFF779
:1093D0007AFC0028EBD140462788019E05F0B8FEB4
:1093E0002A46072531463B46009505F0F8FA0298D3
:1093F00000902388628807214046FFF7D8FDD6E712
:109400000C20D4E70520D2E705F062BA072904D082
:10941000484A103232F8112000E0028D00EB810042
:109420000089904201D2012070470020704710B59A
:10943000032901D0FFDF10BDBDE81040FAF79BBD46
:10944000014600203B4A02E0401C082803D232F8C3
:1094500010308B42F8D17047F0B50F4606460146F2
:1094600087B014463846FCF7ABFBC0B2082842D19F
:109470000020ADF8100003906088032105F0F3FC94
:10948000050000D1FFDF00212846FFF7BFFF78B9B4
:1094900060880021FDF763FFADF81000024603A8C5
:1094A0000090608805AB0021FFF70DFC00B1FFDFE5
:1094B00003980599CDE90010029404AB3246384672
:1094C0006168FDF7F1FAC0B205281BD2DFE800F0B1
:1094D000031A13151300BDF8100000280BD00399D0
:1094E0000423CDE90001608800222946FFF7ABFB89
:1094F000002800D0FFDF07B0F0BD607840F010001A
:109500006070F8E7FFDFF6E710B504462021083069
:1095100014F0BDFF0748002110F1100004EB810397
:1095200030F81120491C1A810629F7D9208DA08412
:1095300010BD0000B405002030B44FF0E02001233E
:109540004FF4006C0021C0F880C11D02C0F88051AA
:109550001C06C0F88041E84A82F80014D21E82F846
:109560000014E64A82F80014E54A53609360C2F89A
:109570004011C2F84411C2F84811C0F880C2C0F8C6
:109580008052C0F88042C0F800C1C0F800411360AA
:1095900030BC704770B401204FF0E023C6024FF09A
:1095A000000CC3F880610402C3F880410506C3F8CB
:1095B0008051D34A50609060D24801680029FCD1A4
:1095C000C2F840C1C2F844C1C2F848C1C3F88062C1
:1095D000C3F88042C3F8805270BC70474FF0E0205F
:1095E0004FF40061C0F88012C910C0F880127047B3
:1095F000002804BFC4487047012804BFC34870470F
:10960000022804BFC248704700B5FFDF002000BD3C
:1096100008B5BB49002298B101282FD002281CBFF1
:10962000FFDF08BD4FF48020C1F80803C1F84803EC
:10963000B8480260C1F84821B5480068009008BDEC
:109640004FF48030C1F80803C1F84803B24B1A60E8
:10965000C1F84021B14BC1031960B149C1F80803F9
:109660004FF0E0230012C3F88001AE480260C1F859
:109670004021C1F80022AC48027008BD4FF4003010
:10968000C1F80803C1F84803A8480260C1F84421A2
:109690009E480068009008BD70B5DFF864C20426DB
:1096A00000240125B0B101284CD002281CBFFFDFE7
:1096B00070BD9F484FF48022012BC0F8401518BFA1
:1096C000CCF80823C0F8404108BFCCF80423CCF8FC
:1096D000442370BD881E20F07F40CCF840054FF435
:1096E0008030CCF80803CCF84041CCF84403012B7F
:1096F00014BF002101218C4B597089490D61DFF89D
:1097000034C2CCF800408C4C4FF0020CC4F800C0BE
:10971000DFF828C2CCF80060DFF808C23D32CCF890
:109720000020C1F800524FF0E0224FF4807CC2F8D4
:1097300080C2C1F80403C2F800C10804804908606F
:109740001D7070BD7F4A4FF40030012BC2F84015E8
:1097500018BFCCF80803C2F8404108BFCCF8040396
:10976000CCF8440370BD67480068704770B5764810
:109770000568774975480860614CD4F840010026B7
:1097800001280AD1D4F8080310F4803F05D04FF423
:109790008030C4F80803C4F84061D4F844010128BB
:1097A0000DD1D4F8080310F4003F08D04FF4003076
:1097B000C4F80803C4F84461012007F060FDD4F840
:1097C000480101280DD1D4F8080310F4802F08D0E7
:1097D0004FF48020C4F80803C4F84861022007F061
:1097E0004EFD5C48056070BD574810B50468584987
:1097F000564808604C490878002808BF03201AD052
:10980000464A4FF000401060454AC00BC2F80803BA
:1098100003124FF0E02C0020CCF88031414B18604F
:10982000C2F84001C2F8000208704A78002A1CBF42
:109830004870002001D007F022FD4648046010BDAA
:109840004FF0E0214FF08070C1F8000270474FF0F8
:10985000E0214FF08070C1F8800270474FF0E021A6
:109860004FF40010C1F8000270474FF0E0214FF4B0
:109870000010C1F8800270472949012008614FF0AB
:10988000E0210002C1F880027047410A43F6095204
:109890005143C0F3080010FB02F000F5807001EBAB
:1098A00050207047430B48F2376C03FB0CF31B0C42
:1098B0004FEA432CC1F800C0DFF89CC003FB0C0347
:1098C00026484CF2F72C5843400D10FB0CFC0CEBD7
:1098D000432303F580735B1213700A681044086019
:1098E0007047194810B5046819491848086008F00D
:1098F0005FF81848046010BD0BE000E018E000E0DD
:1099000000B0004004B500404081004044B1004038
:1099100048B1004048B5004040B5004008F501405E
:1099200000800040408500402C00002044B50040ED
:1099300008B00040048500400885004010850040C4
:1099400004F5014004B00040100502400100000190
:109950001805024014050240F7C2FFFF6F0C01001A
:1099600010B5EFF3108000F0010472B6EB484178B7
:10997000491C41704078012801D108F07DFC002C81
:1099800000D162B610BD70B5E44CE07848B901254D
:10999000E570FFF7E5FF08F077FC20B1002008F044
:1099A00053FC002070BD4FF080406571C0F8045337
:1099B000F7E770B5EFF3108000F0010572B6D74CF1
:1099C000607800B9FFDF6078401E6070607808B989
:1099D00008F056FC002D00D162B670BDCF4810B51E
:1099E000C17821B100214171C170FFF7E2FF002071
:1099F00010BD10B5044608F047FCC849C9780840B6
:109A000000D001202060002010BD2DE9F05FDFF8BC
:109A10000C934278817889F80620002589F8071090
:109A2000064689F8085000782F4620B101280FD04B
:109A300002280FD0FFDF08F034FC98B108F038FCA2
:109A4000A8420FD1284608F037FC0028FAD047E09A
:109A50000125F0E7FFF784FF08F016FC0028FBD093
:109A60000225E8E701208407E060C4F80471AC49EE
:109A70000D600107D1F84412A94AC1F342312432E2
:109A80001160A7494FF0020B34310860C4F804B3E9
:109A9000A060DFF890A2DAF80010C94341F300118A
:109AA00001F10108DAF8001041F01001CAF80010C5
:109AB00000E020BFD4F804010028FAD0284608F0BE
:109AC000FBFB0028FAD0B8F1000F05D1DAF800103E
:109AD00021F01001CAF80010C4F808B3C4F80471EA
:109AE00099F807004C4670B1307860B908F0CCFBAB
:109AF000064608F0BDFD6FF0004116B1C4E9031041
:109B000001E0C4E9030115B12771BDE8F09F012010
:109B10002071BDE8F05F00F0DFB870B5050000D13E
:109B2000FFDF4FF080424FF0FF30C2F80803002102
:109B3000C2F80011C2F80411C2F80C11C2F81011D9
:109B4000764C617008F0A6FB10B10120E0706070E7
:109B50002846BDE8704058E72DE9F0410125AF07E0
:109B60007D616E4CE079F0B1012803D0217A401E6E
:109B7000814218DA08F088FB064608F079FDE179A1
:109B8000012902D9217A491C21720EB1216900E014
:109B9000E168411A022902DA11F1020F0EDC0EB15E
:109BA000206100E0E060FFF7DBFE08F06DFB10B124
:109BB0003D61A57000E0257000202072BDE8F081B5
:109BC0002DE9F05F5848D0F800B0574A574908329D
:109BD00011608406D4F8080110B14FF0010801E0CB
:109BE0004FF00008D4F8000100B101208146D4F8FC
:109BF000040108B1012600E00026D4F80C0100B1F0
:109C000001208246D4F8100108B1012700E00027A6
:109C100048EA090126EA010020EA0A00B84300D018
:109C2000FFDF0025B8F1000F04D0C4F8085101206F
:109C300008F00AFBDFF8E480B9F1000F13D0C4F894
:109C4000005198F8050020B188F80550002008F070
:109C5000FBFA98F8000030B108F016FB18B10120AB
:109C600088F8020020610EB1C4F80451BAF1000F67
:109C70000AD0C4F80C5198F80200464600B9FFDF3C
:109C8000B5703570FFF795FE37B1C4F8105198F8EC
:109C9000040008B1FFF760FF2349091DC1F800B0B7
:109CA00033E770B51D4DE87808B908F0E9FA0120EE
:109CB0008407A061A87850B1D4F80C0120B9002025
:109CC00008F0FAFA0028F7D10020C4F80C014FF090
:109CD000FF30C4F8080370BD2DE9F0411926B5071F
:109CE000C5F808630124AC610020C5F80001C5F87F
:109CF0000C01C5F8100108F0C7FA084F10B1BC708C
:109D00002C6100E03C70FFF72BFE0549B87920314B
:109D10000860C5F804636C6150E700003000002063
:109D20001805004010ED00E01005024001000001A0
:109D300010B50D2000F06FF8C4B26FF0040000F011
:109D40006AF8C0B2844200D0FFDF3A4901200860BF
:109D500010BD70B50D2000F048F8374C0020C4F855
:109D600000010125C4F804530D2000F049F82560D6
:109D70004FF0E0216014C1F8000170BD10B50D2056
:109D800000F033F82C48012141600021C0F8001197
:109D9000BDE810400D2000F033B8284810B5046825
:109DA00026492748083108602349D1F800010128D5
:109DB00004D0FFDF2148001D046010BD1D48001DB8
:109DC00000680022C0B2C1F8002108F066FBF1E78C
:109DD00010B51948D0F800110029FBD0FFF7DDFFBE
:109DE000BDE810400D2000F00BB800F01F0201216B
:109DF00091404009800000F1E020C0F880117047D8
:109E000000F01F02012191404009800000F1E02094
:109E1000C0F880127047002806DA00F00F0000F149
:109E2000E02090F8140D03E000F1E02090F8000429
:109E30004009704704D5004000D0004010050240A2
:109E40000100000110B5202000F075F8202000F07E
:109E50007DF84449202081F8000443490006086049
:109E6000091D42480860F7F74DFA3F49C8310860BC
:109E70003F48D0F8041341F00101C0F80413D0F8B2
:109E8000041341F08071C0F80413364901201C39D5
:109E9000C1F8000110BD10B5202000F04CF8324888
:109EA00000210160001D01602F4A481EE83A106041
:109EB0002F4AC2F808032C4BC8331960C2F80001BE
:109EC000C2F860012B490860BDE81040202000F076
:109ED0003DB825492848EC39086070472249264892
:109EE000E8390860704770B51F4A8069E83A22492E
:109EF00011601F49D1F800610023204D1D4A5C1EEE
:109F00001EB1A84206D300210FE0D1F8606186B1EE
:109F1000A84209D2C1F80031C1F860311460BDE82F
:109F20007040202000F012B81168BDE8704014F0B5
:109F3000DCBAFFDF70BD00F01F0201219140400933
:109F4000800000F1E020C0F88011704700F01F028F
:109F5000012191404009800000F1E020C0F880120A
:109F60007047000020E000E000060240441300209B
:109F700000000240000402400100000100F0010066
:109F80004FF0E0214FF00070C1F88001C1F880026D
:109F9000384B802283F80024C1F80001704700B5D7
:109FA00002460420344903E001EBC0031B792BB1C6
:109FB000401EC0B2F8D2FFDFFF2000BD41F83020C4
:109FC00001EBC00100224A718A7101220A7100BDB1
:109FD000294A002102EBC0000171704710B5044608
:109FE000042800D3FFDF244800EBC40420790128B3
:109FF00000D0FFDF6079A179401CC0B2814200D05F
:10A0000060714FF0E0214FF00070C1F8000210BD08
:10A010002DE9F041194805681849194808310860C8
:10A020001448042690F80004134F4009154C0428E6
:10A0300018D0FFDF16E0217807EBC1000279012A72
:10A0400008D1427983799A4204D04279827157F8D3
:10A05000310080472078401CC0B22070042801D312
:10A0600000202070761EF6B2E5D20448001D05607F
:10A07000BDE8F08119E000E0D405002010050240A1
:10A080000100000144000020FE4B586019721A8044
:10A09000C90014F0FCB910B504460E2114F0D5F92E
:10A0A00017202081207B40F00A00207310BD4FF65E
:10A0B000FF720280032008F0E2BC7047027BD307E6
:10A0C00001D1920703D44089088000207047052001
:10A0D0007047027B920700D54181704701460020FE
:10A0E000098847F2FE12114200D00120E549497A61
:10A0F000002901D040F00800704700B50346007BFE
:10A10000C00701D0052000BD19811846FFF7E6FF02
:10A11000C00703D0187B40F004001873187B40F090
:10A1200001001873002000BD027B520700D509B161
:10A130000089704717207047027B61F3C3020273E6
:10A1400070472DE9F04F0E46017804464FF0010BA1
:10A150000BFA01F047F2FF1100EA010961681D46A0
:10A160004FF6FF73088887B09646984206D0B9F13B
:10A17000000F07D047F2FE12104203D0012007B0B3
:10A18000BDE8F08F40EA090008804FF0000A8DB169
:10A1900085F800A02278002705200221102A72D21B
:10A1A000DFE802F0710D323B506A727C50C7C399F0
:10A1B000CBFDFCFB20780B28ECD00420DFE76068A7
:10A1C000B4F80C80007B80077ED5B8F1170F4BD315
:10A1D000F8F7F8FE4045FAD360684089172801D3A4
:10A1E000404541D1287820F03F00801C2870A5F818
:10A1F0000180032030806168A1F80A806068017BDB
:10A2000021F00201017334E104212970A189A5F82C
:10A210000110E189A5F8031085E0A08A3188C01DEE
:10A220001FFA80F84145D2D3062005F8010BA0891A
:10A230002880E0896880208AA88007200090A38A6F
:10A24000A2693EE0082A10D008212970A189A5F84A
:10A250000110E189A5F8031030806A1D694604F1F8
:10A26000100006F0DEFA10B1CCE01021EDE73088E6
:10A270009DF80010084456E00A202870A089A5F82F
:10A280000100032008E006E10C212970A189A5F84E
:10A290000110E189A5F803103080A8E0A089B6F884
:10A2A00000C00BEB40021FFA82F8C44578D3B8F126
:10A2B000050F75D30E222A70CDF800B0226903EA8B
:10A2C0004003208980B200E079E0714600F096FA00
:10A2D000A6F80080CDE06B48427A002A6FD0521E6B
:10A2E00042724068227B236900EBC205AA88286875
:10A2F000D3F800C01044A0F1080240F808CC586818
:10A3000050608DF800108DF801A028680290A88890
:10A31000ADF8040000216846FBF70AFAA5F804A08E
:10A32000002E01D050463080A3E0287840F0800114
:10A330002970287840F040012970E0893188C01CDC
:10A340001FFA80F841455DD3287820F03F00123095
:10A350002870A189A5F80110032000902089E389C5
:10A3600080B27146226900F049FAA6F80080287888
:10A3700041063CD500067CD58DF800B08DF801A0D3
:10A380003188CDE9025A091DDFF8F8800420ADF8C4
:10A390000410049098F8080003E055E04BE02AE030
:10A3A00030E08DF8140000216846FBF7C1F907463C
:10A3B00030880C303080022F02D0DFB36EE047E0EF
:10A3C0009DF81420D8F8041098F80830404601EBA6
:10A3D000C2019A4216D28A88A2B9427A521C88F8DF
:10A3E00009200D6030888880A6F800A056E06168DA
:10A3F000A08988803DE0218A3288491D1FFA81F8B2
:10A40000424501D2042749E0297821F03F01163165
:10A410002970A189A5F80110E189A5F80310009021
:10A420002089238A80B27146626900F0E7F9A6F8B4
:10A430000080DCE71DE0287820F03F00183028700D
:10A44000207B6870318014E060680188090401D4C1
:10A45000052723E0C088A189884201D006271DE096
:10A460001E202870A6F800B06068018821F4004121
:10A470000180B9F1000F11D002480022008883004A
:10A48000032001E0F4050020A16808F05BFA616890
:10A490002078887007E0A6F800A00327606801888C
:10A4A00021EA09010180384669E62DE9F04F87B0BD
:10A4B0009B46119C0D46030016461AD03078C10702
:10A4C00003D000F03F00192801D9012100E000214C
:10A4D0002046FFF729FE98420BD32088A0F57F4144
:10A4E000FF3906D03078410601D4000603D5082094
:10A4F00045E6072043E600208DF800008DF80100B6
:10A5000030785F1E00F03F0C0122981E4FF0050AC4
:10A510004FF00209B9B2BCF1200F76D2DFE80CF09F
:10A520008C10755F7569758D759E75B775BC75CA2C
:10A5300075D675E3757575F375F175F075EF758CF6
:10A54000052B79D104208DF80000A0788DF8040047
:10A550007088ADF8060030798DF80100707800F051
:10A560003F000C2829D00ADCA0F10200092863D2A0
:10A57000DFE800F0126215621A621D6220001228E4
:10A5800024D004DC0E281BD01028DAD11BE01628BA
:10A590001FD01828D5D11FE02078800701E020784F
:10A5A0004007002848DAF0E020780007F9E7207833
:10A5B000C006F6E720788006F3E720784006F0E74B
:10A5C00020780006EDE72088C005EAE72088C0046F
:10A5D000E7E720888004E4E720884004E1E720786A
:10A5E000800729D5032B27D18DF800A0B6F80100EC
:10A5F00082E0217849071FD5062B1DD381B27078E0
:10A60000012803D0022817D102E0CBE0022000E0AD
:10A61000102006228DF8002072788DF80420801C0E
:10A62000B1FBF0F2ADF8062092B242438A4203D168
:10A630000395ADF80890A8E07AE02078000777D578
:10A640000721B8B28DF800108108ADF80410B0EB06
:10A65000810F6DD10295ADF8062096E02178C906EC
:10A6600066D5022B64D381B208208DF80000707883
:10A6700002285DD3B1FBF0F28DF80400ADF806209E
:10A6800092B242438A4253D1ADF808907CE02078E0
:10A6900080064DD5092003E02078400648D50A20E1
:10A6A0008DF80000A088ADF80400ADF80610ADF8F4
:10A6B000082069E02078000672D50B20ADF8041060
:10A6C0008DF80000ADF8062002955EE02188C905EE
:10A6D00066D5022B64D381B20C208DF8000070780F
:10A6E00004285DD3C6E72088C00459D5012B57D173
:10A6F0000D208DF80000A088ADF8040045E021E0B1
:10A7000026E016E0FFE72088800449D5052B47D3D3
:10A710000E208DF80000A088ADF80400B6F8030004
:10A720005B1FADF80830ADF80600ADF80AA02BE0CD
:10A7300036E02088400433D5012B31D10F208DF82D
:10A74000000022E0208800042AD4B6F80100E0804E
:10A75000207B000724D5032B22D3307800F03F0064
:10A760001B2819D011208DF80000208840F40040EB
:10A77000A4F80000B6F80100ADF80400DB1E0320C9
:10A78000ADF80630ADF80800039559466846FAF76B
:10A79000CFFF050008D016E010208DF80000E9E793
:10A7A000072510E008250EE0307800F03F001B2858
:10A7B00009D01D2807D00320109908F060F92088DF
:10A7C00000F400402080207B400708D52046FFF79A
:10A7D00085FCC00703D1207B20F0040020732846AD
:10A7E000CDE400B587B0032806D18DF800000191B3
:10A7F00000216846FAF79CFF07B000BDF8B51C467B
:10A8000015460E46069F04F0A3FC2346FF1DBCB26E
:10A8100031462A46009404F0E2F8F8BD2DE9FF4FD6
:10A820008FB00546DDE91C471198DDF880B0082897
:10A8300005D0E86901F031F950B11020CDE0208851
:10A84000092140F0100020808BF80010022017E052
:10A85000E96901208871EA694FF420519180E96922
:10A860008872E96942F601000881E969002088736D
:10A870002088112140F0200020808BF80010042057
:10A88000814638780B900A2038704FF0020A05F1A3
:10A89000180056460D9001F0A1FB4C467CE0119843
:10A8A00010280DD1022E0BD0AAEB0400801C80B220
:10A8B00000902198022380B206AA1F9901F0DDF8CA
:10A8C000BDF81A101298814203D9F648007A109008
:10A8D00004E003D10B9808B1387031E02198CDF82D
:10A8E00000A080B24FF002030DF11A021F9901F08F
:10A8F000C4F81E980088811BA1EB090083B2C9F13E
:10A90000FF00984200D203460AEB090292B20DF111
:10A910003008029200202199CDF81480CDE903106F
:10A920001F991098CDE9000195F82010BDF81A0084
:10A93000002201F0D5FB387050B1C0B2832803D09B
:10A94000BDF81A00288334E0022013B0BDE8F08F70
:10A95000BDF83000022E00EB0901CCB20CD09BF800
:10A960000110A14205D1BDF82410814206D0FF2C70
:10A9700004D09BF801401EE08BF80140C9480068F4
:10A980000178052902D1BDF81A1081800AEB040074
:10A990001FFA80FA301986B206AB219A10990D98E9
:10A9A00001F01FFB28B91E980088801BA042BFF64B
:10A9B00076AF022E12D0119810280BD1AAEB04000A
:10A9C000801C80B200902198022380B206AA1F99B1
:10A9D00001F053F81E980680002038700020B4E77C
:10A9E0002DE9F8439446089E02460027F06BB0B369
:10A9F000521F94B2B6F84220A2F57F45FF3D05D024
:10AA00008518AD882A44921D95B200E000252A19C8
:10AA1000B6F840800832424522D84219BCF80100FD
:10AA200022F8020BBCF8030022F8020B98B222F8BD
:10AA3000024B8946904604F079FB4FF00C0C4946D6
:10AA400042462346CDF800C003F090FFA6F84250DE
:10AA5000F16B00202944A41D2144088003E001E09B
:10AA6000092700E083273846BDE8F88310B50B8836
:10AA7000B0F840409C420CD9C46BE018048844B143
:10AA8000848824F40044A41D23440B80106000201B
:10AA900010BD822010BD2DE9F0478AB000259046F8
:10AAA00089468246ADF81C5007274DE00698068877
:10AAB0008088000448D4A8F8006008A8CDE90450B4
:10AAC000CDE90075029503954FF4007300224946C5
:10AAD000304601F005FB04003DD1BDF81C00ADF887
:10AAE0002400069908888A88B04216D1130414D429
:10AAF0000595CDE9007522F4004202950395049571
:10AB000042F480434A88494601F0CDF804000BD155
:10AB10000698818841F40041818006AA09A950461F
:10AB2000FFF7A4FF0400DCD00595CDE90075069879
:10AB30000395029504950088BDF82030002249460F
:10AB400001F0B1F8822C06D106AA07A95046FFF7FA
:10AB50008DFF0400AAD0ADF81C5004E0069881884F
:10AB600021F40041818006AA07A95046FFF77EFF25
:10AB70000028F3D0822C03D020460AB0BDE8F0872D
:10AB80000020FAE730B50446C06B85B0002578B1E7
:10AB90000C208DF80000B4F84000ADF80800E06B20
:10ABA0000391019000216846FBF73FFC8DF80050AF
:10ABB00044F83C5F4FF6FF70E080A58005B030BDE3
:10ABC0002DE9F04105460F46E96B0020069E14462C
:10ABD000002911D0012B0FD1324639462846FFF704
:10ABE0005AFF002808D1002C06D0324639462846A4
:10ABF000BDE8F04100F060BFBDE8F081F8B51D464A
:10AC0000DDF818C0DDE907634C1DBCF800E0A4B214
:10AC1000099FA64501D20720F8BDACF800401724D3
:10AC200003F8014B18805A80052000900B46B8B2FB
:10AC30002A46314600F021FF0020F8BD70B50D46D0
:10AC400004464C2113F023FC04F1080044F81C0FC7
:10AC500000204FF6FF712062E184A0842571172047
:10AC6000208514F82C0F40F00A00207070BD4FF6BC
:10AC7000FF720280042007F002BF30B585B00D4698
:10AC80000446FFF77FFF208F38B101208DF80000C8
:10AC9000002168460195FBF7C8FB00202063606334
:10ACA000A0638BE70006002090F84820920703D4A9
:10ACB00040880880002070470620704790F84820A0
:10ACC000920701D5A0F84610704701460020098878
:10ACD0000A0700D5012011F0F00F01D040F002006A
:10ACE000CA0501D540F004008A0501D540F01000E6
:10ACF0004A0501D540F02000090501D540F040008B
:10AD0000704700B5034690F84800C00701D0062000
:10AD100000BDA3F844101846FFF7D7FF10F0760FD8
:10AD200005D093F8480040F0040083F8480013F879
:10AD3000480F40F001001870002000BD90F8482036
:10AD4000520700D511B1B0F8440070471720704782
:10AD500010F8482F61F3C302027070472DE9FF4FCE
:10AD60009BB00600DDE92CB4289F1E9D2A9B25D0B0
:10AD70002878C10703D000F03F00192801D901212C
:10AD800000E000212046FFF7D9FFB04216D3287813
:10AD900041060FD400F03F011E2909D0218811F48B
:10ADA0007F6F0BD13A884AB1A1F57F42FF3A05D0B7
:10ADB000010606D500F03F00122802D004201FB083
:10ADC000C4E5F8491C984FF0000908728DF81890F6
:10ADD0008DF83C900FAA0A602B9A4A60ADF81C903F
:10ADE000ADF850902A789A4602F03F0C0420711F6B
:10ADF00004F118034FF007084FF0030E1693BCF14F
:10AE00001F0F7DD2DFE80CF07C7C107C257CA97CB8
:10AE1000FD7CFC7CFB7CFA7CFD7CF97C7C7CF87CFA
:10AE2000F77C7C7C7C7CF60094F84820B5F8011017
:10AE3000920701D5032E02D08DF8180039E34FF4A4
:10AE40000060ADF8500061808DF83CE0ADF8401036
:10AE5000F1E2052EF0D1B5F801002083ADF81C0019
:10AE6000B5F80310618300286BD0884269D80020B0
:10AE7000A07220814FF6FF706084169801F0AEF842
:10AE800005208AF800000220804601900AAB5A464D
:10AE90001C99169801F0A5F898BB9DF82E00012882
:10AEA00004D002218AF80110102003E001208AF862
:10AEB000010002200490002203A90BA805F0B1FCB8
:10AEC000F0BB9DF80C00049981423CD13A88801C6B
:10AED000A2EB0801814236DB019800901FFA8BF04B
:10AEE00002230DF12A02299900F0C7FD019808F10B
:10AEF0000208801C81B2019117AA03A90BA801E0E6
:10AF0000B8E223E005F08DFC019900911FFA8BF067
:10AF10009DF80C3017AA299900F0AFFD9DF80C00A0
:10AF20000AAB08EB00011FFA81F801995A46084460
:10AF300080B201901C99169801F053F8002801E0A6
:10AF400001E095E0B7D0B8F1020F03D10A208DF8E7
:10AF500018006DE2A7F800806AE2072EFFF46CAFDC
:10AF6000B5F801002083ADF81C00B5F8031061832B
:10AF700000287DD088427BD80120A072B5F805005A
:10AF800020810020A073E06900F087FD78B9E169B5
:10AF900001208871E2694FF420519180E169887243
:10AFA000E16942F601000881E16900208873F01F21
:10AFB00060841D98A062A4F82480169801F00EF811
:10AFC0008AF800800120804602900020ADF82A0017
:10AFD0002BE000BFB8F1010F1DD0E0698079012896
:10AFE00003D1BDF82800ADF80E00029800901FFABA
:10AFF0008BF007E02BE2ADE13BE1DCE025E29FE0F6
:10B0000076E03BE0042303AA299900F036FD02987C
:10B01000001D80B20290BDF82A00ADF80C00ADF81A
:10B020000E0008F104001FFA80F80AAB5A461C997A
:10B03000169800F0D6FF20B93988A1EB0800042843
:10B04000C8D2B8F1010F81D0E0698079012805D01C
:10B05000BDF82810A1F57F40FF3803D1BDF82800C6
:10B06000ADF80E00029800901FFA8BF0042300E068
:10B0700014E003AA299900F000FD6BE7072E02D027
:10B08000152E7FF4D9AEB5F801002083ADF81C0071
:10B09000B5F80320628308B1904201D90120CBE6C4
:10B0A0000120A07200202081A073052E07D0C8B215
:10B0B000691DE26905F096FB00287FF447AF4FF663
:10B0C000FF706084299803A9029781E8010C06A803
:10B0D00014A9CDE900102878002300F03F02204693
:10B0E0001C99FFF79BFB8146208BADF81C009FE16C
:10B0F000032ED4D14020ADF85000B5F801002083D4
:10B10000ADF81C000DF1300C01230021CDF814C066
:10B110000293CDE903B1299A1C99CDE9001239882F
:10B120000022491E8BB294F8201000F0D9FF8DF850
:10B13000180090BB0B208AF80000BDF8300038E002
:10B14000052EACD18020ADF85000B5F80100208369
:10B15000B5F803106184ADF81C00B1F5007F02D989
:10B160008DF81880A5E141F47C4262840DF1280835
:10B1700000214FF0010CCDE90418CDE902CB299B49
:10B180001C99CDE900133988491E8BB294F8201020
:10B1900000F0A6FF8DF8180030B18328A7D1022057
:10B1A000D6E00000000600200D218AF80010BDF84E
:10B1B0002800401C3BE1D10901EB41030EEB830168
:10B1C000B14204D951067FF56AAF00202FE1B5F8EE
:10B1D0000100ADF81C002A78520609D506228DF828
:10B1E0003C202A78120605D500208DF83C0043E16A
:10B1F0008DF83C804FF0030C4FF00008CDF808C0EC
:10B20000CDE903B8DDE91C23CDF81480CDE9002396
:10B21000A6EB010B1FFA8BF394F82010424600F0C6
:10B2200042FD8DF818008DF83C80297849060DD52F
:10B230002088C00506D5208BBDF81C10884201D19E
:10B24000C4F8288040468DF81880F0E0832801D1AA
:10B250004FF002094FF48070ADF85000BDF81C00AB
:10B260002083A4F822B01D98A0620320A08413219B
:10B27000DAE0052EFFF413AFB5F80100ADF81C00BD
:10B28000B4F840207AB3A2F57F43FE3B2CD00822CD
:10B290008DF83C204FF0050C4FF00008CDF808C0A9
:10B2A000CDE903B8DDE91C23CDF81480CDE90023F6
:10B2B00089B241F40043B5F8032094F8201000F05F
:10B2C000F2FC8DF83C804FF400718DF81800ADF859
:10B2D0005010832813D010B3B4F84010A1F57F406C
:10B2E000FE3809D0E5E0FFE70B228DF83C204FF651
:10B2F000FE72A4F84020CDE7A4F84080D9E05B4678
:10B300002A46009430461D99FFF76AFB8DF8180015
:10B3100008B183284CD1BDF81C0020833FE75B4671
:10B320002A46009430461D99FFF75AFB8DF8180005
:10B33000F0BBB4F84210E06B299A431801A80097BB
:10B3400080E8040C5A88998833F8060BFFF756FCFE
:10B3500081466DE095F80180022E75D15FEA080004
:10B3600002D0B8F1010F6FD109208DF83C0007A879
:10B3700000908DF8408094F820104346002220462B
:10B38000FFF71EFC8DF8410000218DF8421058B9DE
:10B39000B8F1010F15D0B8F1000F05D1B4F8401085
:10B3A000A1F57F40FF380CD0B4F8400048B100E070
:10B3B0003EE000208DF83C004FF48060ADF8500076
:10B3C0000EE00FA82B99FBF730F8814600208DF88E
:10B3D0003C004FF48060ADF85000B9F1020F06D088
:10B3E000F8480068807928B18DF8180028E0A4F8A2
:10B3F000188043E0B9F1000F03D081208DF81800C8
:10B400003CE007A8009094F8201043460122204613
:10B41000FFF7D6FB8DF8180059462046FFF7B2FB20
:10B420009DF8180020B919218AF8001001203880F1
:10B430009DF83C0020B10FA82B99FAF7F6FF814642
:10B44000B9F1000F32D019E016E00620F4E42078BC
:10B45000000711D5012E0FD10A208DF83C00E0889D
:10B46000ADF840005946042007F009FB0820ADF86C
:10B470005000AAE65106E9D54FF004092088BDF82E
:10B48000501008432080BDF8500080050CD5B4F85A
:10B490004010A1F57F40FE3806D11D9820631E980C
:10B4A000606326874FF00309484688E49DF818003A
:10B4B00078B101208AF8000029788AF80110BDF8D7
:10B4C0001C10AAF802109DF818108AF80410052024
:10B4D00038802088BDF8501088432080E4E72DE9AB
:10B4E000FF4F97B0804601780120DDE926A488400F
:10B4F0004FF209010840ADF8200021889B46A1F5D4
:10B500007F424FF00009FF3A02D028B1080703D567
:10B5100001201BB0BDE8F08F249E0020054630704E
:10B520001999189A0988ADF84010A6498DF81C00A1
:10B530000A728DF82C000BA808602598486098F8CE
:10B540000000012837D0022809D003287ED13078A6
:10B5500020F03F001D303070B8F80400E08098F80B
:10B560000000022804D1307820F03F001B303070FA
:10B5700094F84800000769D513AB0020CDE9040317
:10B580000721CDE9001B0322CDE9022ABDF84000C6
:10B5900094F82010C01E83B2B8F80400002200F016
:10B5A0009FFD0028D2D1B8F80400A6F80100BDF82C
:10B5B0004C00C01C03E198F805108DF81C1098F899
:10B5C0000400012806D04FF4007902282BD003286C
:10B5D000BCD171E12088B8F8087010F40060ADF8B3
:10B5E000200033D0172F1CD3F7F7ECFCB84218D348
:10B5F000B4F84600172801D3B84212D1307820F0B1
:10B600003F00C01C3070A6F801700320ADF8400068
:10B61000A4F8467094F8480020F0020084F848002E
:10B620006CE1052585E1208808F1080700F4FE603B
:10B63000ADF8200010F0F00F1ED010F0C00F03D0B6
:10B640003888228B9042ECD1B1B900E06BE1B87838
:10B65000C00711D00020B9680290CDE9030107218D
:10B660000590CDE90010FB88BA8894F8201038883E
:10B6700000F019FB0028D4D1BDF8200080284CD060
:10B6800006DC10280DD020280BD040288AD124E0D9
:10B69000B0F5807F6AD048457ED0B0F5806F97D1F5
:10B6A000E2E0C00601D5082000E010208146052018
:10B6B0008DF82C00002008A9ADF8300001AB0091F6
:10B6C00010AA07A883E80508CDE9046A3B884A4622
:10B6D00007212046FFF7A2F8A8E09DF81C004FF0D4
:10B6E0000A0900289CD113ABCDE904030721CDE959
:10B6F000001B0122CDE9022ABDF8400094F8201079
:10B70000401E83B2208B002200F0EAFC8DF81C0062
:10B710000B203070BDF84C001EE09DF81C004FF06F
:10B720000C09002821D115ABCDE904030721CDE98F
:10B73000001B0122CDE9022ABDF84000628C401EA8
:10B7400083B294F82010208B00F0CAFC8DF81C0006
:10B750000D203070BDF85400401CADF840000520AD
:10B760008DF82C00208BADF83000C7E03888B4F895
:10B7700018C060457FF455AF9DF81C004FF01209CA
:10B7800000281ED1A06AB8B1B878C0073FF449AF0D
:10B790000020B968029000E016E0CDE9030107211E
:10B7A0000590CDE90010FB88BA8894F82010604617
:10B7B00000F079FA8DF81C00132030700120ADF8EC
:10B7C00040009BE000060020B7F800C0208B8445B5
:10B7D000D0D19DF81C004FF016090028E06B06D070
:10B7E000F0B30020ADF808004FF6FF7729E078B1FC
:10B7F000B978C907BED1B4F8421010AACDE9002B20
:10B80000CDE9026A43185A88998833F8060B0BE091
:10B81000B878C007BAD010AACDE9002BCDE9026AEA
:10B82000BA88F9886046BB68FFF7E8F9050065D07B
:10B83000072D79D07DE00F4605AA02A92046FFF723
:10B8400015F9B4F84220BDF808108A4201D000284A
:10B85000F1D0B4F84210E26B00201144088000E0FF
:10B860004CE0A4F8427049E09DF81C004FF0180924
:10B8700040B1208BD0B13888208351462046FFF755
:10B8800081F93BE004F118000090237E94F8201029
:10B8900001222046FFF794F98DF81C000028ECD116
:10B8A000192030700120ADF84000E6E7052551462B
:10B8B0002046FFF767F93CE0208800F40070ADF8FF
:10B8C000200048452FD1B4F84000A0F57F41FE3953
:10B8D00090D1D8F808004FF0160958B1E063B8F8D5
:10B8E0000C10A4F840104FF6FF71A4F8421000218C
:10B8F000018003E04FF6FF70A4F84000BDF820007F
:10B9000030F47F611AD0782300225146042007F0DA
:10B9100019F898F8000020712088BDF8201008431D
:10B9200020800EE000E007252088BDF82010884325
:10B930002080208810F47F6F1DD03EE02188814355
:10B9400021809DF82C0028B16F4841680BA8FAF7B8
:10B950006CFD05469DF81C000028EAD086F8019091
:10B9600001203070208B70809DF81C003071052004
:10B97000ADF84000DDE7208FF8B119990988ADF8DE
:10B980004010DDE9242302A9059481E80C0410AAE3
:10B99000CDE9002BD4E90C231899FFF7DFF9054610
:10B9A00001208DF82C0000210BA8CDF830A0FAF76B
:10B9B0003CFD00B105460020208794F84800400770
:10B9C0000AD52046FFF781F910F0760F04D114F85C
:10B9D000480F20F0040020701998BDF84010018035
:10B9E000284696E500B585B0042807D102208DF8D9
:10B9F0000000019100216846FAF717FD05B000BD6F
:10BA000010B5414A03781168012B02D0022B2BD1CB
:10BA100012E00B780BB1052B01D104230B701368D6
:10BA2000818899801168C388CB8013680189198146
:10BA30001168408948810FE083888B801168C38832
:10BA4000CB80136801891981136841895981116874
:10BA500083898B8100690861D2E90001FAF7E5FC6E
:10BA6000022803D0002800D0812010BD832010BD03
:10BA7000C06B002800D001207047F8B51C46154661
:10BA80000E46069F03F064FB2346FF1DBCB2314601
:10BA90002A46009402F0A3FFF8BD8178012909D15C
:10BAA0000088B0F5205F03D042F60101884201D141
:10BAB0000020704707207047F0B589B00024154674
:10BAC0000E460746ADF8184011E007980188298016
:10BAD000811D0294CDE9034107210594CDE90014AD
:10BAE000838842880088314600F0DDF830B907AA23
:10BAF00006A93846FEF7BAFF0028E6D0822800D112
:10BB0000002009B0F0BD00000006002010B58B78C1
:10BB100083B102789A4205D10B885BB102E08B7940
:10BB2000091D4BB18B789A42F9D1B0F801300C88DD
:10BB3000A342F4D1002010BD812010BD072826D0DB
:10BB400012B1012A27D103E0497801F0070102E090
:10BB50004978C1F3C20105291DD2DFE801F00318BD
:10BB6000080C12000AB10320704702207047042815
:10BB70000DD250B10DE0052809D2801E022808D34D
:10BB800003E0062803D0032803D0052070470020D7
:10BB900070470F2070478120704710B513880B80C5
:10BBA0000B781C061FD5F64CA47A844204D843F0C7
:10BBB00010000870002010BD94682478C44064F31D
:10BBC00004130B701378D17803F0030341EA0321C7
:10BBD00040F20123B1FBF3F403FB1411926800FB64
:10BBE0000120401C10BD906810BD37B5BDF8041091
:10BBF00011809DF8045029061BD5E1490123946862
:10BC0000897A814209D8FE280FD1E80602D58B40F7
:10BC10005B1E00E00023237007E0217883409943F6
:10BC2000C5F30013834019432170107820F01000F1
:10BC300010703EBD2DE9F0410746C81C0E4620F0AD
:10BC40000300B04202D08620BDE8F081082A01D965
:10BC50000E20F9E7CA4D002034462E60AF802881BF
:10BC6000AA72E8801AE0E988491CE980810614D4A8
:10BC7000E17800F0030041EA002040F20121B0FB2E
:10BC8000F1F201FB1201206800F021FB2989084430
:10BC900080B22881381A3044A0600C3420784107E3
:10BCA000E1D40020D0E72DE9FF4F87B01646DDE94B
:10BCB000147A8046994623F4404500F0F8FA0400CF
:10BCC0000BD0207800060AD5AD48817A08988142C9
:10BCD00005D887200BB0BDE8F08F0120FAE7224697
:10BCE00001A90898FFF759FF834600208DF8080046
:10BCF000072F1BD0012221463846FFF71FFF0028DF
:10BD0000E8D12078400611D502208DF80800BDF852
:10BD10000400ADF80C80ADF80E00ADF81060169878
:10BD2000ADF81250CDF818A0ADF814005FEA094044
:10BD300004D500252E46A84601270CE02178E0789E
:10BD400001F0030140EA012040F20122B0FBF2F1D0
:10BD5000804602FB11875FEA494009D5B84507D103
:10BD6000A178207901F0030140EA0120B04201D31B
:10BD7000BE4201D90720ADE7A8191FFA80F9B945DD
:10BD800001D90D20A6E79DF8080020B102A8FAF716
:10BD90004AFB00289ED1B84507D1A0784FEA192167
:10BDA00061F30100A07084F80490199800B1058037
:10BDB000189850EA0A0028D0189830B10BEB06000A
:10BDC0002A46189912F0CAFA0FE017980BEB0608EA
:10BDD00080B25746169E03F0A9F92B46F61DB5B260
:10BDE00039464246009502F0C1FD224601A9089855
:10BDF000FFF7D3FE9DF80400224620F010008DF8D6
:10BE0000040001990898FFF7F0FE002062E72DE991
:10BE1000FF4FDFF86C9182461746B9F80610D9F843
:10BE2000000001EB410100EB810440F20120B2FB74
:10BE3000F0F187B000FB11754E46DDF854802946BD
:10BE4000089800F044FA316832898B46611A0C3147
:10BE500001441144B38889B28B4201D8842039E768
:10BE60000899CEB2310603D5B10601D5852031E758
:10BE7000B9F806C00CF1010C1FFA8CFCA9F806C039
:10BE8000169909B1A1F800C0B10602D5C4F808801E
:10BE900007E0104480B2A9F80800191A01EB0B0062
:10BEA000A0602246FE200899FFF79FFEE7702571EB
:10BEB0002078390A61F301002A0AA17840F00400D1
:10BEC00062F30101A17020709AF802006071BAF863
:10BED0000000E08000252573300602D599F80A702D
:10BEE00000E00127B00601D54FF000084E460024BF
:10BEF0004FF007090FE00295CDE903580595CDE90C
:10BF00000095F0882146149B0A9AFFF7CCFE002882
:10BF1000A5D1641CE4B2BC42EDD30020DAE62DE9E1
:10BF2000F047804600F0C3F9070005D000264446DC
:10BF3000134D40F2012916E00120BDE8F0872046AC
:10BF400000F0B5F90278C17802F0030241EA02225A
:10BF5000B2FBF9F309FB1321006800F0B8F9304493
:10BF6000641C86B2A4B2E988601E8142E7DCA8F1B5
:10BF70000100E8802889801B288100203870DCE7D8
:10BF80000C06002020B1401E1080917000207047E8
:10BF90000120704710B5D54904460088CA889042F0
:10BFA00001D3822010BD096800EB400001EB800244
:10BFB0005079A072D08820819178107901F0030126
:10BFC00040EA0120A081A078E11CFFF7E6FD206196
:10BFD0002088401C2080E080002010BD012181824B
:10BFE00070472DE9FF4F83B04FF6FF780546A3F861
:10BFF000008040681F4680788DF8060068680088D9
:10C00000ADF8040000208DF80A00A88A2C88A04210
:10C0100000D30446AC8242E0A88A401CA882701D6E
:10C020006968FFF773FDC0BB3988414501D1601EC7
:10C0300038806888A04237D3B178307901F00301A5
:10C0400040EA012901A9701DFFF760FD28BB69893D
:10C0500041452ED0002231460498FFF76FFDE0B92C
:10C060006989494519D10598D5F810B0B5F80CC0C3
:10C07000D6F808A080B2CDF800C003F057F8DDF87C
:10C0800000C059460CF1070C1FFA8CFC52464B4677
:10C09000CDF800C002F02DFC58B1641CA4B22046BB
:10C0A00000F005F90600B7D1641EAC82822007B00B
:10C0B00011E67C807079B871F088B8803178F078BA
:10C0C00001F0030140EA01207881A7F80C90287A5A
:10C0D000324607F10801FFF760FD38610020E6E70E
:10C0E0002DE9FF4F87B01C46DDE9158B91460F46C1
:10C0F000DDF864A0079800F0DAF8050008D0287889
:10C10000000607D57948807AB84203D88720E1E550
:10C110000120DFE5C9F309062A4601A93846FFF7E1
:10C120003CFD0746149807281BD000222946FFF73C
:10C1300005FD0028EBD12878400612D501208DF8A6
:10C1400008000798ADF80C00BDF80400ADF80E002B
:10C15000ADF81060ADF8124002A8FAF764F90028B3
:10C16000D5D12978E87801F0030140EA0121AA78C5
:10C17000287902F0030240EA02204E4507D0B1F5CB
:10C18000007F04D9611E814201DD0B20A2E58642B9
:10C1900001D907209EE5801B85B2A54200D925461E
:10C1A000BAF1000F01D0AAF80050189818B1B919C7
:10C1B0002A4612F0D3F8B8F1000F0ED017983E447B
:10C1C00080B244465F4602F0C3FF2146FF1DBCB269
:10C1D00032462B46009402F002FC00207AE52DE95D
:10C1E000F0411D4617460E4600F061F8040008D0E5
:10C1F0002078000607D53D48807AB04203D88720D2
:10C2000022E5012020E5224639463046FFF7C5FCED
:10C2100065B12178E07801F0030140EA0120B0F532
:10C22000007F01D8012000E00020287000200BE5ED
:10C230002DE9F0411D4617460E4600F038F804007F
:10C2400008D02078000607D52848807AB04203D865
:10C250008720F9E40120F7E4224639463046FFF70B
:10C26000C4FCFF2D14D02178E07801F0030240EAED
:10C27000022040F20122B0FBF2F302FB130015B9D9
:10C2800000F2012080B2E070000A60F30101217029
:10C290000020D9E410B50C4600F009F828B1C18897
:10C2A00021804079A070002010BD012010BD0F49F1
:10C2B000CA88824209D340B1096800EB40006FF0A0
:10C2C0000B0202EB80000844704700207047C0B2A8
:10C2D000820609D4000605D50448807A4843401CEC
:10C2E00080B2704708467047002070470C06002057
:10C2F0000649012008707047044900200870704703
:10C300000248007800F0010070470000480000205B
:10C3100010B506F09BFD06F008F8F6F7B1FD11F038
:10C320000DF806F06BFCBDE8104006F01DBD10B521
:10C330000C4601F025FF80B3204600F0A8FA68B350
:10C3400022780F2A09D0102A07D0022A05D0032A02
:10C3500003D0142A2ED0FFDF1DE0A0781E282DD098
:10C360000EDC0C2824D008DC092827D2DFE800F0F6
:10C3700013261726261E1E1A1C0012281ED11BE08B
:10C38000302819D01ADDA0F13A00032816D2DFE8D0
:10C3900000F011150B00002010BD13E010E043F277
:10C3A0000200F9E70420F7E70D20F5E70F20F3E797
:10C3B0000820F1E71120EFE70720EDE70320EBE786
:10C3C000FFDFE8E7FFDFE6E700F061BA70B503469C
:10C3D000002002466FF02F050EE09C5CA4F13006B1
:10C3E0000A2E02D34FF0FF3070BD00EB800005EB4A
:10C3F0004000521C2044D2B28A42EED370BD30B508
:10C400000A240AE0B0FBF4F304FB13008D1830306B
:10C4100005F8010C521E1846D2B2002AF2D130BDE6
:10C4200030B500234FF6FF7510E0040A44EA0020FF
:10C4300084B2C85C6040C0F30314604005EA003475
:10C440004440E0B25B1C84EA40109BB29342ECD3C0
:10C4500030BD000010B50AF0CCF8042803D00AF073
:10C46000C8F8052802D108F0DFFD50B90AF07EF9BE
:10C47000032803D00AF080F9032804D107F06FFDE8
:10C4800008B1012010BD002010BD70B50C46054656
:10C49000062102F0E8FC606008B1002006E00721F8
:10C4A000284602F0E0FC606018B1012020700020F6
:10C4B00070BD022070BD2DE9FC470C46064669465A
:10C4C000FFF7E3FF00287DD19DF8000050B107F091
:10C4D000A2FCB0427CD0214630460DF074FA002810
:10C4E00073D115E008F0B9FAB04271D02146304658
:10C4F0000CF090F8002868D1019D95F8C0005035E7
:10C5000018B9687E08B1012000E00020804603E0F1
:10C51000019D95F8698050354FF0010A95F8350076
:10C520004FF00009A0B195F83600800710D584F8C7
:10C53000019084F800A084F80290A68095F8371046
:10C54000A171298F2181698F618185F835903CE047
:10C55000304602F0FDFD070000D1FFDF384601F054
:10C56000F8FF10F0FF0008D084F801900D21217031
:10C57000A680E08084F802A027E0304602F0D6FDD5
:10C58000070000D1FFDFB8F1000F21D0384602F0DC
:10C5900070F8B8B19DF8000038B90198D0F8E400FF
:10C5A0004188B14201D180F80090304607F0F5FA99
:10C5B00084F801900A21217084F80290A680A97E57
:10C5C000A17100E004E085F819900120BDE8FC8726
:10C5D0000020FBE71CB56946FFF757FF00B1FFDFFE
:10C5E000684601F021FEFF4900208968A1F8C200D9
:10C5F0001CBD2DE9FC4104460E46062002F0DEFB80
:10C600000546072002F0DAFB2844C7B20025A846F9
:10C610003E4417E02088401C80B22080B04202D304
:10C620004046A4F8008080B2B84204D3B04202D29F
:10C630000020BDE8FC816946FFF727FF0028F8D0FD
:10C640006D1CEDB2AE42E5D84FF6FF70208012208F
:10C65000EFE738B54FF6FF70ADF800000DE00621AA
:10C66000BDF8000002F011FC04460721BDF80000EF
:10C6700002F00BFC0CB100B1FFDF00216846FFF7B0
:10C68000B8FF0028EBD038BD2DE9F041D6A00679DF
:10C69000076807F0EFFA0EF049FED54C4FF004089A
:10C6A0001020A4F8388060874FF6FF70A4F8560079
:10C6B000002584F85850A4F85A0084F8315004F842
:10C6C000345BCB4904F8065C25702572C4F8097008
:10C6D0003D316673481E0CF021F9A5731B202082A2
:10C6E0004FF4A4716182A082E1820A21217684F84C
:10C6F00019800321A176E1760E2121770721617748
:10C700000621A177E1772084BDE8F08170B5B54CB2
:10C710000D466060217007F028FAFFF79AFFFFF7D7
:10C72000B3FF207809F019FD08F0BCFA21786068A1
:10C730000CF011F820780EF07BF928460AF0CEFBB9
:10C7400007F0A9FB217860680DF0F4F9BDE87040AE
:10C750000EF0ECBD10B501240AB1002010BD21B1CE
:10C76000012903D00024204610BD022110F034F826
:10C77000F9E72DE9F047040000D1FFDF9C4D0026CA
:10C7800095F8310058B166701420207095F8320089
:10C79000A07095F83300E07085F8316068E0287883
:10C7A00040B12C22A91C204611F0D8FD0F2020708A
:10C7B0002E705DE095F82E0060B10120E07095F8D4
:10C7C0002F00A07095F8300060701020207085F860
:10C7D0002E604DE0864802215A308246FFF709FF5D
:10C7E00000B1FFDFB5F85A90062002F0E7FA0746DD
:10C7F000072002F0E3FA3844C7B2781C00F0FF08C3
:10C80000B5F85A00B84212D1204608F0B9F850BB2A
:10C8100095F8340078B36670122020702021A01C97
:10C8200011F013FE0220A07085F8346020E040452E
:10C830001AD1204607F0C4FAE8B12078122817D19F
:10C84000A0783C2814D1A088072102F00CFB050039
:10C8500000D1FFDF288807F0A0F9A088072102F0A7
:10C8600014FB00B1FFDF03E02146FFF724FE10B107
:10C870000120BDE8F087FFE702215046FFF7B9FE2F
:10C8800018B9B5F85A104945BAD10020F1E770E758
:10C8900010B509F0DFFB00B1FFDF0BF056FF00B170
:10C8A000FFDF08F0C9F90AF002FB00B1FFDF0DF06D
:10C8B0003BF900B1FFDF07F0B8FA00B1FFDF0EF07F
:10C8C000B1F800B1FFDFFFF7C4FEFFF7DDFE07F0B0
:10C8D00035F902F01AFC0EF029FD454800210171DE
:10C8E000012141710222C270017010BD10B5404C8F
:10C8F000207828B10A21BDE810400F2001F059BC72
:10C90000FFF7A8FD08B10C2002E00EF055FD002055
:10C910002071012060710A21E170207010BD70B596
:10C92000334D0446287828B1BDE8704032210F20ED
:10C9300001F03FBC207818B1012801D0122010E08E
:10C9400001F044FC20B10EF082FE08B10C2008E09A
:10C95000207801F023FC04F11703E21D611C0EF0A6
:10C9600083FD2871012068713221E970287070BD43
:10C9700070B51F4C0546207828B1BDE870400B21EA
:10C980000F2001F016BC287818B1012801D0122020
:10C990000EE0FFF75FFD08B10C2009E0287801F0F8
:10C9A000FDFB691C0EF0CFFC08B1002000E0072061
:10C9B0002071012060710B21E170207070BD10B5F5
:10C9C0000B4C217829B13021BDE810400F2001F037
:10C9D000F0BB00880EF03EFE302158B100202071DF
:10C9E00009E000004C000020FFFFFFFF1F000000D7
:10C9F00018060020217101206071E170207010BDC7
:10CA000070B5FF4C0546207828B1BDE87040312153
:10CA10000F2001F0CEBB01F0D9FB08B10C2005E0DE
:10CA2000287800F001000EF00FFE00202071012098
:10CA300060713121E170207070BD10B5F04C20782C
:10CA400028B13421BDE810400F2001F0B2BB01F045
:10CA5000BDFB20B10EF0FBFD08B10C2002E00EF092
:10CA60005AFD00202071012060713421E170207096
:10CA700010BD10B5E24C217829B13621BDE8104037
:10CA80000F2001F096BB0378411CA21D18460EF042
:10CA900043FE08B1002000E00220207101206071F7
:10CAA0003621E170207010BD70B5D54C0546207858
:10CAB00028B1BDE8704037210F2001F07ABB2878FB
:10CAC00001F06CFB691C0EF0D3FD022508280AD08A
:10CAD0000EF011FF38B10168C4F80610808860813B
:10CAE0000020207100E02571012060713721E17084
:10CAF000207070BDC248017819B10F21084601F0BD
:10CB000058BB002101710F218170C170FF2181711B
:10CB10004FF6FF710181BB4949680A7882728A88A1
:10CB200082814988C1810121417101707047B449F6
:10CB30000A781AB147210F2001F03BBB0088A1F809
:10CB40005600012081F8580000220A7148714722DE
:10CB5000CA700870704710B5A94C207828B12B21F5
:10CB6000BDE810400F2001F024BB0821A01D05F0F6
:10CB700075FC00202071012060712B21E170207074
:10CB800010BD70B59E4C217829B1BDE870403F21A1
:10CB90000F2001F00EBB90F90000042816D00328E6
:10CBA00014D098B1011D11D010F1080F0ED010F162
:10CBB0000C0F0BD010F1100F08D010F1140F05D08E
:10CBC00010F1280F02D01220207103E0002506F09A
:10CBD0005EFA25713F20E07001206071207070BD09
:10CBE00010B5874C217829B12A21BDE810400F20CB
:10CBF00001F0DFBAA31D012200F110010FF09BFA32
:10CC0000002020710F20A0702A20E07001206071A8
:10CC1000207010BD2DE9FF41794C207828B14621C4
:10CC20000F2001F0C6FABDE8FF814FF0000884F83C
:10CC30000680B4F85600ADF8040002A9FFF725FC01
:10CC400020B1002101A8FFF7D4FCE8BBBDF8040027
:10CC5000ADF8000002A980B2FFF717FC00B1FFDFBA
:10CC6000BDF8000002F074FA050000D1FFDF28468D
:10CC7000039F01F005FD80F0010697F86950BDF8AB
:10CC8000000002F053FA070000D1FFDF384601F040
:10CC9000F0FC80F0010255EA020019D0A179BDF83C
:10CCA000000004EB410108815549A3791831585C13
:10CCB00065F300005854A37962F341005854A279F7
:10CCC00066F38200505400E00DE0A079401CA07192
:10CCD00000216846FFF78DFC28B9BDF80000BDF8BB
:10CCE00004108842B6D1012084F804806071462186
:10CCF000E170207097E770B5414C0546207828B167
:10CD0000BDE8704042210F2001F053BA09F071FCD8
:10CD1000052804D0284609F00DFA002000E00C2078
:10CD20002071012060714221E170207070BD70B5EA
:10CD3000334C0546207828B1BDE8704052210F20C1
:10CD400001F037BA09F076FA80B10AF09DFB68B1BC
:10CD50002878012800D000200DF075FE00202071F9
:10CD6000012060715221E170207070BD0C20F6E747
:10CD700010B5234C207828B10E21BDE810400F20BB
:10CD800001F017BAA11D002006F088FF00202071D5
:10CD9000012060710E21E170207010BD70B5184C3B
:10CDA0000546207828B1BDE8704040210F2001F0F1
:10CDB00000BA01F00BFA38B10C202071012060712B
:10CDC0004021E170207070BD2946002006F053FF1D
:10CDD0000020F2E770B50A4C0546207828B1BDE87E
:10CDE00070403E210F2001F0E4B909F023FA10B998
:10CDF0000AF04AFB90B128780AF0BFF8287803E0DF
:10CE0000180600204C00002008F045F90020207191
:10CE1000012060713E21E170207070BD0C20F6E7AA
:10CE200070B5FF4C0546207828B1BDE87040172149
:10CE30000F2001F0BEB901F0C9F938B10C20207102
:10CE4000012060711721E170207070BD294601201A
:10CE500006F011FF0020F2E738B5F14D04462878BE
:10CE600028B1BDE838404B210F2001F0A2B922794A
:10CE700061798A4215D0A079E379984211D01F2AAE
:10CE80000FD81F290DD80022114610F0B1FD40B96E
:10CE90000022E079114610F0ABFD10B9207A072886
:10CEA00001D9122015E04FF6FF70ADF8000009F02F
:10CEB0005DFCA8B909F060FC90B909F09AFB78B95B
:10CEC00000216846FFF795FB50B1204605F0F8FFBA
:10CED00000202871012068714B21E970287038BD4D
:10CEE0000C20F6E72DE9FC47CD4C054694F82E00C2
:10CEF00028B12821102001F05CF9BDE8FC8728202A
:10CF000084F83000012184F82E10A8784FF0000931
:10CF10001A2825D00EDC162831D2DFE800F0303098
:10CF20003030302130303030303030303030303010
:10CF3000302121212A2822D00BDCA0F11E000C2850
:10CF40001DD2DFE800F01C1C1C1C1C1C1C1C1C1C23
:10CF50001C0D3A38042812D2DFE800F01102110249
:10CF60002888B0F5706F0AD21F20884684F82F00F9
:10CF700028886946FFF789FA18B1022019E01220C3
:10CF800017E09DF80000019F002806D007F1F60782
:10CF9000019E05D106F1DD0604E007F1DC07F7E7A5
:10CFA00006F1F706684601F034F908B1387818B18F
:10CFB0000C2084F82F00A0E787F80080A878307054
:10CFC00084F82F90684601F02FF996E77CB5944CD1
:10CFD0000546207820B125210F2001F0EAF87CBD1C
:10CFE00028886946FFF751FA002160B102202071BC
:10CFF000A1602173E1800F20A0702520E070012046
:10D00000607120707CBD019A1046503282F83E104B
:10D010008368A360037B237392F83E30002BF5D125
:10D020002888E080E7E710B540B10478406813B184
:10D03000B0F8440003E0B0F8460000E0FB201B29F4
:10D0400008D3814206D8B2F5A47F03D340F6480046
:10D05000824201D9122010BD002010BD70B5704C65
:10D060000546207828B1BDE870404D210F2001F021
:10D07000A0B8012666711F2020710F20A0704D20DE
:10D08000E0702670EA88A98833460020FFF7CBFFBE
:10D0900030B900236A8829881846FFF7C4FF08B111
:10D0A000207170BD04F8426FA888E080E888208174
:10D0B000288860806888A0800020207004F83E0CDA
:10D0C00070BD7CB5564D0446287820B13A210F201A
:10D0D00001F06FF87CBD01266E711F2028710F20B2
:10D0E000A8703A20E8702E7020886946FFF7CDF9C5
:10D0F00008B102200DE0A288618801236846FFF78D
:10D1000092FF30B9A288618800236846FFF78BFF41
:10D1100008B128717CBD9DF80010002000290199FC
:10D120000988E9802871019918D081F81961019A5C
:10D130006188A2F81E11019AA188A2F82011019A13
:10D140006188A2F81A11019AA188A2F81C1101990C
:10D1500081F81861019981F819017CBD81F8F160AD
:10D16000019A6188A2F8F610019AA188A2F8F81035
:10D17000019A6188A2F8F210019AA188A2F8F4102D
:10D18000019981F8F060019981F8F1007CBD70B5DA
:10D19000234C0546207828B1BDE870403C210F2083
:10D1A00001F007B8012666710F20A0703C20E070E6
:10D1B00026706A88298833460020FFF734FF30B98B
:10D1C00000236A8829881846FFF72DFF08B12071CF
:10D1D00070BD04F8426F288860806888A080288825
:10D1E000E080688820810020207004F83E0C70BD2B
:10D1F00070B50B4D287828B1BDE870403B210F2059
:10D2000000F0D7BF95F842002C1D00B1FFDFB5F844
:10D2100048006080B5F84A00A0800120607001E0FD
:10D2200018060020002121700F21A9703B21E97010
:10D23000287070BD70B5FE4D287828B1BDE87040EB
:10D240003D210F2000F0B5BFFB262C1DEE8030469F
:10D2500000F0ABFFA080E680304600F0A6FF208102
:10D2600001206070002121700F21A9703D21E9701B
:10D27000287070BD2DE9FC41ED4C064694F82E0057
:10D2800028B11021084600F094FFBDE8FC811F2062
:10D2900084F82F00102084F83000012784F82E70C5
:10D2A00030886946FFF7F1F878B9684600F0B1FFB9
:10D2B00058B1019D9DF8000050350028019806D016
:10D2C00000F58570017841B904E0022006E0D0F84D
:10D2D000E400F7E795F8351019B13A2084F82F00EB
:10D2E000D3E795F8361089070CD1042101709DF819
:10D2F000000020B901993088D1F8E41048806846D0
:10D3000000F092FF002084F82F0085F83570BCE70C
:10D310002DE9F041C64C0546207828B1BDE8F04122
:10D320001D210F2000F045BF1F20207101206071DA
:10D330001D21E170207009F05CF90C2604283CD016
:10D3400005283AD0A9791220012904D019B102295F
:10D3500001D0032926D1297809B1012922D1E979FF
:10D3600029B1012903D0022901D003291AD16988E2
:10D3700043F6FD720B1F3020934213D2AB881B1F64
:10D3800093420FD22187A88860870027A87907F0E9
:10D39000BCFD90B1E87907F00FFE2878012804D091
:10D3A00030B10CE02071BDE8F0810021022001E0E5
:10D3B0000021012007F02FFE08B12671F3E7277145
:10D3C000F1E770B59A4C217829B1BDE870401E2173
:10D3D0000F2000F0EEBE1F212171012161711E227C
:10D3E000E270217002781221012A00D01AB9407827
:10D3F00018B1012801D0217170BD00260C25012A29
:10D4000008D009F0F6F8052802D008F0D0FD40B1A8
:10D41000257170BD07F090FD618F208F08F017FF18
:10D42000F5E7267170BD2DE9F047814C0746B0F84D
:10D430004600B4F844500E46854200D3054600F03D
:10D44000B4FE0146B4F84600814203D8B7F846005E
:10D4500000F0ABFE8046A146B4F84840B7F844005F
:10D46000844200D3044600F0A0FE0146B9F84A0009
:10D47000814203D8B7F8440000F097FE4FF4A4723D
:10D480001B2C01D0904203D11B2D08D0904506D013
:10D49000F580A6F808807480B08001203070BDE867
:10D4A000F0872DE9FC5F0546AFF6C421604ED1E957
:10D4B00000A196F82E00884628B1BDE8FC5F212126
:10D4C000102000F076BE1F2086F82F00212086F85D
:10D4D00030004FF0010B86F82EB0284600F0B2FE67
:10D4E000002811D109F085F805280CD009F081F841
:10D4F000042808D096F8340028B907F0AEFAA0F551
:10D500007F41FF3901D00C20D0E0062101A801F0B5
:10D510007BFC04007ED003210EF044FCB6F85400DE
:10D52000A4F84400B6F85400A4F8460096F84D005C
:10D530000090B6F8541096F84C3020880A4601F056
:10D5400040FD042867D000B1FFDF208806F024FBEF
:10D5500004F10D07B4F800900421384604F07EFF72
:10D56000494638460EF05BFD32A03F1D0068009032
:10D570000321684604F0FDFE002069460A5C3A5427
:10D58000401CC0B20328F9D3288A6080688AA08032
:10D59000A88AE08096F84F2096F84E1020460EF0AC
:10D5A000E2FE014620460EF017FF4FF0000984F816
:10D5B000569084F857904F46687900F0EFFD6076FA
:10D5C000D5F80600C4F81A006889E083C4F808A0FA
:10D5D00084F80C8084F8ECB004F1F0012046FFF7E9
:10D5E00022FF8DF800700121684604F0C2FE9DF80C
:10D5F000000000F00701C0F3C1021144C0F3401065
:10D6000008448DF80000401D2076092801D208301A
:10D61000207601E017E018E0002120460EF0C2FB62
:10D62000287B07F072FCC0B107F086FC697903E043
:10D6300018060020112233002879AA1D07F0C7FC24
:10D64000070016D022E0092030E02088062101F0F2
:10D650001CFC00B1FFDF072028E0208806F09DFABF
:10D660002088062101F011FC00283FF44CAFFFDFB9
:10D6700049E72146032007F0CEFC070006D16A885F
:10D680002988204608F095FD07000CD0208806F078
:10D6900084FA2088062101F0F8FB00B1FFDF86F84C
:10D6A0002F70BDE8FC9F484684F8E09086F82F0074
:10D6B000F7E738B5FD4C207820B122210F2000F08B
:10D6C00078FD38BD1F202071012565712220E07092
:10D6D000257094F8340010BB08F08BFF052805D0A6
:10D6E00007F0BBF9A0F57F41FF3918D00020207169
:10D6F000684608F0E2FD0028E3D10098008806F0B3
:10D700004CFA00980621008801F0BFFB00B1FFDF52
:10D71000E74884F834500078FCF760FC38BD0C20F2
:10D72000207138BD2DE9F041E04D044695F82E00FA
:10D7300028B1BDE8F0412321102000F03ABD1F20A0
:10D7400085F82F00232085F83000012085F82E0071
:10D75000618840F67B438A1F30209A4251D2A288CA
:10D76000961F9E424DD291424BD8E188B1F5FA7F87
:10D7700047D2218940F67746A1F10A03B34240D24D
:10D78000B1EBD20F3DD96189A289914239D84FF0CE
:10D7900000082088062101F066FB06004FF0020712
:10D7A00007D000F028FD20B1D6F8E400017839B99F
:10D7B00002E085F82F70F6E5D6F81011097809B166
:10D7C0003A201EE005218171D6F8E4004146A0F818
:10D7D0000880D6F8E420A0885081D6F8E420E088BC
:10D7E0009081D6F8E4202089D081D6F8E40002891F
:10D7F00043899A4204D88279082A01D89A4203D3ED
:10D80000122085F82F00CEE522884280D6F8E40069
:10D81000077085F82F10C6E52DE9FE43A34C064698
:10D82000207830B103B02421BDE8F0430F2000F090
:10D83000C0BC012565712420E070257030460EF0D3
:10D8400010FC08B1002000E01220207100282BD12C
:10D8500084F83C503068C4F83D00307984F84100C9
:10D860004FF0000884F83C806946062001F087FAF2
:10D8700000B1FFDF684601F060FA98B9BDF80470A6
:10D88000BDF80400062101F0EEFA060000D1FFDF2A
:10D8900086F8EC50684601F050FA18B9BDF804005B
:10D8A000B842EDD184F80480BDE8FE8370B57F4DA9
:10D8B000064695F82E0028B1BDE8704026211020BC
:10D8C00000F077BC1F2085F82F00262085F8300057
:10D8D000012085F82E003088062101F0C4FA0400EA
:10D8E00007D000F088FC20B1D4F8E400017831B909
:10D8F00001E002200CE0D4F81011097809B13A20B7
:10D9000006E005210170D4F8E4103088488000203A
:10D9100085F82F0070BD6548017819B106210F20E8
:10D9200000F047BC002202710F2181700621C170F6
:10D93000C0F80620C0F80A20F1218171012141714F
:10D94000017070472DE9F041584D064695F82E00BC
:10D9500028B1BDE8F0412C21102000F02ABC1F2086
:10D9600085F82F002C2085F83000012085F82E0046
:10D970003088062101F077FA040007D000F03BFC64
:10D9800020B1D4F8E410087830B901E0022026E094
:10D99000D4F81001007808B13A2020E08C2000274C
:10D9A000005D10F0010F19D0D6F802004860D6F8DB
:10D9B0000600886054F8E40F718910228181206884
:10D9C00006F10C010E3010F0C9FC2168032008702C
:10D9D00021683088488085F82F70E4E40C2085F8B1
:10D9E0002F00E0E470B5314D04460C26287828B1AC
:10D9F000BDE8704018210F2000F0DBBB08F0B6FE38
:10DA000003284BD008F0B8FE032847D0A07908B10E
:10DA100001282DD1607928B1012803D0022801D036
:10DA2000032825D1A07B28B1012803D0022801D0EA
:10DA300003281DD1607BD8B1C00819D162884FF48A
:10DA40008040824202D82188814203D9207901286E
:10DA50000ED118E0207930B1012814D0022805D069
:10DA6000032805D102E0202A0BD30CE0A0290AD21A
:10DA70002079042805D12088202802D36188884293
:10DA800001D912260AE0607906F070FA30B12079E7
:10DA900085F83600204606F0D3FA064601202E719E
:10DAA00068711821E970287070BD00001806002008
:10DAB0004C00002010B5FE4C217829B11A21BDE898
:10DAC00010400F2000F075BB01781F2902D91220E9
:10DAD000207106E0002121710278411C104606F0F9
:10DAE00026FB012060711A21E170207010BD10B575
:10DAF000EF4C217829B12021BDE810400F2000F023
:10DB000058BB01781F2902D91220207106E000219C
:10DB100021710278411C104606F0F8FA012060716C
:10DB20002021E170207010BD2DE9FC41E04C2178EE
:10DB300029B1BDE8FC411B210F2000F03ABB0127B1
:10DB400067710C21217100780026012804D000287B
:10DB500079D01220207190E006F0D2F9002819D077
:10DB600006F017FA94F83600A8B1012813D004285B
:10DB700011D008F001FE00287FD108F0F7FD18B1A0
:10DB800008F0F4FD022878D1002009F0F9F900B17D
:10DB9000FFDF267171E008F0E9FD00286DD108F083
:10DBA000EBFD002869D106F036F9A0F57F41FF3979
:10DBB00063D1072101A801F027F9BE490546886015
:10DBC000280000D1FFDF032128460DF0EDFF284695
:10DBD00006F0E1FB34F8540FA5F8440034F80409CA
:10DBE000A5F84600E278A17828460EF027FC014609
:10DBF000002228460EF05BFC6078009014F8043B8D
:10DC0000288834F854190A4601F0DBF980B1042859
:10DC100000D0FFDF2888072101F037F900B1FFDFCE
:10DC20000720207105F58C712846FFF7FCFB24E0E6
:10DC3000288805F0B1FF284609F0A2F900B1FFDFFE
:10DC40002671EFE7FFE708F091FD032803D008F005
:10DC500093FD032811D108F08CFD0546002009F042
:10DC6000B2F850B9267145B1288805F096FF28888A
:10DC7000072101F00AF900B1FFDF1B20E0702770D7
:10DC8000BDE8FC812DE9F041894C0646207828B199
:10DC9000BDE8F0412D210F2000F08BBA308807211C
:10DCA00001F0E1F805004FF0010720D095F8F900E8
:10DCB00040B995F85C00112801D0122802D195F8DE
:10DCC000360150B10C2020710F20A0702D20E07083
:10DCD0003088E080677127706DE51022B11C05F176
:10DCE000FA0010F03BFB85F8F9700020EBE702200A
:10DCF000E9E770B56E4C0546207828B1BDE8704064
:10DD00002E210F2000F055BA2888072101F0ABF82A
:10DD1000022178B190F8F9202AB990F85C20112AF4
:10DD200004D0122A02D00C20207104E080F8F910EF
:10DD30000020F9E721710F20A0702E20E0702888C4
:10DD4000E080012060712070AEE62DE9FC47584C60
:10DD50000646207828B138210F2000F02AFABDE8C5
:10DD6000FC8770884BF68032122190420AD848B165
:10DD70004FF0000830886946FEF787FB20B102208B
:10DD8000207110E021710EE0019800F15009851C0E
:10DD90002F887288394648460DF0FCFE2888B84224
:10DDA000F6D184F80480012060713821E170207080
:10DDB000D5E77CB53E4C0546207820B145210F20A3
:10DDC00000F0F7F97CBD28886946FEF75EFB38B1A4
:10DDD00002202071012060714521E17020707CBD1E
:10DDE00001987F22014680F8582080F859200022AF
:10DDF00080F85A20A87801F8280FE8784870287928
:10DE000088702271E6E71CB5294C217821B11321D5
:10DE10000F2000F0CEF91CBD00886946FEF735FBE7
:10DE200008B1022005E0019890F82810012902D0DD
:10DE30000C20207106E0582100222271095C217219
:10DE40000088E080012060711321E1700F21A17032
:10DE500020701CBD2DE9F041154C0546207828B1F5
:10DE6000BDE8F04143210F2000F0A3B9A87808B124
:10DE7000012803D1A888B0F5FA7F01D912202071BA
:10DE80002888072100F0EFFF0126C8B1002780F89D
:10DE9000F070A988A0F8F21080F8CC60A978012968
:10DEA00000D0002180F8F01090F8CD0030B103E0F0
:10DEB000180600204C00002009F0AEF9277101E09F
:10DEC0000220207166714320E070267073E42DE912
:10DED000F041FE4C0546207828B1BDE8F0414821CC
:10DEE0000F2000F066B92888072100F0BCFF01234D
:10DEF00058B382886D88C688418803EB4207BD42CB
:10DF000017D342F210777E43BF107943B6FBF1F18D
:10DF1000491E89B24FF4FA76B14200D931468D429A
:10DF200000D22946491C521CB1FBF2F15143491E53
:10DF30008AB290F8221101B90284E2800020207197
:10DF400063714820E070237035E40220F7E770B574
:10DF5000DE4C0546207828B1BDE8704049210F20ED
:10DF600000F027B92888072100F07DFF90B1A9783B
:10DF700011F0010180F8CF1004D090F8CD0008B165
:10DF800009F04AF900202071012060714921E170F7
:10DF9000207089E50220F6E770B5CC4C0546207864
:10DFA00028B1BDE8704041210F2000F002B908F00F
:10DFB000DDFB08B10C2017E0297889B10A290FD0C0
:10DFC00014290DD01E290BD0282909D0322907D0B9
:10DFD0004B2905D0642903D0FF2901D0122003E08A
:10DFE000284609F08AF80020207101206071412143
:10DFF000E170207058E5B5490A781AB14E210F201A
:10E0000000F0D7B8427862B1827852B1C27842B19A
:10E01000027932B1C2881B2A03D303781BB1012BCA
:10E0200001D0122007E0A1F854200278D0F80100B6
:10E0300042B1086500200871012048714E22CA7063
:10E0400008707047C864F5E710B5A04C207828B177
:10E050004F21BDE810400F2000F0ABB808F0EAF8FF
:10E0600040B109F011FA28B10AF05CFC0BF054FD44
:10E07000002000E00C202071012060714F21E17030
:10E08000207010BD10B5914C207828B15021BDE80A
:10E0900010400F2000F08DB808F0CCF840B109F026
:10E0A000F3F928B10AF04DFB0BF03AFD002000E037
:10E0B0000C202071012060715021E170207010BD92
:10E0C00070B5824C0546207828B1BDE870405121DA
:10E0D0000F2000F06EB8287800F0010008F018F961
:10E0E000287800F0010009F060F80020207101207C
:10E0F00060715121E1702070D6E470B5734D044613
:10E10000287828B1BDE870404C210F2000F051B8AC
:10E1100000F05CF808B10C200DE0601C0DF0E4FB91
:10E12000207800F0010005F030FF207800F00100B9
:10E1300006F0FEFE00202871012068714C21E97074
:10E140002870B1E470B5614C0546207828B1BDE86F
:10E1500070404A210F2000F02CB808F007FB10B9DE
:10E1600008F00AFB08B10C2003E0287805F0EFFF67
:10E1700000202071012060714A21E170207093E439
:10E1800010B50178532907D2514A52F8211019B11C
:10E19000801C8847012010BD002010BD18B1022846
:10E1A00001D00120704700207047C000703080B25D
:10E1B0007047464A92F83130002B06D182F832007F
:10E1C00082F83310012082F83100704710B508F052
:10E1D00010FA04280DD008F00CFA052809D008F030
:10E1E000C5FA032805D008F0C7FA032801D000209B
:10E1F00010BD012010BD90F8691041B990F8C01011
:10E2000029B190F8C000042801D0012070470020F7
:10E2100070470178406821B190F8690010B1002082
:10E220007047E8E7012070470178012909D140686B
:10E2300090F8CD10002904D0002180F8CD1008F00E
:10E24000EBBF704710B5038843F6FD711A1F8A4271
:10E2500023D24288141F8C421FD29A421DD8C289F1
:10E2600040F67B43911F994217D2018A8C1F9C4232
:10E2700013D28A4211D8428AB2F5FA7F0DD2828A2D
:10E2800040F67744A2F10A03A34206D2B2EBD10FC3
:10E2900003D9C18A028B914201D9302010BD017986
:10E2A00011B1012910D107E0417929B1012903D029
:10E2B000022901D0032907D1007B58B1012809D0D8
:10E2C000022807D0032805D0122010BD1806002010
:10E2D00040E801000020F8E73F3070470844C01DC7
:10E2E000424301F13F00104480B2704770B51D46B3
:10E2F0000446A818049BC01D00FB03F205F13F0073
:10E30000104486B2B14238BFFFDF1E21204610F014
:10E310009CF8A6F11E0080B2A5756080B0F5004F94
:10E3200088BFFFDF608805F13B01884238BFFFDF0F
:10E330006088401BA0F13B011B2934BF1B203B38E8
:10E34000208070BD408870472DE9F04F0D46C18890
:10E35000044600F11E08008921F4004320F4004225
:10E3600021F4004620F400474FF0010A4FF0000965
:10E370009A4208D100F4004001F4004188421CBFD9
:10E380000020BDE8F08FB7420BD9A17DB81B401A21
:10E39000C01F85421BDC08EB060000210580418080
:10E3A0001EE06088A17D801B401AB0F1070B0ED4DF
:10E3B000BBF11B0FB8BFFFDF5D45D4BF29461FFA75
:10E3C0008BF1681A0204120C18BFBA4204DD84F8FB
:10E3D00014900020BDE8F08F08EB06000180428019
:10E3E00084F814A0BDE8F08F2DE9F041044600F157
:10E3F0001E02C08820F40043207D002808BFBDE82D
:10E40000F081D0180288438813448B423CBF00201F
:10E41000BDE8F081002791429CBF0180478013D95D
:10E42000891A0D042D0C45800ED0E088A61D20F41D
:10E430000040854288BFFFDF30884FF4004121EA69
:10E4400000002843308009E0A27D0088D31D1044DD
:10E45000C01D81B26288A01D00F044FB2775012019
:10E46000BDE8F08130B4B0F804C0C488034600F1C0
:10E470001E052CF400402844A44503D10020188236
:10E4800030BC7047B3F80CC00488A44509D3408859
:10E49000ACEB040CA0EB0C0084B20CEB0500C01E2E
:10E4A00006E0A4EB0C049D7DA4B2AC446044001DC6
:10E4B000B1F800C0A44588BF0C80B3F80CC0BCF113
:10E4C000000F0CBF4FF0010C4FF0000C82F800C0A1
:10E4D0000988198230BC70472DE9F041044600F1EB
:10E4E0001E01808820F400404518208A002808BFBB
:10E4F000BDE8F081A189084480B2A08129886A889A
:10E500001144814238BFFFDF28886D88A2894119F4
:10E510000027914219D175B1A088261D20F4004032
:10E52000A84238BFFFDF30884FF4004121EA0000E5
:10E530002843308008E0A27D1044C01D81B2D31D65
:10E540006288201D00F0CEFAA78127820120BDE855
:10E55000F0812DE9F0474189B0F804800027044696
:10E5600000F11E0A414518BF4FF400493AD000BFE0
:10E5700021F40040504446886EB1608904F10A05D8
:10E5800020F40040B04238BFFFDF288829EA0000AD
:10E590003043288021E0A37D008803F1070C184454
:10E5A0006389C01D23F400456288284480B204F1C9
:10E5B0000A0190420BD2121A92B20CF11B0C624566
:10E5C0002CBF03F4004229EA030004D204E0801ABD
:10E5D00080B229EA030210430880781C618987B25F
:10E5E0004145C5D13846BDE8F0872DE9F047B0F880
:10E5F00008800B46044600F11E01B0F80A9080889E
:10E6000028F4004C01EB0C05804504BF0020BDE858
:10E61000F087002A1CBF281D106023B1A27D291D90
:10E6200018460FF09BFE2F886D888DB1E81987B2D0
:10E63000208904F1080620F40040A84238BFFFDF1B
:10E6400030884FF4004121EA00002843308009E07F
:10E65000A07D6288C119C91DC31D89B204F10800DB
:10E6600000F040FAC84504BF208960813846BDE803
:10E67000F0878188C08881420CBF0120002070474C
:10E680008188008988420CBF01200020704730B487
:10E690008488C28800F11E0324F4004C22F4004157
:10E6A000634494421BD08289048A15191C885A88B5
:10E6B000A3189D4216D312B18A4210D212E0837D74
:10E6C0000CF1070C1A196244408892B2801A80B289
:10E6D0002233984201D211B104E08A4202D130BC07
:10E6E0000020704730BC012070472DE9F007B0F8DA
:10E6F00006C0048900F11E0702462CF400457E196D
:10E7000024F400492CF4004A002024F400434FF084
:10E710000108D1450AD104F400440CF4004C6445CE
:10E7200004D05082BDE8F00700207047AB4207D903
:10E7300092F816C05B1BA3EB0C03DC1F002308E060
:10E74000B2F802C0947DACEB050CACEB040CACF160
:10E750000704002CE5DBB2F80EC0BCF1000F0DD0B1
:10E76000B6F800C075884DB15B1B50758B42D8DB85
:10E77000D0893844A0EB0C00C01E09E0A4EB0C04C7
:10E7800050758C4208DB907DD38918443044001DBD
:10E790005182BDE8F00770478B42A8BF82F8158010
:10E7A000E6DABEE72DE9F05F044600F11E0AC088F4
:10E7B000934620F400400AEB0005608A894608B1C0
:10E7C000484502D20020BDE8F09FE089002804BF40
:10E7D0004FF00008464607D0B5F800806E8808EB79
:10E7E0000601884218BFFFDF607D4FF0000750EA46
:10E7F000060101D048B332E0E08938B1A17D01447F
:10E800004819B4F817108180617E8171E18908EBA5
:10E8100009004944E18128806F80BBF1000F0BD0D3
:10E82000A07D2988C31D0144C91D89B26288A01D2D
:10E8300000F058F9E78137E0A07DE18908442844D9
:10E840008188A4F8171080792DE0E089B4F81710BA
:10E850005044A0EB080020F8031D617E817006EB98
:10E86000090086B2E089BBF1000F4844E081A5F8B9
:10E8700000806E800ED0E088A51D20F40040B042DC
:10E8800038BFFFDF28884FF4004121EA0000304301
:10E890002880CFE7E0895044A0EB080030F8031D42
:10E8A000A4F8171080786076678227750120BDE88C
:10E8B000F09F01461E308A88CB8822F4004C6044C9
:10E8C0009A4203D08989002908BF70470020704709
:10E8D00000F11E03807D01F1040C60441060088883
:10E8E000002804BFD81E106008884988084480B2F8
:10E8F00070472DE9F04115460A4600F11E061C46F8
:10E90000807D131D034410885788069900281CBF7A
:10E91000C01C80B226D088429CBF081A80B213D98E
:10E92000401AA042A8BF20461FFA80F85818424655
:10E9300029460FF0E7FC002818BFBDE8F0814544E8
:10E94000A4EB080084B2002001198F423CBF4FF0B5
:10E95000FF30BDE8F081304422462946BDE8F04151
:10E960000FF0D0BCFA1C97B2F61ED4E72DE9F041A7
:10E9700000F11E071D46807D0B1D034416460888C6
:10E980000024B1F80280069A00281CBFC01C80B287
:10E990001FD090429CBF101A80B20DD9801AA84295
:10E9A000A8BF284684B29918224630460FF0D6FCFC
:10E9B000281B85B2264400204119414506D8391844
:10E9C0002A4630460FF0CAFC601984B22046BDE8E2
:10E9D000F08108F103011FFA81F8FF1ED9E72DE944
:10E9E000F04116460A4600F11E071D46807D131DA4
:10E9F000034410880024B2F80280069900281CBF46
:10EA0000C01C80B21FD088429CBF081A80B20DD9AA
:10EA1000401AA842A8BF284684B258182246314658
:10EA20000FF09CFC281B85B226440020411941456B
:10EA300006D838442A4631460FF090FC601984B25B
:10EA40002046BDE8F08108F103021FFA82F8FF1E9C
:10EA5000D9E770B5044600F11E01C288808820F411
:10EA600000431944904205D0A289002A04BF228A9B
:10EA7000002A01D0002070BDB1F800C04D8885B1DA
:10EA8000261D20F40040A84238BFFFDF30884FF435
:10EA9000004121EA0000284330800020208201202C
:10EAA00070BDA07D0CF10701C31D084481B26288CE
:10EAB000201D00F017F8F0E70021C1814175418267
:10EAC0000175704703881380C289002A04BF0020A3
:10EAD0007047C28800F11E0322F400421A440A6003
:10EAE000C089704710B4B0F800C02CF40044214431
:10EAF00089B24FF4004491420AD2521A92B21B33A7
:10EB00009A422CBF0CF4004224EA0C0104D204E027
:10EB1000891A89B224EA0C021143018010BC7047A3
:10EB20002DE9F04188464FF6FC7102F103021E46C2
:10EB3000040002EA010509D00027E01C20F00300D0
:10EB4000A04200D0FFDF201D01210CE00127F4E7E7
:10EB5000024628442FB9B14201D2034600E0002307
:10EB60001360491CC9B2B142F2D9011BC8F80010A8
:10EB7000002F04D10EB1201D00E000202060BDE870
:10EB8000F081024600201168002902D00846096879
:10EB90001160704702680A60016070474FF6FC73AD
:10EBA000C91C1940101A001F90FBF1F0C0B2704749
:10EBB0004FF6FC73C91C1940001D01FB0200704791
:10EBC000F8B5D24D04460E46A878A04200D8FFDF23
:10EBD00005EB8607B86A50F8240000B1FFDFB8687B
:10EBE000FFF7CFFF05000DD0B86A062E40F824507D
:10EBF0000AD0082E00D3FFDFC548294650F826204A
:10EC0000204690472846F8BDC048C24B7A30A0F154
:10EC10002E0200902946204609F0E6FCF2E72DE995
:10EC2000F84F8046DDF828901E4603EB0900934616
:10EC30008A46C4B25FEA080707D00025FF2800D93A
:10EC4000FFDFBAF1000F03D101E00125F6E7FFDF96
:10EC500008F1030020F00301414500D0FFDFCB4560
:10EC600000D9FFDF65B9A94A00204C324FF6FF7189
:10EC700010705180A74A1070A44A7A3210705180E7
:10EC8000A24880F800B046708470C470047144716A
:10EC900080F80690DFF878B2C67100260BF1400BC1
:10ECA0008146FF1C27F003000746002D02D109EB27
:10ECB000860188603BF8162019F8063001D04FF025
:10ECC00000006946FFF72CFF0098761CF6B2074457
:10ECD000082EE6D3FF1C27F003002346064675B135
:10ECE000002002226946FFF71BFF00983118002020
:10ECF00003464E46C91C21F003021DB110E0C9F8BD
:10ED00004800EEE706EB80070021BA6206E000BF8C
:10ED1000D7F828C04CF82130491CC9B2A142F7D31A
:10ED2000401CC0B202EB84010828E3D3A1EB080029
:10ED3000AAF800000020BDE8F88F10B5044603F0E3
:10ED400005FF08B1102010BD2078704A618802EBE1
:10ED5000800092780EE0836A53F8213043B14A1C58
:10ED60006280A180806A50F82100A060002010BD60
:10ED7000491C89B28A42EED86180052010BD70B569
:10ED800005460C46084603F0E1FE08B1102070BDB0
:10ED9000082D01D3072070BD25700020608070BD54
:10EDA0000EB56946FFF7EBFF00B1FFDF6846FFF7DE
:10EDB000C4FF08B100200EBD01200EBD10B50446F1
:10EDC000082800D3FFDF5148005D10BD3EB5054661
:10EDD00000246946FFF7D3FF18B1FFDF01E0641C90
:10EDE000E4B26846FFF7A9FF0028F8D02846FFF7ED
:10EDF000E5FF001BC0B23EBD44498978814201D97C
:10EE0000C0B27047FF2070472DE9F0410C4605461F
:10EE1000062901D0072C10D13C4FB86CFFF7B1FE8A
:10EE200002004FF6FF7604D00221B86CFFF7B6FE61
:10EE300000E030462880B04202D10020BDE8F081D9
:10EE40002146FFF7BDFE040002D1288800F050F8EB
:10EE50002046F3E7A0F57F42FF3A01D0082901D30D
:10EE600000207047ACE6A0F57F42FF3A0BD008299E
:10EE700009D2264A9378834205D902EB8101896A37
:10EE800051F820007047002070472DE9F0410446FA
:10EE90000D46A4F57F4143F20200FF39CED0082D84
:10EEA00001D30720CAE719494FF000088A78A24227
:10EEB000C4D901EB85072146BA6A52F82460002EB6
:10EEC000BCD0134A08462032314652F825209047DC
:10EED000B96A062D41F8248001D0072D02D12046C1
:10EEE00000F006F83146B868FFF754FE0020A5E7A9
:10EEF00010B5064CC2B20221A06CFFF759FE0146C4
:10EF0000A06CBDE81040FFF745BE0000740600206D
:10EF10008CE901005800002001469F48002200684B
:10EF20000260037A00EB830040F80C2F81801146C9
:10EF300000F022B92DE9F05F9846DDF830B0DDF839
:10EF400028A01546894604004FF0000623D000276C
:10EF5000E01C20F00300A04200D0FFDF65B30120D9
:10EF6000FFF7BAF900FB05620AEBCB001618012087
:10EF7000FFF7B2F900FB05620B9805EB450108EBC2
:10EF8000C000104400EB4100143000EB850000EBA2
:10EF9000850617B110E00127DAE77F48A6EB850761
:10EFA000A9000460257204F10C000C3F60600FF0B2
:10EFB0006EFAB8B2FFF7B0FF0020C9F80060BDE8F4
:10EFC000F09F2DE9FF4F744C814681B020689A462E
:10EFD0008B4600B9FFDF2068027A4A4503D94268B0
:10EFE00052F8291021B143F2020005B0BDE8F08FBC
:10EFF000006800B9FFDF01210E9A0398FFF76EF950
:10F00000C61C4FF6FC752E40584601215246FFF7AC
:10F0100065F9C01C00EA050808EB0600001D85B272
:10F020005D4800270068046801E027460446206820
:10F0300038B1A188A942F8D13946204600F0A4F899
:10F0400013E005F10800A18880B2814229D3394636
:10F05000204600F099F8A0880022411B6019026048
:10F060008180394600F088F8A580A08860802680DD
:10F07000251D0E9F0123039A314628460097FFF76E
:10F0800035F92088414628445A460123CDF800A08E
:10F09000FFF72CF9404800684168002041F82940FA
:10F0A000A3E70420A1E770B53B4C0546206800B9F2
:10F0B000FFDF2068017AA94210D9426852F8250082
:10F0C00060B14188002342F82530036081801946F1
:10F0D00000F052F8216800200A7A08E043F20200AA
:10F0E00070BD4B6853F820306BB9401CC0B28242EF
:10F0F000F7D8002002E08A88104480B2096800290D
:10F10000F9D1FFF709FF002070BD70B5224D2868C6
:10F1100000280AD0002404E02046FFF7C4FF641C46
:10F12000E4B22868007AA042F6D870BD70B51A4ED5
:10F1300005460024306800B9FFDF3068017AA94233
:10F1400004D9406850F8250000B1041D204670BD68
:10F1500070B5114E05460024306800B9FFDF3068F5
:10F16000017AA94206D9406850F8251011B131F84A
:10F17000040B4418204670BD19B10A68026008608B
:10F18000704705490968F8E7006809B108607047E9
:10F1900001490968FAE700006000002070B50446E4
:10F1A00000780E4601281AD0072802D00C281AD160
:10F1B00015E0A068216905780B2D0CD0052003F01F
:10F1C0005EFC052D0FD0782300220520D4F8101006
:10F1D00003F0B8FB07E0782300220620F8E70520BB
:10F1E000216903F04CFC31462046BDE8704001F037
:10F1F000A7B910B500F13902C3799478411D64F0C4
:10F2000003042340C371DB070DD04B7954792340AD
:10F210004B710B79127913400B718278C9788A424D
:10F2200000D9817010BD00224A710A71F5E741785A
:10F23000012900D00C21017070472DE9F74F86B0ED
:10F2400000208C690D468DF8040009780127FA48E2
:10F2500016464FF0070A4FF011094FF00A0B2A2902
:10F2600078D2DFE811F02A00110352036903A803E2
:10F27000B303CC03FA030F043B04620481049A0431
:10F28000D504E604050510053005540577059C05F1
:10F29000C605E005EE050F0627063006630685065F
:10F2A000D6060D071B074B076A0779078A07C407AD
:10F2B000FB072708E407E807ED0714B120781D28AD
:10F2C00029D0D5F808805FEA080043D001208DF8E6
:10F2D0000400686A059003208DF808008DF809B0D5
:10F2E000286A0390A8880028EFD098F8001091B100
:10F2F0000F2910D27ED2DFE801F07D144CDCFDFC3A
:10F30000FBFAF9F8F7089FF6F500022822D124B19C
:10F3100020780C2801D0002770E302208DF804002B
:10F32000ACE10620696A03F0AAFBA8880728EDD1A2
:10F33000204601F000F9022809D0204601F0FBF830
:10F34000032808D9204601F0F6F8072803D2012047
:10F35000207005E011E2002CB7D020780128D5D12B
:10F3600098F80400C11F0A2903D300BF85F81CB018
:10F3700089E2A070D8F80010A163B8F80410A18742
:10F3800098F8060084F83E000120287003202070C1
:10F3900046E00728BAD1002C97D020780D28B5D1A7
:10F3A00098F8031094F83B20C1F3C000C2F3C002E8
:10F3B000104201D00E2000E00F20890707D198F8F5
:10F3C00005100142D2D198F806100142CED194F82E
:10F3D0003D2098F8051020EA02021142C6D194F8A7
:10F3E0003E2098F8061090430142BFD198F80400DF
:10F3F000C11F00E045E20A29B8D2617F814201D9EC
:10F400000620C2E3D8F800106160B8F8041021812A
:10F4100098F80600A072012028700E2020700320AA
:10F420008DF80400686A059004F139000290601DAF
:10F4300003901730049067E2412890D1204601F0F4
:10F440007AF8042802D1E078C00704D1204601F000
:10F4500072F80F289ED1A88CEF6880B24FF0400A56
:10F46000D4F82480FFF762FE394608274246534607
:10F470000097FFF77BFA0E208DF80400686A05906C
:10F48000606A0290002101A8FFF788FE2078042816
:10F4900006D0A07F38B1012805D0032806D0AEE3FE
:10F4A000052020700BE284F8009034E712202070D1
:10F4B00066E01128C1D1204601F03DF8042802D1B0
:10F4C000E078C00719D0204601F035F8062805D1AC
:10F4D000E078C00711D1A07F02280ED0204601F0AD
:10F4E0002AF808E0AFE07DE09AE16EE14EE106E146
:10F4F000E5E0CBE01CE011289FD1102208F10101CA
:10F5000004F148000EF02AFF607801280DD0122087
:10F510002070E078C00703D0A07F88B301282FD0E7
:10F5200085F800B08DF804B0F0E384F800A027E07F
:10F5300011288FD1204600F0FEFF082804D0204675
:10F5400000F0F9FF132885D12869D8B16869C8B1DE
:10F5500004F17800102208F1010107460EF0FEFECA
:10F560002078082812D014202070E078C0070FD02F
:10F57000A07F022818D06178022912D00328CFD1A9
:10F580000420FDE300208DF80400F6E00920EBE7FD
:10F590000B202870296901204870206CC1E90107FF
:10F5A00092E208B1012870D10B202870296981F8F6
:10F5B00001A0606A4860206AC1E9020778E2206C15
:10F5C000E2780068C2F34402521ED04000F001000D
:10F5D00040F0800000E000200874E06A48617CE2AE
:10F5E0000746F9E31128D0D1204600F0A4FF0A28ED
:10F5F00002D1E078C00704D1204600F09CFF152816
:10F60000C3D1102208F1010104F148000EF0A6FE5A
:10F6100020780A2812D0162020701220287029691C
:10F620000920487004F15800486020308860103884
:10F63000C860206C0861ACE3C4EA01000B202070B4
:10F64000E4E22870D9E102289FD1204600F073FF40
:10F65000042804D3204600F06EFF082809D3204672
:10F6600000F069FF0E2890D3204600F064FF1228B6
:10F670008BD2A07F022888D18DF80490686A05900B
:10F6800098F801008DF80800FBE36CE20228AAD18B
:10F69000204600F050FF00286FD0204600F04BFFBE
:10F6A0000128F9D0204600F046FF0C28F4D00520B0
:10F6B0008DF8080098F801008DF8090065E7112819
:10F6C000FCD1002CFAD020781728F7D16178E06AB5
:10F6D000022912D05FF0000101EB4101182606EB70
:10F6E000C1011022405808F101010EF037FE05203B
:10F6F000696A00F013FF26700DE60121ECE70B2884
:10F70000DCD1002CDAD020781828D7D16178E06AD3
:10F7100002292CD05FF0000101EB4101102202EB25
:10F72000C1014158B8F8010008806078E16A0228F8
:10F7300020D0002000EB4002142000EBC20009584A
:10F74000404650F8032F0A60406848600520696A07
:10F7500000F0E4FE6078022810D04FF00000204452
:10F76000407A20F001000CD14FF001010BE04FF086
:10F770000101D1E74FF00100DCE77FE24FF001002B
:10F78000EDE74FF000012144487279E3112895D14B
:10F79000002C93D02078192890D16078E16A022853
:10F7A00011D0002000EB40021C2000EBC200102210
:10F7B000085808F101010EF0D1FD0520696A00F03A
:10F7C000ADFE1A20F5E00120ECE7082898D1002CC6
:10F7D00098D020781A2893D1E06A98F8012001780F
:10F7E00062F347010170E16AD8F8022041F8012F65
:10F7F000B8F8060088800520696A00F08FFE6078FE
:10F80000022807D04FF000002044407A20F0020187
:10F810002BD033E04FF00100F6E7204441722FE394
:10F820001128B4D1002CB4D020781B28AFD1617836
:10F83000E06A02291CD0002101EB4101202202EBE9
:10F84000C1011022405808F101010EF087FD05208A
:10F85000696A00F063FE607802280CD04FF0000067
:10F860002044407A20F0040108D14FF00100D4E791
:10F870004FF00101E0E74FF00100F1E74FF0000029
:10F88000CBE785F81CA0FAE33078012884D11C224C
:10F8900004F11C0071680EF0A6FDE079C10894F82F
:10F8A0003B0001EAD001E07861F30000E070217FC5
:10F8B000F1BB217803290AD0C0073FF4F9AD03203A
:10F8C00028708DF804B0686A059041209EE3607F3F
:10F8D000A17888423FF694AD02272771E17920464E
:10F8E00021F0E001E171617A21F0F0016172A17A09
:10F8F00021F0F001A172FFF77CFC2F708DF804B0AD
:10F90000686A05908DF808A0F2E33078112888D154
:10F910008DF804A0696A0591B1680391ADF808A05B
:10F9200008466168016021898180A17A817100E0C7
:10F930006AE004202070A4E230781128A6D18DF866
:10F9400004A0686A0590301D02AB07C883E8070071
:10F950004120ADF8080008460C210170A88CD6F8AB
:10F960000C8080B24027D4F82090FFF7F1FB41468D
:10F970004FF008084A463B46CDF80080FFF72FF8C5
:10F98000002101A8FFF70AFCE07820F03E00801C6F
:10F99000E0702078052801D00F200AE0A07F002821
:10F9A0003FF4C3AD0128FBD003287DD184F800804B
:10F9B000B1E42070AFE430780328A8D17068016802
:10F9C000A1664068E0660520287035E23178032999
:10F9D0009DD171680A68226749686167216C51B9D5
:10F9E000A17F19B1012901D0062029E185F800A0E5
:10F9F0002064606401E085F800A00327F3E3317818
:10FA0000022984D1317909B1297737E1A17F02290F
:10FA100010D00329EFD16178012910D0A17994F891
:10FA20003A2001290FD02064E178C90713D0012AB8
:10FA30000ED010E0B0680028E7D020640BE0A27977
:10FA400094F83A10EDE7B1680029DED02164EBE7C5
:10FA5000F0680028D9D06064CDE78DF804B0696AF9
:10FA60000591E1785846C90709D06178022903D188
:10FA7000A17F29B1012903D0A17F032900D008204B
:10FA8000287012E230781128BFD1B06828620920AE
:10FA90002870E0782969C0070FD081F801A0206A9A
:10FAA0004860606A886000E0ABE004F16800C8600C
:10FAB000A07F02287FF48FAD81E501204870206C83
:10FAC000486004F16800886004F13800C860201DB7
:10FAD0000861206B4861606B88611FE2E1783078D3
:10FAE000C90701D0062100E00A2188428DD1207883
:10FAF000072817D084F800908DF804A0686A059054
:10FB0000286A0390ADF80890032100F8011B102229
:10FB100071680EF023FC002101A8FFF73FFB0020D5
:10FB20002862C2E408202070E6E730781128ABD1C3
:10FB30008DF804A0686A0590B0680390ADF808904D
:10FB4000042100F8011B102204F168010EF006FCEC
:10FB5000002101A8FFF722FB2078092801D01320FB
:10FB600027E784F800B016E0E1783078C90701D0C3
:10FB7000062100E00A21884286D1102204F14800C3
:10FB800071680EF0BFFB10B104202877A2E3207843
:10FB900009283FF4C5AC0C2053E5E078C10735D007
:10FBA000A17F012902D002291BD02CE00D20287052
:10FBB000296981F801B06078012809D0206A48607D
:10FBC000606A886004F16800C8601030086104E56C
:10FBD000606A4860206A886004F17800C860103864
:10FBE000F4E7C0F3440114290DD24FF0006101EB9A
:10FBF000B0104FEAB060E0706078012801D01020AA
:10FC000055E40620D5E6607801288AD00E2018E554
:10FC1000307809288BD185F800B010208DF80400C9
:10FC2000686A059070680290002101A8FFF7B6FA93
:10FC3000E9E7E078C00706D0A07F01281FD10F2098
:10FC400028700420F8E015202870296902204870E7
:10FC5000206C48606078012805D004F17800886045
:10FC60001038C8605AE104F1680088601030F8E785
:10FC700030780228CED1307908B1287728E31020D7
:10FC800028700F20D8E030781328F7D185F800903D
:10FC900029690820487070684860607801280DD094
:10FCA00004F1680088601030C860206B0861606BE8
:10FCB000486104F158008861A06A21E004F17800ED
:10FCC00088601038F0E730780728D7D160780128AD
:10FCD0001AD1A078A16A0A18C0F1100110460EF0DE
:10FCE000B4FB1220287029690920487004F15800DB
:10FCF0004860203088601038C860206C086141E09E
:10FD0000C861E06A086209E11320C9E0CBE03078FD
:10FD10000828B3D1102204F1480071680EF0F2FAFD
:10FD200008B10B2031E720780B28EDD02046FFF7F3
:10FD300060FAA078A16A0A18C0F1100110460EF00E
:10FD400084FB1620287008208DF80400686A05904E
:10FD5000002049E03078112890D1B0682862142042
:10FD6000287029690920487004F158004860103053
:10FD700088601030C860606C08616078012800E01D
:10FD80009EE006D004F139004861206B8861606B09
:10FD9000B6E7601D4861606B8861206BB0E7307822
:10FDA000082892D18DF804A0686A0590286A03900B
:10FDB000ADF808900D2100F8011B102271680EF0BB
:10FDC000CDFA002101A8FFF7E9F900202862617847
:10FDD000012902D01520ECE569E2162129700821DD
:10FDE0008DF80410696A05910290A0788DF80C00D6
:10FDF0007EE130780B288CD116202870607802289C
:10FE000002D12046FFF7F5F9A07871680A18C0F111
:10FE1000100110460EF019FB08208DF80400686AE6
:10FE200005907068E0E730780F2895D1E079C00739
:10FE30007BD01720287009208DF80400686A05908F
:10FE400056E13078102887D11422311D04F11C00AE
:10FE50000EF0C9FAE16A208DA1F80900E16AA078E4
:10FE6000C871E179E26A01F003011172E16A627A14
:10FE70000A73E16AA07A81F824006078012876D0BC
:10FE8000B3E13EE26078022801D0012000E00020CA
:10FE90002044407AC0070BD0E078C00708D1192071
:10FEA00028708DF804B0686A05908DF808901FE1FD
:10FEB0001E2071E63078112874D1B06828621A20AB
:10FEC00028700520B8E7307803286BD16078E26AA3
:10FED000022801D0012000E0002000EB40011420A6
:10FEE00000EBC1015158726813680B6052684A6098
:10FEF0001B212970D5E9041205234B70636A4B60FE
:10FF00006778E36A022F01D0012700E0002707EBA2
:10FF1000470700EBC7001858C1E90202686A486247
:10FF2000069800F024FBFFF75BBB87E130780E28D2
:10FF300038D16078E26A022801D0012000E0002078
:10FF400000EB4000102101EBC000022310580932E1
:10FF500071680CF0E9FD1C202870296904204870A4
:10FF6000206A4860E06A09308860F84879E65AE11A
:10FF700030780D2816D16178E06A022901D001217C
:10FF800000E0002101EB4101182707EBC101A27835
:10FF9000405871680EF0E2F96178E06A022902D0F7
:10FFA000012101E0A9E0002101EB410107EBC101C2
:10FFB0004058A1780844C1F110010EF046FA8DF8BE
:10FFC00004A0686A0590286A0390ADF8089006219D
:10FFD00001706278E16A022A01D0012200E0002269
:10FFE00002EB420207EBC202401C895810220EF0BD
:10FFF000B5F9002101A8FFF7D1F8002028621D20E3
:020000040001F9
:1000000028708DF804B0686A05900B208DF8080000
:100010006EE03078112870D18DF804A0686A0590E0
:10002000B06803900B20ADF80800039880F800A09A
:100030006278E16A022A01D0012200E0002202EB8C
:100040004202102303EBC20289580988A0F801106C
:100050006178E26A022901D0012100E0002101EB70
:100060004103142101EBC30151580A6840F8032FE2
:1000700049684160002101A8FFF790F818E729E1DD
:100080006078022801D0012000E000202044407A5E
:10009000800701D51F2003E721207DE53078112856
:1000A0002BD18DF804A0686A0590B0680390ADF874
:1000B0000890082707706178E26A022901D00121BF
:1000C00000E0002101EB41031C2101EBC301401CB6
:1000D000515810220EF042F9002101A8FFF75EF8F6
:1000E000202028708DF804B0686A05908DF808709B
:1000F000314601A8FFF752F815E775E0307811286E
:1001000072D18DF804A0686A0590B0680390082049
:10011000ADF80800039809210170E16909784908E0
:100120004170E16951F8012FC0F802208988C1802F
:10013000002101A8FFF732F8AEE76078022801D06D
:10014000012100E000212144497A490701D52220FC
:10015000A6E6012849D068E03078112844D1B0687B
:10016000286223202870296904204870206A48608A
:10017000E06A09308860764873E530780D2833D11D
:100180006178E06A022901D0012100E0002101EB41
:100190004101202707EBC1011022405871680EF081
:1001A000DDF88DF804A0686A0590286A0390ADF820
:1001B000089080F800B06278E16A022A01D001223A
:1001C00000E0002202EB420207EBC202401C895809
:1001D00010220EF0C3F8002101A8FEF7DFFF002077
:1001E00028626078B5E791E037E02420D4E46078B5
:1001F00002280BD000202044407AC10702D0E178C9
:10020000C90705D0810705D51920A9E40120F2E727
:100210001720A5E4400701D51B20A1E41C20207075
:100220006078012801D01820B6E42720B4E4282003
:1002300028700B2000E63078122849D12920ABE441
:100240002078012844D00C2842D02046FEF7EFFF4A
:100250000C208DF80400686A059039E030784FF082
:100260002608112805D012203070032785F8008059
:100270004CE08DF804A0686A0590B06803900220F5
:10028000ADF80800039805210170297F4170002115
:1002900001A8FEF783FF0B208DF80400686A059023
:1002A000314601A8FEF77AFF074685F80080012F46
:1002B0000ED02BE001208DF80400686A0590042020
:1002C0008DF80800287F8DF809000020287712E0BB
:1002D000287F80B11D202070252028708DF804B063
:1002E000686A059002208DF80800314601A8FEF7E3
:1002F00055FF07460AE00CB1FE2020709DF804006F
:1003000020B1002101A8FEF749FF0AE409B03846F0
:10031000BDE8F08F2DE9F04F0C4601274E690978B2
:1003200085B09046BA464FF00209072021B1012955
:100330004ED002291FD1C8E0217901290AD0022913
:1003400015D0032910D0042915D11BE0BCEA010007
:10035000FE2F0000707801280CD10620616A02F09F
:1003600067FB002807D11AE01D20307017E0717874
:10037000022901D0052796E031780C2927D18DF884
:1003800004000EE03078011F042902D30E38032840
:100390001DD2B07F02281AD12089022817D38DF8E8
:1003A000049084F800A020899DF80410884203D2AC
:1003B0000A208DF800003FE01121083488F8001071
:1003C00094E80E00C8E901120327C8F80C306AE06F
:1003D00098F80010112966D18DF80000616A049127
:1003E000D8F80850029521794FF00B0B012906D05F
:1003F000022929D0032911D0042954D15AE0ADF89B
:10040000049085F800B0207E4F4600F01F00687011
:1004100000216846FEF7C2FE377043E0ADF8049055
:1004200005202870207E68704E4600216846FEF741
:10043000B5FE26708DF800B0606A049041466846AB
:10044000FEF7ACFE07462EE0ADF8040085F800A0EC
:10045000207F6870607F00F00100A870A07F00F02E
:100460001F00E870E17F2971C0071FD094F82000B9
:1004700000F00F00687194F8210000F00F00A871DF
:1004800000216846FEF78AFE2868B063A888B08716
:10049000A87986F83E00A069407870772879B07016
:1004A0000D2030700027384605B031E70020A871D4
:1004B0006871E5E7ADF804900E202870207E687022
:1004C00000216846FEF76AFEECE7FE2030708DF8EA
:1004D00000A0606A049004208DF80400207E8DF84E
:1004E0000500EDE700B50023012285B005280FD0F7
:1004F00006280BD102208DF8002004918DF804000D
:100500008DF8053000216846FEF748FE05B000BDB5
:100510008DF8002004918DF80420F1E770B50C46A9
:10052000054602F0ACFA21462846BDE87040782323
:10053000002202F007BA08B1007870470C2070471B
:1005400070B50C0005784FF000010CD021702146E9
:10055000F3F745F974482178405D884201D10320C2
:1005600070BD022070BDF3F73AF9002070BD027B28
:10057000032A05D000220A704B780B2B02D003E02F
:10058000042070470A770A62027B9300521C0273B0
:10059000C15003207047F0B585B00F4605460124D1
:1005A000287B05EB800050F8046C7078411E0C2904
:1005B0000AD25D493A46123101EB8000314650F8CB
:1005C000043C2846984704460CB1012C11D1287BE5
:1005D000401E10F0FF00287301D00324E0E70D2037
:1005E0008DF80000706A0490002101966846FFF7BC
:1005F000A7FF032CD4D005B02046F0BD70B515463A
:100600000A46044629461046FFF7C5FF064674B160
:100610002078FE280BD1207E30B10020287029469A
:1006200004F10C00FFF7B7FF2046FEF700FE30464E
:1006300070BD704770B50E46044688210DF027FF47
:100640000225012E03D0022E04D0052070BD01200A
:10065000607000E065702046FEF7E9FDA577002098
:1006600070BD28B1027E1AB10A4600F10C01C5E73F
:100670000120704730B5044687B00D46062002F0D1
:10068000FEF92946052002F0FAF92078FE2806D066
:1006900000208DF8000069462046FFF7E2FF07B012
:1006A00030BD7FB50E4600218DF80C1041780B2926
:1006B00003D00C2903D0002405E0846900E04469DC
:1006C0000CB1217E91B16D4601462846FFF74FFFE0
:1006D000032809D1324629462046FFF78FFF9DF8AF
:1006E0000C10002900D0042004B070BD04F10C05EA
:1006F000EAE710B590B00C4607900B480421801E25
:1007000008900A488DF8191009900F92694606A8BA
:10071000FFF7C7FF002805D11022204601990DF0F0
:100720001DFE002010B010BDDEE90100BCEA010092
:1007300070B50D46040011D085B1210128460DF099
:1007400084FE10224E4928460DF008FE4C48012137
:100750000838018044804560002070BD012070BDD4
:1007600070B5474E00240546083E10E07068AA7B2D
:1007700000EB0410817B914208D1C17BEA7B91425E
:1007800004D10C2229460DF0BDFD30B1641C308827
:100790008442EBDB4FF0FF3070BD204670BD70B57A
:1007A0000D46060006D02DB1FFF7DAFF002803DB67
:1007B000401C14E0102070BD314C083C2088628839
:1007C000411C914201D9042070BD6168102201EBE7
:1007D000001031460DF0C2FD2088401C208028709A
:1007E000002070BD70B514460D0018D0BCB10021BA
:1007F000A170022802D0102811D105E0288870B11C
:100800000121A170108008E02846FFF7A9FF002809
:1008100005DB401CA070A8892080002070BD01204D
:1008200070BD70B5054614460E000BD00020307028
:10083000A878012808D005D91149A1F108010A8832
:1008400090420AD9012070BD24B1287820702888F0
:10085000000A5070022008700FE064B1496810224D
:1008600001EB0011204610390DF078FD2878207337
:100870002888000A607310203070002070BD0000CE
:100880006C0000202DE9F041FE4C207EE17D884285
:1008900008BFBDE8F0810126FB4D0027E07D215C0B
:1008A00001EB810205EB8200037C052B18D0037C51
:1008B000062B23D0037C072B34D0437C002B08BFAE
:1008C000FFDF29D04774E07D16280EBF0020E07DB1
:1008D000401CE075481CC0B255F8222007211AE0E0
:1008E0000674E07D16281ABFE07D401C0020E075EC
:1008F000481CC0B255F8222002210CE00674E07DAD
:1009000016281ABFE07D401C0020E075481C55F8F1
:100910002220C0B203219047207EE17D8842BDD1D4
:10092000BDE8F0810674E07D16281ABFE07D401C0A
:100930000020E075481CC0B255F822200821EAE7E3
:1009400070B5D24D0C2085F82900A5F53B70002428
:1009500080F8CD4180F8CC4100F5F4700476C47580
:1009600005F12C000CF03CFFA5F58E70047585F8A0
:100970002B40601E2C60A86085F8254085F8224039
:1009800085F8234085F8244085F82140C048A5F12A
:10099000E80104704470002000EB800201EB820249
:1009A0001474401CC0B20B28F6D30120F8F730FEB7
:1009B0000020F8F72DFE012085F82600F9F7E0FA6F
:1009C000B448F9F7ECFAB44C2070B448F9F7E7FAF8
:1009D0006070BDE87040F8F7AFBD10B5F8F7DAFD0C
:1009E000AD4C2078F9F7F4FA6078F9F7F1FAA74CF2
:1009F00094F82800002808BF10BDF8F7DAFF00209F
:100A000084F8280010BD0B20704770B59F4C94F8F7
:100A1000260000281CBFFFDF70BD94F82B000028C3
:100A200008BFFFDFF8F79FFE62690025811A6FF0AB
:100A30007F43B1F5800F24BFA2EB000CBCF5800F03
:100A40000DD38B4203D2991A0844411C07E0634539
:100A500028BFFFDF05D2181A1044401C414200296C
:100A600000DBFFDF012684F8266084F82B5094F821
:100A700029100420844A01EB810102EB81010874F2
:100A8000A068B0F1FF3F04D0B01EA0600120F8F7CD
:100A9000BFFD0020F8F7BCFDF8F7A0FD25600DF0C4
:100AA00043F8F8F7E9FE7E48056005604FF0E02165
:100AB0004FF40040C1F88002F2F73FFA7448007822
:100AC000022804D0032805D194F8230010B184F83B
:100AD000226001E084F82250BDE87040F8F7B0BE13
:100AE000034669490B2000BF00EB800201EB820244
:100AF00012F8042C22B1401E10F0FF00F4D1704710
:100B000000EB800201EB8201012241F8143C01F864
:100B1000042C7047012804D0032808BF002926D0E0
:100B200000E021B3594B4FF0000C83F821C0584A24
:100B30000028907014BF022882F803C00BD0072948
:100B400015D2DFE801F01404060C0E1012001B2071
:100B500000E03A20D070012083F82100704758202F
:100B6000F8E77720F6E79620F4E7B520F2E70020D3
:100B70007047474810B54078F8F787FE80B210BD3F
:100B800030B5421E4049002500EB800001EB800497
:100B90000A2A02D814F8040C00B9FFDF14F8040C78
:100BA000012818BFFFDF04F8045C30BD70B53D4C70
:100BB00094F8CD0194F8CC1188420CBF0125002592
:100BC000F8F7D1FDF8F761FE94F8CD1194F8CC2137
:100BD00091420CBF01210021A942E9D170BD30B57D
:100BE0000D46314A44190021101A71EB010038BF3B
:100BF000FFDF2E488542C8BFFFDF2D488542B8BFC2
:100C0000FFDF2C488442A8BF2B4804DA002CAABF7F
:100C10002046284830BD201830BD70B51A4900EB79
:100C2000800001EB8004254A54F8101D607A0028EA
:100C300052F8202011440CBF04200220084420F068
:100C40007F40F8F722FE94F90850174A4419002112
:100C5000101A71EB010038BFFFDF14488542C8BF8E
:100C6000FFDF13488542B8BFFFDF12488442A8BFA8
:100C7000114804DA002CAABF20460E4870BD201887
:100C800070BD0000E808002004090020EC090020E5
:100C90007E000020F12701007C0000208508010073
:100CA00000F5004000070020FF7F841E0020A10700
:100CB00000E05EF80080841E00807BE120EA0100F5
:100CC0002DE9F04F0646FF4885B00068C005C00D0D
:100CD00011D0103840B20028B8BF00F00F0000F16A
:100CE000E020B4BF90F8140D90F80004400908BF4C
:100CF0004FF0010A01D04FF0000A307800281FBFE2
:100D00000128002005B0BDE8F08F307900280CBF25
:100D100004210221EC4ABAF1000F52F8200001EB45
:100D2000000903D1E949002081F827006C4602AA96
:100D30002146B068F8F7B6FD9DF90820F068211D3E
:100D400010440122C01C1F28B8BF019208DB03AA6F
:100D5000F8F7A8FD9DF80C0010B10198401C019017
:100D6000DDE900100844401D20F07F400190A1EB18
:100D7000090020F07F40009070798DF80A000098FB
:100D80000390F8F7F0FC009A019B121A181AD04948
:100D900022F07F4220F07F40B2F5800F26D28142C0
:100DA00024D3CA4890F82950009CCA4F181B20F041
:100DB0007F486FF07F40001BAB4604900C2D24D081
:100DC00005EB850007EB80026FF07F435068011B45
:100DD000B1F5800F12D3A4EB000CBCF5800F0DD33E
:100DE0008B4205D204990844411C07E000205FE0D3
:100DF000634509D2191A0819401C41420029BCBF99
:100E0000AB46957CDADB00E0FFDF5D4525D00BEBE0
:100E10008B0007EB80026FF07F4091680B1BB3F5EE
:100E2000800F12D3A4EB010CBCF5800F0DD39842B8
:100E300003D204980844431C07E0604528BFFFDF45
:100E40000BD2431A1819401C4342002B05DD9DF8B4
:100E50000A00927B904228BF0C460C2D18BF9DF8CB
:100E60000A1010D005EB850007EB80004268121BCA
:100E700022F07F42424506D2827B914228BF84689D
:100E8000857C0C2DEED10098A04205D004EB080023
:100E900020F07F400094019000990398814206D091
:100EA00001EB090020F07F40F8F7EFFCB060012073
:100EB000864991F82710002904BF05B0BDE8F08FDE
:100EC000BAF1000F3FF42EAF05B0BDE8F08F2DE969
:100ED000F04F064687B00C467F480CF089FC4FF077
:100EE0000108002835D07D4F387D002818BFFFDF6E
:100EF0003E742079794D05F10C0228726079687290
:100F00002946A068F8F7CEFC95F90C000F2804DDFF
:100F10001F3828732868401C286095F90C00E16888
:100F20002E1D0844C01C1F28B8BFC6F8008009DB6E
:100F30006A463146F8F7B6FC9DF8000010B13068FB
:100F4000401C30602078A87287F8148007B0BDE894
:100F5000F08F634D95F8CD0116281ED095F8CD0180
:100F600095F8CC11401C884200D1FFDF554800683D
:100F7000C005C00D1AD0103841B20029BDBF01F024
:100F80000F0000F1E02090F8140D01F1E020A8BF5F
:100F900090F80004400909D104E095F8CC0100283C
:100FA000E4D1E2E72078002818BFFFDF4C4890F832
:100FB000CD1101EB810100EB81000674207801283E
:100FC00000F04A81022843D0454890F8CD1101EB4A
:100FD000810100EB8105207928726079687205F142
:100FE0000C022946A068F8F75DFC95F90C000F2863
:100FF00004DD1F3828732868401C286095F90C1000
:10100000E0682E1D0844C01C1F28B8BFC6F8008029
:1010100009DB6A463146F8F745FC9DF8000010B13F
:101020003068401C30602078A8722D4890F8CD11AF
:1010300016290EBF002190F8CD11491C80F8CD1162
:1010400025480CF0EBFB07B0BDE8F04FF8F7F8BB14
:10105000234890F8CD1101AA01EB810100EB810733
:101060006946E068F8F71EFC9DF904000F28CCBF24
:101070000120002000993D1D08440190A068C01C7B
:101080001F28B8BFC5F8008009DB6A462946F8F773
:1010900009FC9DF8000010B12868401C286002205F
:1010A000B872607978722079387200280CBF0421F8
:1010B0000221054A52F82000014403917A68481D34
:1010C00010440FE004ED00E020EA0100EC090020EC
:1010D000FFFF3F0004090020180A0020D00800206C
:1010E000000700200199009008440399401A0590D8
:1010F000FD4C002084F82700F8F735FB3860019993
:101100008046084420F07F40F86094F829000C28BD
:101110007ED0214691F8290000EB8002A1F1E80081
:1011200000EB82025668009A324422F07F4202921B
:1011300097F809B091F829503446111B21F07F4AE5
:101140006FF07F41891BA94604910C2D23D0E748FD
:1011500005EB850100EB81026FF07F435068011BB6
:10116000B1F5800F24BFA4EB000CBCF5800F0BD3AE
:101170008B4203D204990844411C05E0634509D21F
:10118000191A0819401C41420029BCBFA946957C88
:10119000DBDB00E0FFDF4D4524D0D44809EB8901BB
:1011A00000EB81036FF07F429868011BB1F5800F5F
:1011B00012D3A4EB000CBCF5800F0DD38A4203D2EE
:1011C00004990144491C07E0624528BFFFDF09D2AA
:1011D000121A1119491C4942002903DD997B8B45DC
:1011E00028BF04460C2D18BFC04910D005EB850060
:1011F00001EB80004268121B22F07F42524506D26A
:10120000827B934528BF8468857C0C2DEED100E05D
:101210001BE0A64205D004EB0A0020F07F402646E2
:101220000290029AA6EB080020F07F40A2EB080291
:10123000059922F07F42B0F5800F06D2914204D387
:101240000398304420F07F403860A74890F827008A
:1012500000287FF44DAFE8E6A548851915F8010C84
:10126000002818BFFFDF05F8018CADE60020F8F775
:10127000BFB90120F8F7BCB99E48007870472DE946
:10128000F0419A4E00274FF00308012506F1E804CB
:1012900050B301285BD0022800F0E98003281CBF6E
:1012A000FFDFBDE8F08194F829000C2808BFFFDFBC
:1012B00084F8267084F82B5094F8290000EB800005
:1012C00006EB800080F81080F8F7C1FA94F8290046
:1012D00094F82910401CC0B201EB810156F821207E
:1012E000BDE8F0410521104794F829000C2808BFFB
:1012F000FFDF84F8267084F82B5094F8290000EB67
:10130000800006EB800080F81080F8F7A0FA207FBC
:10131000002818BFFFDF84F825500020F8F778F97F
:10132000A168B1F1FF3F04D0012300221846F8F76D
:10133000B3F994F8290094F82910401CC0B201EBCD
:10134000810156F82120BDE8F0410121104794F8B1
:1013500029000C2808BFFFDF84F8267084F82B5082
:1013600094F8290000EB800006EB800080F81080E4
:10137000F8F76DFA0120F8F74BF994F825000028EA
:101380001CBFA068B0F1FF3F0DD094F8290094F87D
:101390002910401CC0B201EB810156F82120BDE8A4
:1013A000F04106211047207F012815D002281FD0C8
:1013B000032833D004281CBFFFDFBDE8F08194F878
:1013C000201060680123411A00221846F8F764F9DA
:1013D00094F82800B8BB37E094F8240028B184F8CA
:1013E0002470F8F73BFA84F823502777BDE8F081A2
:1013F00094F8280018B9F8F7B3FA84F8285094F84C
:10140000290094F82910401CC0B201EB810156F864
:101410002120002190472777BDE8F081217B60687B
:101420000123411A00221846F8F736F994F82400EF
:1014300028B184F82470F8F711FA84F823500220B8
:101440002077BDE8F08103E0F8F78AFA84F82850A5
:1014500094F8290094F82910401CC0B201EB8101D6
:1014600056F82120002190472577BDE8F0812148DA
:101470000078BDE8F041F8F7B1BD10B51A4C94F80A
:1014800029000C2808BFFFDF94F8290094F82910E0
:10149000401CC0B2154A01EB810152F82120BDE881
:1014A0001040042110472DE9F84F8046087C104C6D
:1014B000401EC6B20D46A05D01281DD0022825D0D1
:1014C000297CDFF828A0481EC4B204EB84020AEB92
:1014D0008206371D0A2821D801EB81000AEB800023
:1014E00010F8040CD8B919E0EC0900200409002018
:1014F000E00900207C000020A87A012814BF022007
:101500000020A05518BFBDE8F88FD9E7A87A0128B8
:1015100018BFFFDF0021A972A155D1E7FFDF307CA2
:10152000DFF8289407280BD11720009099F817208E
:1015300009F11803494620460BF0A6FE012030743D
:10154000307C012804D0A87A012818BFFFDF02D020
:10155000A87A01284BD1FE4B307C022818D099F88C
:101560001800162872D099F8180099F81710401C26
:10157000884200D1FFDF0120707499F8180009F843
:10158000004099F81800162800F09E8100F093B9E9
:10159000F04A92F829000146A04207D0014600EB2C
:1015A000810003EB8000807CA042F7D192F829C033
:1015B00084450CD192F8291001EB810103EB8101E4
:1015C000897C82F82910012182F82A1009E000EBB9
:1015D000800203EB820201EB810103EB8101927C2B
:1015E0008A7400EB800003EB80000C218174287A60
:1015F000D949002851F820A02968A1EB0A010CBFA5
:1016000004200220081A20F07F423A60D5E9000148
:10161000084420F07F407860A87A022818BF287B11
:101620001ED038727868401D20F07F407860687A5C
:10163000B872287A06257872032872D2002870D0F2
:1016400000F022FE00286DD0A1E0FFE799F8170016
:10165000002890D18EE700BF89F81800BDE8F88F08
:10166000287A00280CBF0420022000EB0A036868D7
:10167000591D00EB010BB9484078504503D9B549D5
:1016800091F8231011B10BF1060003E0A0EB0A0062
:101690005844801DAF4991F829C0BCF10C0F25D0EA
:1016A00091F829C00CEB8C0EA1F1E80C0CEB8E0C20
:1016B000DCF804C0624519D0DFF8A4C291F8291003
:1016C00001EB8102A24901EB82014A688968A2EB21
:1016D000080222F07F42A1EB080121F07F419042F5
:1016E00098BFB2F5800F9DD28C459BD34044A0EBB0
:1016F0000B0020F07F4139601944E86821F07F41F8
:101700000A1A6FF07F4CB2F5800F24BF431AB3F56D
:10171000800F11D3944506D2ACEB00000844421C64
:101720000AE034E02FE09C4528BFFFDF1DD2ACEB80
:1017300001010844401C4242002A16DD0520307495
:1017400099F81800162819D099F8180099F8171068
:10175000401C884200D1FFDF99F8180009F80040CA
:1017600099F8180016287BD0A5E03868ABF1050180
:10177000084420F07F407860002052E799F8170075
:101780000028E9D1E7E7CAF138054FF0320A73487B
:101790000178012918BF03290AD14078504507D99B
:1017A0006C4991F82310002904BFA0EB0A000544FE
:1017B0006B4B3868A0EB0802786822F07F41A0EB01
:1017C000080020F07F4C8D4298BFB1F5800F1BD2EE
:1017D000634519D35F4991F829300C2B30D091F82B
:1017E00029504FF00C0BDA46594905EB850301EB04
:1017F0008303D3F808C0ACEB080C944531D8AB4652
:101800009D7C0C2DF0D193E00520307499F81800E0
:10181000162810D099F8180099F81710401C884223
:1018200000D1FFDF99F8180009F8004099F8180076
:10183000162849D03FE099F817000028F2D1F0E7C8
:101840000220307491F829000C2818BF91F8290063
:10185000B07481F82940012081F82A00BDE8F88F92
:1018600032E00C2D1CBFAA46002261D00AEB8A038D
:1018700001EB8303D3F804C0ACEB080C84452CD2F5
:101880009A7B97F80AC0944520D30520307499F8C4
:101890001800162813D099F8180099F81710401C52
:1018A000884200D1FFDF99F8180009F8004099F844
:1018B0001800162808D099F81800401CCCE699F8B2
:1018C00017000028EFD1EDE70020C5E693F812A03D
:1018D0000122BAF10C0FC9D103E0002A08BFAA46C1
:1018E00026D02F461A4807EB870100EB8108062215
:1018F00088F8102099F81800162838D099F81800A0
:10190000411C99F81700814200D1FFDF99F81800B7
:1019100009F8007099F8180016280EBF002099F8F1
:101920001800401C89F8180098F81270BA45D9D1EF
:101930000220074F307407F1E80090F82910A942FF
:101940001AD186F812A080F829400BE0E8080020A0
:1019500004090020EC09002020EA01007E0000209C
:10196000FFFF3F00012180F82A10BDE8F88F99F8A9
:1019700017000028CAD1C8E70C2D0CD0BBF10C0F02
:1019800008BFFFDF0BEB8B0007EB8000847486F849
:1019900012A0BDE8F88FBBF10C0F08BFFFDF0BEB07
:1019A0008B0007EB800084740C20B074BDE8F88FC6
:1019B0002DE9F04F83B0F7F7D6FE05464FF00C0B3C
:1019C000FE4C94F829100026A4F1E8094FF0010814
:1019D0000C292FD094F82920214602EB820209EB32
:1019E0008202127C042A25D091F8292002EB82027F
:1019F00009EB8202127C032A04BF03B0BDE8F08F1A
:101A00002A4620696169801A491BED4B20F07F400E
:101A100021F07F4106283CBF03B0BDE8F08FB0F550
:101A2000800F24BF03B0BDE8F08F8B423CBF03B0F2
:101A3000BDE8F08FA068B0F1FF3F18BFFFDF84F86A
:101A4000256094F82900DF4F0C2809D094F829006C
:101A500000EB800009EB8000007C042808D01AE02D
:101A600094F82100B8B1F8787870B878387012E03E
:101A700094F829B00BEB8B0009EB800080F8108004
:101A800094F8290000EB800009EB8000807C84F84A
:101A9000290084F82A80DFF830A39AF8CD019AF85B
:101AA000CC11884219D000BF9AF8CC0100EB80001D
:101AB0000AEB80012846FFF7F6FC9AF8CC011628BD
:101AC0000EBF00209AF8CC01401C8AF8CC019AF88D
:101AD000CD019AF8CC118842E6D1DFF8F0A29AF84D
:101AE000140028B151462846FFF7DDFC8AF814603F
:101AF000BBF10C0F06D00BEB8B0009EB8000017CD7
:101B000001292BD094F829000C2800F0ED8094F8DE
:101B10002A00002800F0F78084F82A6094F8290051
:101B200000EB8001AA4800EB8102A0F50173D2E925
:101B30000101D268C3F80423C3E9BF01607E002815
:101B40000CBF4FF004094FF00209A249022811F816
:101B50002010217318BF012834D123E0072101741C
:101B6000DFF874A29AF81800162816D09AF8180010
:101B70009AF81710401C884200D1FFDF9AF818002D
:101B80000AF800B09AF8180016280EBF00209AF83C
:101B90001800401C8AF81800B4E79AF817000028CB
:101BA000ECD1EAE720690844421B22F07F42382A40
:101BB00008D903213238617620F07F40206132203D
:101BC000207309E0322907D294F8280058B9F7F7B2
:101BD000C7FE84F8288006E094F8280018B1F7F7CB
:101BE000E8FE84F828607B7884F8203094F80CA014
:101BF00038780621A3EB0A02012818BF032804D174
:101C000084F82480002AC8BF911D94F822B0BBF14B
:101C1000000F18BF891C206901905044484420F0EF
:101C20007F406060BAF1000F14BF022000202077CF
:101C300094F82400002808BFBBF1000F37D060489B
:101C40000090D4F810E0D4F814C0AEEB050E2EF0DE
:101C50007F4EACEB050C20462CF07F4C714598BFB5
:101C6000BEF5800F1FD2009961451CD3002A0FDDFD
:101C70000199BAF1000FA1EB020101611944494435
:101C800021F07F4141600CBF0121032121770EE04B
:101C900004DA002B0CBF02210421F7E7BBF1000F8F
:101CA00008BFFFDF03E080F8246084F82260207F13
:101CB00040B12069012300EB090100221846F7F723
:101CC000EBFC02E00120F7F7A3FC94F829000123C4
:101CD00000EB80013E4800EB8100616890F90C2028
:101CE0000020F7F7D9FC0EE00120F7F791FC002067
:101CF000F7F78EFCF7F772FC94F8280018B1F7F7A5
:101D000058FE84F8286094F8220028B1F7F7A6FD61
:101D100084F8236084F8226094F8210018B1F878E0
:101D20007870B878387094F8240030B184F8236063
:101D30003878002808BF84F824602748017EC07DD9
:101D4000814203D025484078F8F748F984F8278085
:101D500003B0BDE8F08F70B5184C054682B094F81A
:101D600029000C2808BFFFDF94F8290000EB800051
:101D7000174E06EB8000007C032818BFFFDFA06829
:101D8000B0F1FF3F18BFFFDF94F8290001AA00EB74
:101D9000800006EB8000694690F90C002844F7F7B4
:101DA00081FD9DF904000F28CCBF0120002000997F
:101DB00008446168084420F07F4111E0EC090020EC
:101DC000FFFF3F007E00002000070020D008002019
:101DD0000409002020EA0100E80800207C0000201F
:101DE000A16094F82500002804BF02B070BD012353
:101DF00002B00022BDE870401846F7F74DBC744AA7
:101E00000B1A02F1010CB3EB9C0F3CBF1846704754
:101E100010B5441AB4EB9C0F3CBF184610BD9A4253
:101E200003D2101A0844401C10BD94429EBFFFDF2D
:101E3000002010BD511A0844401C404210BD01232F
:101E4000002201460220F7F727BC0220F7F7E0BB8B
:101E5000F7F789BC2DE9F0415E4C054682B094F855
:101E60002B00002808BFFFDF642D50D35A48002202
:101E7000401B72EB02004AD3584890F8CD1190F8FD
:101E8000CC01814243D15648007D00283FD194F8CF
:101E90002900DFF8508100EB800008EB8006206805
:101EA00001AA28446946F7F7FDFC9DF904000028C3
:101EB00002DD0098401C0090B168009872680F180D
:101EC000BA1A22F07F42B2F5800F20D2B27C0C2ADF
:101ED00009D002EB820208EB82025268511A21F00B
:101EE0007F41814213D3A068B0F1FF3F05D00120AC
:101EF000F7F78EFB4FF0FF30A06020682844206089
:101F000027F07F40606102B00120BDE8F08102B09F
:101F10000020BDE8F0812DE9F8430646401EC7B217
:101F2000304807EB870100EB8104207C002808BFC4
:101F3000FFDF2A4A92F8CC1192F8CD0181420DD0F0
:101F400001EB810302EB83031B7CB34210D0162903
:101F50000CBF0021491CC9B28142F1D120484FF089
:101F6000170800F11805017D29B3007CB04222D189
:101F70000020BDE8F883207C05281FBF207C0628B0
:101F8000207C07280AD184F81090CDF80080EA7DE3
:101F900005F11803144938460BF076F9607C68B1F6
:101FA0006674CDF80080EA7D05F118030E493846C5
:101FB0000BF06AF902E04FF001090026207C0128AD
:101FC00004BF607C0028D6D10120BDE8F883000062
:101FD000FF7F841EEC090020FF1FA10700070020DF
:101FE000D008002004090020E8080020F0B5734A5A
:101FF000D2F80032724D002401212E7856B9714E6C
:102000003460704F03263F1D3E606E4F04260C3730
:102010003E602970C2F80042D1601160694C4834BA
:10202000D16425688542FBD35160D160C2F800328B
:10203000F0BD2DE9F041044680074FF000054FF058
:10204000010604D560480560066024F00204E0043F
:102050004FF0FF3705D55D484660C0F8087324F49B
:102060008054600003D55A48056024F08044E005A0
:102070000FD55248C0F80052C0F8087351490D609E
:10208000091D0D604F4A04210C321160066124F4D1
:102090008074A00409D54F484660C0F80052C0F8CB
:1020A00008734D48056024F40054C4F38030C4F331
:1020B000C031884200D0FFDF14F4404F14D04748AD
:1020C0004660C0F8087346488660C0F80052C0F801
:1020D000087344490D600A1D16608660C0F80873D5
:1020E0000D60166024F4404420050AD53E48466041
:1020F0008660C0F80873C0F848733C48056024F453
:1021000000640BF0EBFC3A48044200D0FFDFBDE86E
:10211000F08170B5202500224FEA020320FA02F177
:10212000C90719D051B201F01F060124B4404E096D
:10213000B60006F1E026C6F88041C6F880420029C4
:1021400006DA01F00F0101F1E02181F8143D03E00E
:1021500001F1E02181F80034521CAA42DED370BDA7
:1021600070B5174C0D466060FFF763FF6068FFF7BE
:10217000D0FF2846F7F7D1FC0BF0E0F800F0D5F8D7
:102180000BF0ACFC0BF0F7FBF7F7FAFEBDE8704084
:102190000BF082B910B50A4C6068FFF74AFF60681F
:1021A000FFF7B7FF0BF09AFCF7F77BFD00206060AC
:1021B00010BD03484068704702207047008000400F
:1021C0008400002004850040FC1F004000C0004047
:1021D00004E5014000D0004004D5004000E000408C
:1021E00000F0004000F5004000B0004008B500409D
:1021F000FEFF0FFC70B51F490A68BAB100231D46E7
:1022000001244A68521C4A60092A00D34D600E79A5
:1022100004FA06F20E6816420AD072B60B689343AF
:102220000B6062B649680160002070BD052070BD7A
:102230005B1C092BE5D3FFDFF8E74FF0E0214FF4FB
:102240008000C1F800027047EFF3108111F0010F18
:1022500072B64FF0010202FA00F20648036842EA41
:102260000302026000D162B6E7E702480021016084
:10227000416070478C000020012081070860704792
:10228000012081074860704712480068C00700D0ED
:10229000012070470F48001F0068C00700D00120D0
